:020000040000FA
:040000006FD00400B9
:101000006F00900F00000000000000009020002002
:10101000A4220020A9BDF9F55C23002000000000F7
:10102000000000005C230020902000200000000051
:101030000000000090200020000000009020002010
:101040000000000090200020902000209020002030
:101050009020002090200020682800209020002070
:10106000000000009020002090200020EC230020B1
:1010700090200020C22300209020002090200020FB
:101080009020002090200020902000209020002020
:101090009020002001A04111B7170040985F3AC688
:1010A000945F3247E39CE6FE3245410182800111A4
:1010B00013078008F337078093F787083EC20100C3
:1010C0000100B7170040930570052380B70413068D
:1010D00080FA2380C7040100010083C6B70493F699
:1010E000F60DA385D704238007049246F3A6068055
:1010F0000100010093760502D5CEF336078093F602
:10110000860836C4010001002380B7042380C70489
:1011100001000100B70614007D89558D88C70100C4
:1011200001000100010023800704A246F3A6068007
:101130000100010073370780137787083AC6010062
:1011400001002380B7042380C704010001000100CF
:1011500001003727004093061005A303D7802380A2
:101160000704B247F3A70780010001009307800836
:10117000F3B7078093F787083ECE01000100B71749
:101180000040130770052380E704130780FA2380CB
:10119000E7040100010003C7B70413670708A3852C
:1011A000E70423800704F247F3A70780010001004A
:1011B0000561828093760504BDC6F336078093F6F9
:1011C000860836C8010001002380B7042380C704C5
:1011D00001000100B7061400938606047D89558D31
:1011E00088C7010001000100010023800704C246F6
:1011F000F3A6068001000100733707801377870884
:101200003ACA010001002380B7042380C70401000B
:1012100001003727004093062005A303D7802380D1
:101220000704D24781B773370780137787083ACC12
:10123000010001002380B7042380C70401000100DE
:1012400098471367070C98C723800704E24719BF24
:101250000111814601468145114506CE5D24930763
:101260008008F3B7078093F787083EC601000100A6
:10127000B7170040130770052380E704130780FAAF
:101280002380E7040100010003C767041367170008
:101290002383E70423800704B247F3A707800100F4
:1012A0000100F2400561828041118146014681457D
:1012B0001145812C13078008F337078093F78708BF
:1012C0003EC401000100B7170040130670052380DB
:1012D000C704930680FA2380D70401000100FD555E
:1012E0002396B70223800704A245F3A505800100D9
:1012F000010073370780137787083AC601000100A1
:101300002380C7042380D7040100010003C76704BA
:10131000136717002383E70423800704B247F3A76A
:1013200007800100010001A0BD473305F50201005F
:101330007D1575FD8280411122C426C206C6AA848D
:10134000014463179400B2402244924441018280D8
:1013500005041305803E4204C13F4180DDB7000013
:101360009305000273A04580824573901534924026
:101370002242B2424243D2436244F2440255925561
:101380002256B2564257D2576258F25806499649E9
:10139000264AB64A464BD64B664CF64C065D965DE1
:1013A000265EB65E465FD65F09617300203041114C
:1013B000B7170040985F3AC6945F3247E39CE6FE59
:1013C000324541018280B71700401307000323888C
:1013D000E702854717170000232EF782730020309D
:1013E000411122C406C6370400201C408297F5BF75
:1013F00037370040834747009146BD8B6389D7004C
:1014000099466394D700834757407300203097165E
:10141000000083C6A6809387160017060000230FDE
:10142000F67E0347870093870164B6972380E70021
:10143000B7E70400BC4F094689451705000003457E
:10144000F5788297D9B72303048015472303E480F6
:1014500001002302A480828083076480E3CE07FE1C
:1014600023030480828083076480E3CE07FE034564
:101470004480828083076480E3CE07FE2302A48039
:101480008280411126C44AC24EC006C61377F50BAE
:10149000AD47AA892E8995446306F700194565373B
:1014A000653F8D444E854537FD59FD1463983401E1
:1014B000B240A24412498249410182801355090178
:1014C0001375F50F453F2209CDB7011126CC06CE85
:1014D000B704080051371545BD37713769372AC63B
:1014E000A53F32459377150089EB136515001375F9
:1014F000F50FF240E24405618280FD14E9FC0145EC
:10150000CDBF397126DC4ADA4ED852D656D45AD2DB
:101510005ED006DE62CE66CCB7E700E07D5783AAD8
:10152000070022C603AA470023A0E71823A2E71852
:10153000B7170040130770052380E704130780FAEC
:101540002380E70483C74704930B75FFB684E20743
:1015500093FBFB0F8546AA892E8B328937240040E6
:10156000E187015763FA76016308D50089461307BE
:1015700000026313D5000157D98F93F7F70FB71CFB
:1015800000402382FC0411472303E4801305F00F7D
:101590005D3D094CD135636D7C11B7050700DA95C7
:1015A00037870700795563F2E504B3879500636ECA
:1015B000F702370B0800A94733EB65016399F90679
:1015C00089E48144513D26850DA0DA850945553DC4
:1015D00005090345F9FFFD14050B693D81C49377A7
:1015E000FB0FFDF7DD3569FD7D55B717004013078B
:1015F00070052380E704130780FA2380E70403C7FC
:101600004704418B2382E704F250B7E700E023A0B0
:10161000571123A24711E25432445259C259325A47
:10162000A25A125B825B724CE24C21618280A54718
:101630006395F90685691309F00FB3069900B37431
:101640002B01B6941349F9FFB3749900856B337974
:101650006901416B9387F9FFB3F7270199E363FCB5
:10166000340193D94900C147E3E637FF99BF0569C3
:10167000C1697D19D9B71305800D63886901130508
:1016800000026384790113051008CA85DD3B353DEE
:1016900021DD4E99B3843441D9B7DA852D45D53350
:1016A000CA94E30099F205097D3BA30FA9FED5BFBB
:1016B0009387F9FF93F7F70F6361FC0C83C71C0452
:1016C00013073008631FF70437070800636BEB0448
:1016D000B3079B00B706100063F5D704334BEB004C
:1016E00089476393F9068980D549E38C04ECDA8550
:1016F0000945413B11090327C9FF91472320E48095
:1017000003076480E34E07FE23033481FD17EDFBDE
:10171000FD14110B81C49377FB0FE9FF7D3371F545
:10172000E1B5B717004003C75704B70708001377A0
:10173000070219E3B78707007955E378FBEA330717
:101740009B00E3FFE7F855B58547E382F9F2DA85B8
:101750002D45053B9389F4FFE38504E6293393F790
:10176000390091EB83260480032709009307490081
:10177000E39AE6E43E89CE84F1BFB5476396F9006B
:101780001305900BC93135BDB1471305B00AE38B82
:10179000F9FE99476391F904B7050800B365BB00EA
:1017A0002D45C53181448D4BA1497539639674012E
:1017B000832704802320F9008504E39834FF8327DE
:1017C000048013172B01635507002312F900D5BBC2
:1017D0002322F900FDB39D476399F9028145130562
:1017E000B0044531BD442320090023220900FD59DE
:1017F0009D3993F77400CA9703C70700FD14398D0C
:101800002380A700E39634FF6DBBA1476392F904E0
:101810006D398144630D0B008D479304C003630849
:10182000FB009304000563048B01930440041375CB
:10183000C507E30895D819453931393905452131AE
:1018400026850D3909453D314931E31C05D669BB73
:1018500091476399F90013056006F536F53E1305C7
:1018600090090DB7E38F09D4F154A9BB197106C2D1
:1018700012C416C61AC81ECA22CC26CE2AD02ED210
:1018800032D436D63AD83EDA42DC46DECAC0CEC2C0
:10189000D2C4D6C6DAC8DECAE2CCE6CEEAD0EED2F0
:1018A000F2D4F6D6FAD8FEDA97050000938505360D
:1018B0008841E700050092402242B2424243D243AF
:1018C0006244F244025592552256B2564257D257BC
:1018D0006258F25806499649264AB64A464BD64BB4
:1018E000664CF64C065D965D265EB65E465FD65F3C
:1018F00009617300203000009721002093818170DE
:1019000017510020130101F017F5FFFF1305C56FF4
:10191000970500209385056F171600201306C6FD56
:1019200063FAC5008322050023A055001105910527
:10193000E3EAC5FE17550000130585FF9715002043
:10194000938585FB171600201306C62963FAC50088
:101950008322050023A0550011059105E3EAC5FE89
:101960001715002013050528938581766377B50048
:10197000232005001105E36DB5FEFD42739002BC06
:101980008D4273904280B7220000938282887390C8
:101990000230970200209382E26693E23200739055
:1019A0005230972200009382C230739012346FC07D
:1019B0002465730020303D432A876373C302937705
:1019C000F700BDEFADE5937606FF3D8ABA960CC3EE
:1019D0004CC30CC74CC74107E36BD7FE11E28280B2
:1019E000B306C3408A069702000096966780A60059
:1019F0002307B700A306B7002306B700A305B70067
:101A00002305B700A304B7002304B700A303B7005E
:101A10002303B700A302B7002302B700A301B70056
:101A20002301B700A300B7002300B700828093F51D
:101A3000F50F93968500D58D93960501D58D61B7E9
:101A4000939627009702000096968682E78086FA92
:101A50009680C1171D8F3E96E374C3F8A5B7B717DC
:101A6000004003C777051377E70FA38BE70413073D
:101A700000F8A38DE7043D47238CE70413075003C8
:101A8000A38CE70403C7A7051377D70F238DE704BB
:101A90008280B717004003C7E7020D894111137711
:101AA000C70F498F93068008F3B6068093F6860821
:101AB00036C601000100930670052380D704930603
:101AC00080FA2380D704010001002387E7022380E6
:101AD0000704B247F3A7078001000100410182809B
:101AE00041112A83014E930E407E130F0019930F6C
:101AF000400663E56E129308001913034006B3789D
:101B00001503854E0D4FA14F337365020D891335B3
:101B1000150063EFBE121308F6FF7946729842086B
:101B2000135808013307C70213D61700BE073297B0
:101B30006146B3F6C60213068070B386C6023697B6
:101B4000A166F58F42075D8FB716004083C7F60286
:101B500093F70708A303F1000346710083C7F60259
:101B600093F70708E394C7FE83477100B716004058
:101B700093F7F70F6388071293078008F3B707807E
:101B800093F787083EC401000100B7170040930691
:101B900070052380D704930680FA2380D7040100C0
:101BA000010023AA070383C6170393E60608A38848
:101BB000D70223800704A247F3A707800100010092
:101BC0001166B71700407D16D45BC85F9385470345
:101BD000A98EF18EF5FA93068008F3B6068093F687
:101BE000860836C601000100930670052380D704DD
:101BF000930680FA2380D7040100010098C103C72F
:101C0000170313670704A388E70223800704B2477A
:101C1000F3A7078001000100410182807D13336832
:101C2000E3039308E016630E08003368F303930898
:101C3000D016630808009378330093B8180093888F
:101C4000D81633081E01131E0801135E0E0155B588
:101C50006393E503054863860800014863030300B6
:101C60002A8871087298FD15131E0801C205135EBB
:101C70000E01C18179BD13F8150063F4BF00790826
:101C8000D5B713381800E5BF83C7F60293F70708E6
:101C9000A303F1000346710083C7F60293F7070818
:101CA000E394C7FE8347710093F7F70FF1DFE9B5BF
:101CB00031714AD966CB06DF22DD26DB4ED752D5FD
:101CC00056D35AD15ECF62CD6AC96EC7AA8C02D8EC
:101CD000EF00901C2A8993078008F3B7078093F7D9
:101CE00087083EDA01000100B717004013077005AE
:101CF0002380E704130780FA2380E7040100010032
:101D000003C7F7021377770FA387E70203C7F7022A
:101D100013678700A387E70223800704D257F3A73E
:101D20000780010001000545AD33130780C133472B
:101D3000E902116A93070AE893065002BD69930B02
:101D4000A004814A014B13048008930470057D1A96
:101D5000B347F9023307D7023EC0FD873ECC9387D5
:101D600009A69309803E3347F7023AC27D873AC4F9
:101D7000334739038549B399990193D93940B3065B
:101D8000D702B30B7703B3C6F602B3CBFB0236C65A
:101D9000FD8636C893D6FB4136CEB7460F009386F4
:101DA00006243349D9028566938606FAB3969601CE
:101DB000B389E902130760553309D902930600106D
:101DC000B389E9023349D902B3C9F902931639003C
:101DD00036CA37190040FD8636D0930D090493D7D3
:101DE000F9413ED2F336048093F6860836DC0100D2
:101DF0000100930770052380FD00930680FA23807D
:101E0000DD00010001008346390593F6860FA30922
:101E1000D9048346390593E61600A309D904238023
:101E20000D00E256F3A6068001000100130C80FAB3
:101E3000116DF336048093F6860836DE010001004A
:101E4000930770052380FD0023808D0101000100B0
:101E500083463905216693E60602A309D904835611
:101E60000905B3E6A6012318D90483560905D18EC6
:101E70002318D90423800D00F256F3A60680010032
:101E800001008346390593F60602638A0618034665
:101E90003905218A6DDE0818EF00100473360480BE
:101EA00013768608B2C20100010023809D002380C2
:101EB0008D0101000100B717004003C637051376F6
:101EC000F60DA389C70403C6370513660602A38966
:101ED000C704835609052166B3E6A6012318D90471
:101EE00083560905D18E2318D90423800D00964608
:101EF000F3A60680010001008346390593F6060229
:101F00006386061483463905A18AEDFE97000020FA
:101F1000E7806018AA8636D497000020E780A017D3
:101F2000A256E30AD5FE835609054255B3E6A6013B
:101F30002318D904C12783463905A18AEDDE03564B
:101F400009058346290582473376CA00B306DA02BB
:101F500093D5F641B296B388F640E24733B8C6004F
:101F60002E983308F840A247B3B616013308D8407C
:101F700063C70701631DF800924763FA1701C24760
:101F8000634DF80E63950701B24763E8F80E894682
:101F900063E7660FF2469315180013D3F8015E86C7
:101FA00013951800B365B30042D646D4EF206061A4
:101FB0003258050B137BFB0F63470001631208388F
:101FC000A258638F083613081500B336A800B695DB
:101FD00013D6F5013298B336C800AE9613581800E0
:101FE000FE06B3E606017336048013768608B2C691
:101FF0000100010023809D0023808D01010001006C
:102000000356C902B296C206C1822316D9022380A2
:102010000D00B646F3A606800100010019BDF33697
:10202000048093F68608B6C00100010023809D005D
:1020300023808D01010001008346390593E60602E5
:10204000A309D90423800D00864605BDF33604801C
:1020500093F68608B6C40100010023809D0023800A
:102060008D01010001008346390593E60602A309AC
:10207000D90423800D00A646A5BDE30D0BF0F33671
:10208000048093F68608B6C801000100930680FA22
:1020900023809D002380DD00010001008346390577
:1020A00093F5FC0F93F6860FA309D90483463905EF
:1020B000CD8EA309D90423800D00C646F3A6068061
:1020C00001000100130580FA03463905930639051E
:1020D0001D8A631496297336048013768608B2CC61
:1020E00001000100130680FA23809D002380CD00AB
:1020F0000100010003C606001376F60D2380C6001A
:1021000003C60600136606022380C600835609052F
:102110001166D18E2318D904835609052166D18E04
:102120002318D90423800D00E646F3A6068001009B
:102130000100130680FA8346390593F60602638888
:10214000062483463905130C3905A18AFDDA0818DF
:102150006123F336048093F68608B6D001000100AF
:10216000930680FA23809D002380DD00010001009A
:1021700083460C00116693F6F60D2300DC008346BF
:102180000C0093E606022300DC0083560905D18E7D
:102190002318D904835609052166D18E2318D90442
:1021A00023800D008656F3A6068001000100130669
:1021B00080FA8346390593F6060263850620834636
:1021C0003905A18AEDFE97000020E780C0EC2A8C3B
:1021D00097000020E78020ECE30C85FF835609057B
:1021E00011664255D18E2318D90429238346390517
:1021F00013063905A18AFDDAF336048093F68608C2
:10220000B6D401000100930680FA23809D0023804C
:10221000DD00010001008346060093F6F60D230061
:10222000D60023800D00A656F3A60680010001000B
:102230008356090503462905D247B376DA003306EB
:10224000CA021305800C9355F6413696330DF640BD
:102250008257333CD6002E9C3336A601330CFC400B
:10226000330CCC403308850392564E86B335A50314
:102270003305A503C295EF20C03463468001631E79
:102280000C16630C0D16130615003335A6002E959B
:102290009356F5013696B335D600AA959396F50177
:1022A00005828585D18E6346B000639D051A638BD8
:1022B000061A0356C90215823305D6003336C50007
:1022C000B2956348B000639105241306F00F637D57
:1022D000A622894663F3561593078008F3B7078053
:1022E00093F78708BED60100010037170040930717
:1022F00070052300F704930780FA2300F704010018
:1023000001008356C70289678117D58FC207C18331
:102310002316F70223000704B657F3A7078001002E
:102320000100FA506A54DA544A59BA592A5A9A5A48
:102330000A5BFA4B6A4CDA4C4A4DBA4D29618280ED
:102340001308F5FF3335A800FD152E951356F5013A
:102350003298B336C800AA9651B1F336048093F68A
:102360008608B6CA0100010023809D002380AD00CD
:102370000100010083463905CD8EA309D9042380CD
:102380000D00D646F3A606800100010035BBF336EA
:10239000048093F68608B6CE0100010023809D00DC
:1023A0002380CD00010001008346390593E6060233
:1023B000A309D90423800D00F646F3A60680010088
:1023C000010095BBF336048093F68608B6D201006F
:1023D000010023809D002380CD0001000100834681
:1023E000390593E60602A309D90423800D00965609
:1023F000F3A60680010001006DBB9306F5FF33B51F
:10240000A600FD152E959355F501AE96B3B5B60011
:10241000AA951396F501858269B5F336048093F683
:102420008608B6D801000100930680FA23809D003B
:102430002380DD00010001008356C90205660116F4
:1024400093F6F60FD18EC206C1822316D9022380DD
:102450000D00C656F3A6068001000100850A93FA16
:10246000FA0F49B233E6B60045C20356C902330536
:10247000D0403338A000B305B040B3850541158284
:102480006345B000D1E16371A608894663F0560543
:1024900093078008F3B7078093F78708BEDA010037
:1024A0000100B7170040130770052380E7041307E6
:1024B00080FA2380E7040100010003D7C7027D8B67
:1024C0002396E70223800704D65781BDF3360480A4
:1024D00093F68608B6DC01000100930680FA23809B
:1024E0009D002380DD00010001008356C9020566BE
:1024F000011693F6F60FD18EC206C1822316D902B9
:1025000023800D00E656B9B793078008F3B707801C
:1025100093F78708BEDE01000100371700409307DC
:1025200070052300F704930780FA2300F7040100E5
:1025300001000356C70293975600B297C207C183A2
:102540002316F70223000704F657C1BB914763EE39
:10255000B702174700001307A7C98A05BA959C411F
:10256000BA978287B717004003A7470B1345F5FFBB
:10257000698F23AAE70A03A7070B698F23A8E70A35
:1025800003A7070A798D23A0A70A8280B717004006
:1025900083A6470B1347F5FFF98E23AAD70A83A614
:1025A000070B558D23A8A70A83A6070A758F23A0BA
:1025B000E70A8280B717004003A7470B498F23AA79
:1025C000E70A03A7070B1345F5FF45BFB717004000
:1025D00083A6470B1347F5FF758F23AAE70A03A7C6
:1025E000070A598D4DB7B717004003A7470B498F0E
:1025F000EDB7914763EEB70217470000130787C096
:102600008A05BA959C41BA978287B717004003A7FD
:10261000470D1345F5FF698F23AAE70C03A7070DA4
:10262000698F23A8E70C03A7070C798D23A0A70CBB
:102630008280B717004083A6470D1347F5FFF98E38
:1026400023AAD70C83A6070D558D23A8A70C83A614
:10265000070C758F23A0E70C8280B717004003A7F3
:10266000470D498F23AAE70C03A7070D1345F5FF74
:1026700045BFB717004083A6470D1347F5FF758F79
:1026800023AAE70C03A7070C598D4DB7B7170040D5
:1026900003A7470D498FEDB7B7170040884742059C
:1026A00041819377050491EB9377F5013755E80164
:1026B000130505803345F50282809377050C1307D7
:1026C00000046397E7009377F50137459C1CCDB76D
:1026D0002165130505D0828037E700E01C43544391
:1026E000A183E206D58F1CC1FD572320F7182322B2
:1026F000F718828013178500B7E700E023A0E710E2
:10270000618123A2A7108280B7F700E08847CC47F9
:102710008280814737370040A14663C4C7003285B5
:1027200082800345B740E38EA6FE3385F50003455E
:10273000050085072304A740CDB79707002093879E
:1027400067479C43138781763E95636EE500174784
:102750000020130727EB6368A70017070020232B2F
:10276000A7443E858280FD57EDBF411122C406C6B5
:102770002A841D372947B307E502B2408D83B3D7BA
:10278000870222449507B3D7E70237370040C207D4
:10279000C1832316F7004101828071654111130541
:1027A000052006C6D937B7370040130770F82381D4
:1027B000E7000D47A381E70013070004A380E700AB
:1027C00005472387E700B240410182803737004048
:1027D000834727001A0593F7F703C98F93F7F70F7D
:1027E0002301F7008280B737004003C7170019C9DB
:1027F000D98DA380B70003C7070013678700238024
:10280000E700828093C5F5FFF98DA380B700828031
:10281000B73700402147B736004091E1828003C6B8
:10282000B700E30CC7FE05050346F5FFFD15C2051D
:102830002384C600C181D5B7411122C406C62A84AB
:10284000A13D2947B307E502B2408D83B3D7870284
:1028500022449507B3D7E70237370040C207C18348
:102860002316F7404101828071654111130505204F
:1028700006C6D937B7370040130770F82381E74001
:102880000D47A381E74013070004A380E7400547F5
:102890002387E740B24041018280CC41411106C606
:1028A000328503C6150083C5050022064D8E4206FB
:1028B0008D654186138875A2630C0611634BC804AD
:1028C000138845A26300060D634AC800938535A2AC
:1028D0006301B6082390060029464DA0138855A22F
:1028E0006305060D938565A2E316B6FE8D451D466C
:1028F00063E6E5081146198E63F3C7003E86B7E725
:1029000004002390C600FC47974500009385C5FC52
:102910009DA0138895A263030611634E060D1388CC
:10292000A5A263000613938505A5E315B6FA99459C
:102930001D4663E5E504198E63F3C7003E86B7E7DD
:1029400004002390C600FC479705002093850527C7
:102950001DA09D451D4663E3E5022146198E63F3E4
:10296000C7003E86B7E70400FC472390C6009705E2
:10297000002093852527BA9582970146B24032857B
:1029800041018280AD451D46E3EAE5FE3146198EE0
:1029900063F3C7003E86B7E704002390C600FC47F8
:1029A0009745000093850589F9B7B1451D46E3E7D2
:1029B000E5FC3546198E63F3C7003E86B7E7040091
:1029C0002390C600FC47974500009385A58765B70F
:1029D0008D451D46E3E4E5FA1146198E63F3C70001
:1029E0003E86B7E704002390C600FC4797450000E9
:1029F000938545EF49B78D451D46E3E1E5F811465E
:102A0000198E63F3C7003E86B7E704002390C60023
:102A1000FC47974500009385A5EEB1BFA5451D462F
:102A2000E3EEE5F42946198E63F3C7003E86B7E767
:102A300004002390C600FC47973500009385C57EAF
:102A40001DBFB5451D46E3EBE5F23946198E63F32C
:102A5000C7003E86B7E704002390C600FC479735C1
:102A600000009385657B01BFB7E7040003A307134C
:102A700097060020938646F14146A545170500209C
:102A8000130585E702832D4559EF03C50500094766
:102A90006317E50803A84500411106C6034718005F
:102AA00032850346080022074168518F930828FEAB
:102AB0006308170363E9E80005186303070523901B
:102AC000060029451DA8130648FE630BC70215180A
:102AD000E31707FF15463E87637BF602154705A8F7
:102AE0003E8691C30546B7E70400FC472390C60025
:102AF0004206CC45418282970145B2404101828025
:102B00001306700F3E876374F6001307700FB7E764
:102B100004002390E600FC4713160701D9BF239059
:102B20000600054582808280416779176304E504C9
:102B3000411122C406C685472A84639FF500B7E782
:102B4000040022852244B24003A387139705002086
:102B50009385050A4101028389476399F500B7E728
:102B6000040083A7070B8545829771D9B2402244A0
:102B7000410182808280797122D452CC2E842A8AAB
:102B8000973500009385456E173500001305856F56
:102B900006D63AC626D24AD0B68432894ECEEF1037
:102BA000D05FA685173500001305C56EEF10F05EE7
:102BB0002945EF10D0628347840093F70702E1E7CD
:102BC000834904008947054532476396F908544014
:102BD00083C7160083C60600A207D58FC166138679
:102BE00016FE638CC7028D16638FD7068D6693869B
:102BF000269029456391D706B7E70400A2852254A1
:102C000003A34714B250F249A6864A869254025949
:102C10005285624A8547456102832D450DEF930732
:102C2000700F354563E99702B7E70400FC47484455
:102C30001306700FCA8582978149970700209387F2
:102C4000E7FB9C43014581CB9C4391C74E8526867B
:102C5000CA8582970145B250225492540259F249D2
:102C6000624A456182802D457DF79307700F354597
:102C7000E3E397FEB7E70400FC4748441306700FF0
:102C8000CA8582975DBF2145F9B7411122C437E457
:102C900004008327841326C2AA84416506C69705CB
:102CA00000209385E5F47D1582978327C40A1705D4
:102CB00000001305A5E78588829795C003230413B8
:102CC0002244B2409244970600209386A6DD4146F6
:102CD000C545170500201305E5CB41010283B2402D
:102CE0002244924401454101828019C59707002082
:102CF00023A6A7F001458280454582801147636A7B
:102D0000A70A973600009386E6540A0536951841BF
:102D1000411106C63697AE87B28502871307700F3A
:102D20006145639DE700B7E70400FC471306700F99
:102D300017050020130585F082970145B240410137
:102D4000828005476145E39BE7FEB7E70400FC4747
:102D5000054617050020130565E9F9BF1307700F35
:102D60006145E39DE7FCB7E70400FC471306700FDD
:102D700017050020130505FCC1B71307700F614547
:102D8000E39EE7FAB7E70400FC471306700F170548
:102D900000201305A5094DB715476145E390E7FAF3
:102DA000B7E70400FC47154617050020130585E426
:102DB00061B709458280411126C2B7E4040083A7A8
:102DC000C41322C44AC006C62E84970500209385EA
:102DD00025E22A898297058905C5970700209387F0
:102DE00067BB83D7A70BA28503A3440D2310F40070
:102DF0002244B24092444A8502490146410102837D
:102E0000B2402244924402494945410182809707D9
:102E10000020238707DE9707002023A507DEB717CA
:102E2000004003A7070CB706C0FFFD16758F23A04F
:102E3000E70C03A7070DB7064000558F23A8E70C42
:102E400003A7070C3D9B23A0E70C03A7070D1367FF
:102E5000070123A8E70C8280B717004003A5470CA1
:102E600083A7470C598113451500C18B058999E348
:102E7000136525009707002083C787D86380A702C2
:102E800097070020238EA7D611C9970700209387A4
:102E900067D703A307006303030002838280114501
:102EA0006FE01FE1411193962500AA852D4506C6C6
:102EB00097F0FF1FE780E064B24001454101828046
:102EC000011122CC06CE3714004026CA4AC84EC68D
:102ED00052C483447405034AB405834984050349F5
:102EE0009405EFE0DFB78347A40593F4F40F137A5A
:102EF000FA0F93E71700230DF40493F9F90F1379F0
:102F0000F90FB717004003C7A705058B6DFF03D561
:102F1000C705A38D4705238C3705A38C2705A38BF5
:102F20009704F2406244D2444249B249224A0561C0
:102F3000828041119397050122C406C626C2C1872B
:102F40002E8463DC0700B7E40400FC54829719C1A7
:102F5000BC5482972165218D3DA093F7150013C5C0
:102F6000150095E393F7250085C7FD35B7E7040005
:102F7000BC4F1306000A894517050020034505C903
:102F8000829713452400B24022449244410182803A
:102F90009397250163D50702B7E4040083A7C41EF5
:102FA0008297F53DBC4C37F60200130606E08965B2
:102FB00017050020034585C58297096569BF93976A
:102FC00015010145E3D107FC173500001305453312
:102FD000EF107031B7E70400BC4F13060064916531
:102FE00017050020034585C282971165ADB72D7185
:102FF000232A9110FD74E98C232C811023282111A0
:10300000232631112A84AE893289930600100A865C
:10301000A6852D45232E111097F0FF1FE780604EE7
:1030200013154401B7E70400FC4751810A051396C4
:103030002900CA850A958297A68585660146254599
:1030400097F0FF1FE780E04B0A86A68593060010E5
:10305000294597F0FF1FE780C04A8320C111032450
:10306000811183244111032901118329C1101561A4
:103070008280B7F7070003C70701411106C622C4C3
:1030800026C24AC0A547631AF7009537B2402244CA
:103090009244024901454101828013942500AA848B
:1030A0003289A286AA850146254597F0FF1FE78051
:1030B0004045A2864A86A685294597F0FF1FE780EE
:1030C0004044E9B71D71A2CC37E404005C5C485869
:1030D00086CE4946973500009385051E829701E903
:1030E000173500001305851EEF10F01F01A0B7F67D
:1030F00000E0795798CAFD57DCCA0567B7E700E0DA
:1031000023A0E7101306F00290C223A0E7180100E5
:103110000100370700201847130600048145970671
:10312000002023A3E6AE4157A38AE7403C440808A9
:103130008297970700209387E7F03EC8856713873B
:103140000760231AE1001D673ACC37070105130712
:1031500007103ACE9387B7D31307B00F2310E102BD
:103160002312F102054797F7FFFF9387275A2301A0
:10317000E1023ED817070000130707D397070000A6
:10318000938747D4B7F50700BAC23EDC17070000A3
:10319000130767EE970700009387A7D0814630009A
:1031A000E1051945BAC43EDE97F0FF1FE7806035A0
:1031B00018088147994630003E9603460600850769
:1031C0000507A30BC700E398D7FEC24791C7035773
:1031D000410185676373F70001A0B7E7040083A787
:1031E000470A08088297AA8501C917350000130508
:1031F000250FEF10807A01A0F64066442561828099
:10320000411126C2B7E4040083A7040806C622C4FD
:1032100017050000130525D2829717040020130418
:10322000E49E2300A4003128DD3603450400224437
:1032300003A38405B240924413060032896541011C
:103240000283797106D622D413078008F3370780EA
:1032500093F787083EC201000100B71700409305AD
:1032600070052380B704130680FA2380C704010089
:10327000010083C6F70293F6A60FA387D702238027
:1032800007049246F3A60680010001007337078009
:10329000137787083AC4010001002380B704238014
:1032A000C7040100010003C7F70213672700A387C3
:1032B000E70223800704A247F3A70780010001006B
:1032C0000545EFE00FFDE13E014781468147054698
:1032D00085451305407EEFE0BF8037E404003C44A1
:1032E0006800514681458297B707C0A83EC8B78796
:1032F000E803938707D03ECA97F7FF1F9387270BF2
:103300003EC67C5868008297B25022544561828044
:10331000011122CC37E404008327041A06CE8297D9
:10332000EF00B07D8547A307F100832744171306FC
:10333000F1008545130550308297173500001305BD
:1033400065FCEF10407AF240624405618280828021
:10335000411122C491462A8417060020130686CD07
:103360009D652D4506C697F0FF1FE7808019B7F7CA
:10337000070003C70701A5476313F70001A09306E1
:10338000001001469D65254597F0FF1FE7806017F7
:1033900097070020238087CA2244B240914617062F
:1033A0000020130626C99D652945410117F3FF1F1B
:1033B000670023155171CAD137E904008327C90476
:1033C000A2D52E8686D7A6D32E84AA8517050020DF
:1033D000130545B682979707002083C7A7B5130743
:1033E000700A638BE70E636CF7001307600A638251
:1033F000E704BE502E549E540E596D61828013070F
:10340000800A638AE7141307900AE394E7FE8D4766
:103410006309F41A97350000938585FA1735000083
:10342000130545E6EF10605717350000130585F6C4
:1034300015A08D476306F40297350000938545F883
:1034400017350000130505E4EF102055173500006F
:10345000130585EDEF1060542945EF10405851BF1A
:103460008547173500001305E5ED17F7FF1F230308
:10347000F77AEF104067B7750200B76602000146A1
:10348000054597F0FF1FE780C007930760F817070F
:1034900000202301F7AA97070020A38E07A893070F
:1034A0000026170700202329F7A8E577938707212F
:1034B000170700202314F7A8B145970700202380A1
:1034C00007A897070020A38CA7A6170500201305BF
:1034D00065A6EF10A00531BF914763E187029735DC
:1034E00000009385E5ED173500001305A5D9EF1011
:1034F000C04A173500001305E5E6A9BF9704002070
:1035000083C484A39707002083C7F7A2A204DD8C9D
:103510008327C9046D142286970500209385D5A1C1
:10352000280082978E0493160401B7750200C182A9
:103530003000A695094597F0FF1FE78080FC9307B0
:1035400070F8170700202307F79E9945970700207A
:10355000A384A79E9DBF914763E187029735000032
:10356000938505E6173500001305C5D1EF10E0423D
:1035700017350000130585E0F1BD9704002083C4D2
:10358000A49B9707002083C7179BA204DD8C832789
:10359000C9046D142286970500209385F5992800AB
:1035A00082978E0493160401B7750200C182300021
:1035B000A6950D4597F0FF1FE780A0F4930780F8CC
:1035C00049B717350000130525DEEF10C05113056C
:1035D000C01297F0FF1FE78000D60145EFF0CF8FB4
:1035E0000D45BD33294597F0FF1FE780C0D497F004
:1035F000FF1FE780E0C5F5BB41114AC097F6FF1FEA
:1036000083D6A661328917F6FF1F0356065C22C4D3
:1036100026C206C6AA842E84ED2E6306090297F7F9
:10362000FF1F83C7375F85C319CC97F7FF1F83C779
:10363000675E91EBA2852244B240024926859244FE
:1036400041016F00B06EB2402244924402494101F0
:1036500082808347550083454500173500001305D8
:10366000E5D8A207DD8D6F10403317350000130534
:10367000E5D66F1040478D4763F2B70A011126CA9D
:1036800006CE22CC0344350097F4FF1F83C4A45810
:10369000973500009385C5D6B337800017F7FF1F15
:1036A000230BF75609C497350000938525D61735A7
:1036B0000000130525D6EF10402E97F7FF1F83C794
:1036C0008755638397003D2C97F7FF1F83C7A75447
:1036D0009DC385472306F100B7E7040083A747177A
:1036E000700085451305503082971735000013058B
:1036F00065D3EF10403F9967938757EE2316F1008B
:10370000680085479145A30781002307F100EF007A
:10371000F061F2406244D244056182808280894730
:1037200063F2B708011122CC06CE26CA83442500D5
:1037300085472A846398F404914763F0B7040345EE
:1037400045008347340022055D8D97F7FF1F239EB8
:10375000A746A1269967938767EE2314F100834754
:10376000340023059100A305F100834744009545EB
:1037700028002306F100EF00705BF2406244D2445F
:1037800005618280FDF89967938767EE2314F10045
:1037900097F7FF1F83D76743A305F10023050100B7
:1037A000A183F1B782800111996722CCD51717F454
:1037B000FF1F130454462314F1008347040026CA54
:1037C00097F4FF1F938464452305F10083D7040019
:1037D00028009545A305F100A18306CE2306F1003C
:1037E000EF00D05403D604008345040017350000D1
:1037F0001305C5C4EF10601AF2406244D24405615B
:1038000082809D677971D9172316F10097F7FF1F02
:1038100083C7774006D62307F1008DCFB7E70400B2
:10382000FC47414697F5FF1F9385C56F1305F100CF
:1038300082976800CD45EF00704F97F5FF1F83C555
:10384000953D17350000130565C2EF100015B25005
:1038500045618280B7E70400BC47414681451305B6
:10386000F1008297F9B7B76702036971938757AA86
:103870003EC4856789072316F10097F7FF1F9387DA
:10388000973983C7070023248112A3070100230768
:10389000F10097F7FF1F9387473883D7070037E476
:1038A0000400232611122318F10097F7FF1F9387B6
:1038B000C73183D70700414648082319F1007C44EB
:1038C00097F5FF1F938505668297F1452800112221
:1038D0002312A1027C442C002810794682973C4494
:1038E000130561041306900D8145829730109305EE
:1038F000700F0145EFF08FC08320C11203248112A5
:1039000055618280B7C7A55A01119387C7333EC45A
:1039100097F7FF1F83C727303EC6B7F7070003C7D7
:10392000070106CE22CCA5476313F70001A011645E
:10393000930504F0930600100146254597F0FF1FFC
:10394000E78020BC3000930504F0A146294597F09C
:10395000FF1FE78000BB97F5FF1F83C5C52B1735F9
:103960000000130525BBEF104003F24062440561DF
:10397000828001119165A1463000938505F02D45A7
:1039800006CE97F0FF1FE780C0B72247B7C7A55AFA
:103990009387C7336312F702B2451735000013054A
:1039A00025AFB335B00097F7FF1F2386B726EF008A
:1039B000D07EF240056182808145173500001305F5
:1039C00065AF97F7FF1F23880724EF00107D1D3F89
:1039D000CDB7C16769768146FD17050613970601C5
:1039E00041836364B7003E8582803307D500034777
:1039F0000700B98F214713F8170085836305080076
:103A0000B18FC207C1837D171377F70F6DF7850656
:103A1000F1B749C1A547054763FFB70683471500BE
:103A2000034705003168A207D98F13978700A18348
:103A3000D98FC207C1831308C8550547639D070581
:103A4000411106C622C426C203442500914763FDE6
:103A50008702930754006399F502A301C5002182F0
:103A60002302C5009304340091C6A302D500A182AD
:103A70002303D5002A84A685A93F26942300A40009
:103A80002181A300A4000147B240224492443A8518
:103A90004101828005473A858280B7C7A55A011146
:103AA0009387E7343EC42AC6B7F7070003C7070168
:103AB00006CE22CC26CAA5476313F70001A0916465
:103AC0002A84938504EE930600100146254597F05D
:103AD000FF1FE78000A33000A146938504EE29452F
:103AE00097F0FF1FE780E0A1A285173500001305BE
:103AF00065A4EF00906A853BF2406244D2440561C0
:103B0000828001119165A1463000938505EE2D4517
:103B100006CE97F0FF1FE780C09E2247B7C7A55A81
:103B20009387E7346313F702B24517350000130596
:103B3000659A97F7FF1F239AB708C205C181EF0066
:103B4000D0651533F24005618280D147D1451735E4
:103B500000001305259A17F7FF1F2318F706EF003B
:103B6000D06317F5FF1F03554506053FE1BF41111F
:103B700026C206C622C493F71500AE848DCBAD676E
:103B8000371700409387A7AA1CC3B7E70400BC4FB0
:103B900013060019854517F5FF1F0345F5028297A7
:103BA00013C51400B240224492444101828093F72D
:103BB0002500C5CB97F5FF1F83C50506854793C430
:103BC000240063E5B70299C997F7FF1F83C79704DD
:103BD00091C7854513850164EF00501513950401C5
:103BE00097F7FF1F238A070241816DBF03C4016459
:103BF00083C7116422045D8CAD679387B755630A50
:103C0000F40463ED8700A9679387A7556307F4045D
:103C100097F7FF1F83C717008DC719A8B167938750
:103C2000C755630CF400B5679387D755E312F4FECC
:103C300013850164EF00900F29A0054613850164E8
:103C4000653AA2851735000013058590EF00F05402
:103C500071B713850164F53AEDB71385016431340A
:103C6000CDB793F74500014595DF173500001305E3
:103C7000658FEF005067EF00101213C544001DB7A9
:103C80001567B71700401307575598C3D8439D666B
:103C9000558FD8C3D843FD76758FD8C3D8431367E3
:103CA000F70FD8C335671307C7CC98C3828041117B
:103CB0001305800406C622C426C2371400404AC039
:103CC00097E0FF1FE780A03E8327840A8D451305F8
:103CD000002093E707202324F40AEFE03F87B7E4AE
:103CE0000400EFE07FB8C8581309840C1304C40C17
:103CF000EF00705F8327C4FF8545414593E70708C0
:103D0000232EF4FEEFE0FF8E8D4513050008EFE053
:103D10005F8EEFE09FA80145EFE05FAB854505456D
:103D2000894717F7FF1F230BF7EEEFE0DFAB3707ED
:103D30000004B7E700E023A0E710EFF0AFB8EFF022
:103D40002FCC05397D3BEFF0AFDC8D450D65EFE005
:103D50005F8A1385017485671CC589672320250147
:103D600040C12326250100C95CC983A7841E829710
:103D700083A70408170500001305A5DF829797F7AE
:103D8000FF1FA383A7E4BC4C1306006485458297FC
:103D9000C53D97E0FF1FE780A06401119307700FF6
:103DA0002316F10006CE97F7FF1F83C7F7E78DE7CD
:103DB000B7E7040083A7870D17F6FF1F034646E108
:103DC0006C0017F5FF1F035565E682973335A00099
:103DD00097F7FF1FA38AA7E4F24005618280411193
:103DE0009397050122C406C626C2C1872E8463D4D8
:103DF0000702B7E40400FC5417F5FF1F034545DD37
:103E0000829719C1BC5482972165218DB24022440A
:103E100092444101828093F715009DC3B7E70400E7
:103E200083A7471A17F6FF1F1306C6CE9385817521
:103E300017F5FF1F0345C5D9829713451400F9B73D
:103E400093F7250099CFB7E70400BC4F1306006431
:103E5000894517F5FF1F0345A5D782971345240011
:103E600075B793F785009DC7B7E7040003A8871AC5
:103E70001307401F97F7FF1F83C787D58146130697
:103E80004006994517F5FF1F035545DA029813457B
:103E90008400ADBF93F745000145ADDBB7E40400F6
:103EA00083A7041817F5FF1F035545D88297BC4C0C
:103EB00013060064914517F5FF1F034565D18297EE
:103EC00013454400A1B797F7FF1F83D727D6639602
:103ED000A70217F7FF1F231CB7D417F7FF1F2319DB
:103EE000C7D417F7FF1F2316D7D42E861725000037
:103EF00013054574BE856F00502A17250000130571
:103F0000E5746F00503E03574500011106CE22CCE8
:103F100097F7FF1F83D787D1172500001305057377
:103F20006310F706C167F91717F7FF1F2320F7D0B3
:103F300037E4040097F7FF1F23AC07CE7C4C89457C
:103F400017F5FF1F0345C5C882977C4C914517F5AF
:103F5000FF1F0345E5C7829797F7FF1F83C7A7CBCE
:103F600095C78547A307F100832744171306F1007F
:103F7000854513055030829717250000130585628B
:103F8000EF007036F24062440561828097F7FF1FB0
:103F900083C777C81725000013058565F5F38547A6
:103FA000A307F100832744171306F1008545130585
:103FB000503082971725000013050561D1B77D1594
:103FC000954763EEA718172700001307675A0A05DD
:103FD0003A951C41011122CC06CE26CABA972E84EE
:103FE0008287172500001305E566EF00D02F05A294
:103FF00003C725009947631CF7002E8529378345A1
:104000006400172500001305E565EF00101997F708
:10401000FF1FA38107C01725000013056566F1B7D0
:1040200003C7250095476317F702C16717F7FF1FFE
:104030000357C7BFF91703D5A5006307F702B7E712
:10404000040083A7C717829717250000130545644E
:10405000EF007029854717F7FF1FA30DF7BA172543
:1040600000001305656551B797F7FF1F2390A7BCA4
:1040700083D7E500B7E40400096617F7FF1F23188C
:10408000F7BA83D705011306069017F5FF1F0345FE
:1040900025B417F7FF1F231DF7B883D72501A145C6
:1040A00017F7FF1F2317F7B8BC4C8297BC4C1306B9
:1040B0000064914517F5FF1F034585B182970356AC
:1040C000E4008355A400172500001305A55DEF004B
:1040D000D00C49B7172500001305C55E39B783C555
:1040E00025009147639AF5028547172500001305BF
:1040F000E55EA307F100EF00101FB7E7040083A7F8
:1041000047171306F1008545130550308297F2409A
:104110006244D244056182809947639DF5002285FF
:10412000DD3383456400172500001305A553EF0018
:10413000D006F1BF9547639FF5008347140017250C
:1041400000001305A559E39207EA1725000013059F
:10415000A55A61BD172500001305855AC9BF828085
:104160006D71232481102326111023229110328493
:1041700001CD89476306F5028320C1100324811015
:1041800083244110516182801725000013050558D2
:10419000AE84EF005015A2852685EFF04F9BE9BF56
:1041A000B7E70400FC472800829717250000130595
:1041B000A556EF0050138347810039C01307000B49
:1041C000638EE7001387A7051377F70F8D4663E922
:1041D000E602A2852800EFF0EF9D79BF8547E3FD59
:1041E00087F883459100172500001305A553B335C3
:1041F000B00097F7FF1F238FB7A0EF00007AADBF85
:1042000003479100A207D98F35671307D755638DF0
:10421000E7066366F7022D671307B7556381E70664
:1042200031671307C7556386E70429671307A75546
:104230006392E702A2852800EFF02FC335BF3967EC
:104240009306E7656383D70663E9F6001307E7552E
:104250006388E704A285280089B73D679306F75570
:10426000638AD7041307F766E396E7FEEFF06FD98A
:1042700021B70146A2852800EFF00FB8F5BDA28551
:104280002800EFF00FBDCDBD8947E3F787EE93051A
:10429000E4FFC205C1811305A100EFE06FD7E9BDBE
:1042A000A2852800EFF02FBDC1BDA2852800EFF048
:1042B0000FC7D9B5EFF02FCFC1B5411122C417F404
:1042C000FF1F1304E486AA86172600001306C62BD8
:1042D0002285C14506C6EF00F0010357440097F759
:1042E000FF1F9387E7852393E70003576400239418
:1042F000E700B240224441018280130101DE232CF9
:10430000812037E4040083270408232E1120232A68
:104310009120232821212326312117050000130590
:1043200045AC829717F9FF1F1309898A994785447D
:104330002300A9002318F100972500009385C52DBF
:1043400093074006172500001305C5F32314F11049
:104350002304910097F9FF1F9389298C3D2D83D564
:104360000900172500001305E522052D2945852D97
:1043700003D5090099378327441730008545130575
:10438000503082978327441717E6FF1F1306467B9A
:10439000CD451305703082978327441717E6FF1F1A
:1043A00013060678B54513056030829783274417B6
:1043B000100889451305103182978327441730026E
:1043C00089451305203182978327441593050032D0
:1043D0000D45829783274415930500321145829736
:1043E000A3019100230291002304910023240110D2
:1043F000230801008327841630029145130570407D
:1044000082978327841613063100854513050040E3
:1044100082978327841650008545130510408297A4
:10442000832784161008854513052040829783272B
:104430008416300085451305504082978327041564
:104440007D558297832744137D5582977D55EFE0F4
:10445000DF838327440C8297EFE00FE183278414E6
:1044600017E6FF1F1306C66CD5450145829789479D
:104470001306700F814508082302F100EFD0AFD377
:104480008D471306700F814528022308F100EFD0F5
:104490008FD291472304F11097E7FF1F938707748A
:1044A000984383C747003AC42306F100EFF0AFBB3F
:1044B000500085450545EFE07F8410089305700F97
:1044C0000945EFE0BF8330029305700F0D45EFE023
:1044D000FF82300095451145EFE05F82C16717E725
:1044E000FF1F1307A774F9171CC32322070017E542
:1044F000FF1F1305A56DEFE04FFF8327C41D17E5D0
:10450000FF1F1305E57182973C4803450900854567
:1045100082978320C12103248121832441210329FF
:1045200001218329C1201301012282800111C16769
:1045300026CA06CEAA8422CC17E5FF1F0355056FB5
:10454000F9176305F50437E40400832784122E86E7
:104550002315B10001478146ED4582977C440356FF
:10456000A1002AC6A68582972C0017E5FF1F0355D8
:10457000E56BEFE05F8419C9172500001305C50A34
:104580009D238327C412ED4528008297F2406244A0
:10459000D2440561828001118547A307010017E716
:1045A000FF1F2303F768B7E7040083A7471706CE6A
:1045B0001306F1008545130550308297F2400561DE
:1045C0008280014863C6050E63DB06003306C040E7
:1045D000B337C000B306D0401348F8FF9D8EB687AE
:1045E0003283AA8EAE886391061863FCC50C4167BE
:1045F0006361E61EB70700016365F63693568601D0
:10460000E147172700001307671336970347070092
:10461000BA97130700021D8F19CBB395E500B35766
:10462000F5003313E600B3E8B700B31EE5001356F8
:104630000301B3D7C80293160301C18213D70E0139
:10464000B3F5C8023385F602C205B3E8E50063FAA4
:10465000A8009A981387F7FF63E4680063E9A8321B
:10466000BA87B388A840B3D5C802C20E93DE0E0144
:10467000B3F8C802B386B602C208B3E8D80163FB38
:10468000D8009A981387F5FF63E56800F91563E38E
:10469000D800BA85139507014D8D8145630908003F
:1046A0003305A040B337A000B305B0409D8D828094
:1046B0003305A040B337A000B305B0409D8D7D58B1
:1046C00021B701E605433353D3024167636AE30E22
:1046D000B7070001636BF32893568301E14717275F
:1046E00000001307A705369703470700BA9713077B
:1046F00000021D8F65EB93180301B3866540135FBD
:10470000030193D80801854513D70E01B3D7E603FB
:10471000B3F6E60333861703C206558F637AC700E4
:104720001A979386F7FF636467006365C726B687A9
:10473000118FB356E703C20E93DE0E013377E70302
:10474000B388160342073367D701637B17011A97B3
:104750001386F6FF63656700F91663631701B28677
:1047600013950701558D1DBF63E1D504C16763E152
:10477000F604B707000163E2F61E93D8860161478D
:1047800097270000938787FBC69703C3070093070B
:1047900000023A93B3876740E9EB63ECB61C33350C
:1047A000C500134515008145D5BD81450145FDB5C1
:1047B0009307F00F63F2D71C93D886002147C9B73F
:1047C0001307F00F9A86E37C67F093568300A147A6
:1047D00039B71307F00FB286E375C7E29356860028
:1047E000A14705B53313E30033D6F500135F03018A
:1047F000335EE603B396E500B357F500DD8E9318FC
:10480000030193D80801B31EE50093D50601B377E1
:10481000E6033387C803C207CD8F63FBE7009A978F
:104820001306FEFF63E3671663F1E716791E9A9796
:10483000998F33D6E703139706014183B3F7E70354
:104840003385C80293960701D98E63FBA6009A961A
:104850009307F6FF63E7661263F5A61279169A9638
:1048600093150E01898ED18D45B533576600B396E9
:10487000F600D98EB3D8650013DF0601B3DEE80376
:10488000139E060133536500135E0E01B395F500C8
:10489000B365B30013D705013316F600B3F8E80388
:1048A0003303DE03C20833E7E800637B6700369713
:1048B0009388FEFF6369D70C6377670CF91E369700
:1048C000330767403353E703C205C1813377E703FA
:1048D000B3086E024207D98D63FB1501B695130725
:1048E000F3FF63EED50863FC15097913B695C20E84
:1048F000416FB3EE6E001307FFFFB3F6EE0013D364
:104900000E01718F4182338EE602B3851541B38665
:10491000C60293580E013307E302BA96C6963306D1
:10492000C30263F3E6007A9613D306011A9663E294
:10493000C5026385C500768581458DB341677D17C6
:10494000F98EC206337EEE00B317F500F296E3F45B
:10495000D7FE1385FEFF814591B393D806014147E9
:1049600005B593560601C14769B993560301C1477E
:10497000BDB3814505451DB3B688014711B53A83DE
:10498000BDB73E86F1BDC68E25BF328E55B5F9172F
:104990009A98C1B9F9171A9761BB39713EDA2ED2CC
:1049A00032D436D63AD842DC46DE97E7FF1F9387EB
:1049B000672222CC804326CA06CEAA8409C41C4C96
:1049C00099E32285F9230C4454102686228536C6A5
:1049D000EF00D059F2406244D2442161828001113B
:1049E00097E7FF1F9387071F22CC804306CEAA8537
:1049F00019C41C4C89E72AC62285612BB245104494
:104A000022856244F24005616F10403B011126CAC5
:104A10004AC806CE22CC4EC652C4AA842E8901C5ED
:104A20001C4D91E3BD239C4C804499E3268595233E
:104A300097270000938787E2631CF402C0408357E6
:104A4000C400A18BB1C71C48A1C7FD59294A1C4409
:104A500083450900FD17B1E91CC463DE0706228601
:104A6000A94526851122FD576308F502294535A081
:104A700097270000938787E06314F4008044C1B750
:104A800097270000938787DBE31BF4FAC04445BFF8
:104A9000A2852685512A55D97D55F2406244D244DB
:104AA0004249B249224A056182801CC4050963D784
:104AB0000700184C63CBE700638945011C4013874E
:104AC000170018C02380B70059B7228626856928A9
:104AD000E31F35F7D1B71C401387170018C02947CB
:104AE0002380E70061B797E7FF1F9387A70EAA858A
:104AF000884329BF35713ECBA6DA36C73AC942CDC5
:104B000046CF97E7FF1F9387E70C86DEA2DC84433E
:104B100063DB05009307B0089CC07D55F6506654D2
:104B2000D6540D61828093078020231AF1002AC495
:104B30002ACC814799C19387F5FF3EC83ECE7401C8
:104B4000FD572E8426852C00231BF10036C2EF0072
:104B50007013FD576355F5009307B0089CC05DDCEA
:104B6000A247238007005DBF011122CC26CA4AC894
:104B700006CE4EC6AA842E89328401C51C4D91E30F
:104B8000092997270000938767CD6319F406C04071
:104B90001C4C1CC48357C400A18BC9C31C48BDCF87
:104BA0001C4808409379F90F1379F90F1D8D5C4863
:104BB0006346F500A2852685752C2DE51C44050568
:104BC000FD171CC41C401387170018C02380370131
:104BD0005C486389A7008357C400858B81CBA947B4
:104BE0006316F900A285268571240DEDF24062441A
:104BF0004A85D2444249B249056182809727000024
:104C00009387C7C76314F400804459B797270000FF
:104C10009387C7C2E31EF4F6C0449DBFA2852685D4
:104C200021203DDD7D59D9B7411197E7FF1F9387BB
:104C300067FA26C2844322C44AC006C62A892E8443
:104C400089C49C4C99E32685A92697270000938761
:104C5000E7C0631CF402C0400317C40093170701A8
:104C6000C18393F68700B5EE93F607019DEEA54745
:104C70002320F900136707042316E4007D55B24092
:104C80002244924402494101828097270000938781
:104C9000E7BE6314F4008044C1B7972700009387F0
:104CA000E7B9E31BF4FAC04445BF918B8DC74C585C
:104CB00089C9930744046384F5004A859123232A14
:104CC00004028357C4002322040093F7B7FD231680
:104CD000F4001C481CC08357C40093E787002316C8
:104CE000F4001C4881EF8357C4001307002093F79A
:104CF00007286385E700A2854A85A5218357C4005C
:104D000013F7170005C75C4823240400B307F040DD
:104D10001CCC1C480145A5F78317C40013F70708EE
:104D200039DF93E707042316F40089BF898B014715
:104D300091E3584818C4F1BF83D7C500011122CCB4
:104D400026CA06CE4AC84EC613F78700AA842E8408
:104D500071EFD841634DE000B841634AE00001457E
:104D6000F2406244D2444249B249056182805854BB
:104D70007DD703A904009396370123A0040063DDC7
:104D8000060670488357C400918B99C75C401D8EFE
:104D90005C5899C33C401D8E5C540C50814626855E
:104DA0008297FD570357C400631DF5009440F547F3
:104DB00063E8D706B70740208507B3D7D700858BB0
:104DC000A5C31C48232204001CC09317370163D8D5
:104DD0000700FD576314F5009C4091E368C84C58E8
:104DE00023A02401ADDD930744046384F5002685E8
:104DF0000129232A0402A5B70C50014685462685C1
:104E00000297FD572A86E31FF5F69C40A5DF7547FC
:104E10006385E70059476394E70423A0240181B721
:104E2000136707042316E4007D551DBF83A9050100
:104E3000E38709F203A905008D8B23A0350133090F
:104E40003941014791E3D84918C4E35A20F11C5471
:104E50000C50CA864E86268582976349A0008357E8
:104E6000C40093E707042316F4007DBFAA99330911
:104E7000A940E1BF9C49B9CF011122CC06CE2A84BA
:104E800011C51C4D81E72EC62922B2459727000087
:104E90009387C79C639BF5004C408397C50095C7DB
:104EA00022856244F240056141BD97270000938747
:104EB000E79C6394F5000C44CDB7972700009387D7
:104EC000E797E39CF5FC4C44C9BFF24062440145BE
:104ED0000561828001458280411122C406C62A8470
:104EE0002316B5002317C500232005002322050043
:104EF000232405002322050623280500232A050074
:104F0000232C0500214681451305C505EFC0BFAA26
:104F1000971700009387C7F55CD097170000938719
:104F200027F81CD497170000938767FC5CD4971769
:104F30000000938727FF00D01CD8B24022444101D3
:104F4000828097050000938525F389AA411126C226
:104F5000130680069384F5FFB384C4024AC02E89E9
:104F600022C406C693854407A1262A8401CD2320A6
:104F7000050023222501310508C4138684068145D6
:104F8000EFC07FA32285B2402244924402494101EE
:104F900082801C4DBDE3411106C622C49707000064
:104FA000938767FA1CD597270000938727989C431F
:104FB0002324050423260504232805046314F5008F
:104FC00085471CCD2A841D2848C02285052808C491
:104FD00022852D2048C4484001469145F53D0844AE
:104FE0000546A545D53D48440946C945F53585479B
:104FF0001CCCB2402244410182808280411197271B
:1050000000009387A79226C284434AC006C69C4CE0
:1050100022C42A8999E32685AD3F93848404804481
:10502000DC40FD1763D607009C40B9CF8440C5BF64
:105030000317C40039E7C17785072322040623201C
:10504000040023220400232404005CC42328040059
:10505000232A0400232C0400214681451305C4059E
:10506000EFC07F95232A0402232C04022324040486
:10507000232604042285B24022449244024941017D
:1050800082801304840671BF91454A85C13588C06A
:1050900051FDB1472320F9000144E9BF797122D4C1
:1050A0004AD052CC56CA5AC85EC606D626D24ECE72
:1050B0002A8AAE8A130485040149054BFD5B09EC7D
:1050C000B25022544A8592540259F249624AD24A55
:1050D000424BB24B45618280044483294400FD1950
:1050E00063D409000040E1BF83D7C400637BFB00A9
:1050F0008397E40063877701A6855285829A336996
:10510000A90093848406E1BF1971A6DAAE84839561
:10511000E500A2DC86DE328463DC050083D7C400B0
:1051200023A0060093F7070885E7930700401DA01A
:10513000300836C6EF009064B246E34105FE724780
:10514000BD67F98F7977BA9793B717009CC2F1BF03
:10515000930700041CC0F6506654D65401450961FB
:10516000828083D7C500011122CC06CE26CA4AC848
:10517000898B2E8489CF930774041CC01CC8854773
:105180005CC8F2406244D2444249056182807400A6
:105190003000AA84953FA2452A892685112A01ED6F
:1051A0008317C40013F7072069FFF19B93E72700DB
:1051B0002316F400C9B7970700009387C7D89CD47B
:1051C0008357C40008C008C893E707082316F400F3
:1051D000A2475CC8B24791CF8315E4002685EF0053
:1051E000905C01C98357C400F19B93E71700231615
:1051F000F4008357C4003369F9002316240151B722
:10520000DDC583A7C5FF411122C406C626C213848B
:10521000C5FF63D307003E94AA84EF00B06F97E701
:10522000FF1F938727A19C4391EF2322040097E758
:10523000FF1F23A187A02244B2402685924441014A
:105240006F00706D637EF40014403307D4006396E2
:10525000E7009843DC43369718C05CC0C9BFBA87E3
:10526000D84319C3E37DE4FE94433386D700631F1C
:1052700086001040B29694C33386D700E31DC7FA68
:1052800010435843B29694C3D8C375B76375C4002E
:10529000B1479CC04DB71040B306C4006316D70099
:1052A00014435843B29614C058C0C0C369B7828033
:1052B000011126CA93843500F19806CE22CC4AC843
:1052C0004EC6A104B14763FBF404B14463EAB404DD
:1052D0002A89EF00306497E7FF1F9387A7959843CB
:1052E0003A8429E897E7FF1F938707959C4389EB4A
:1052F00081454A85EF00F03497E7FF1F23AEA79260
:10530000A6854A85EF00F033FD59631B3507B14789
:105310002320F9004A85EF00106029A0E3D804FAA1
:10532000B1471CC10145F2406244D2444249B249EE
:10533000056182801C40858F63C10704AD4663F61A
:10534000F6001CC03E9404C001A85C4063158702AF
:1053500017E7FF1F2320F78E4A85EF00D05B130568
:10536000B4009307440061993307F5404DDF3A9448
:10537000898F1CC04DBF5CC3C5B72287404095B71D
:10538000130435007198E30085FCB305A4404A85F9
:10539000EF00302BE31935FB9DBF01114AC803A96B
:1053A000850022CC52C45AC006CE26CA4EC656C26A
:1053B0002E84328B368A63ED260983D7C50013F716
:1053C000074849C704408C495848AA8AB389B44061
:1053D0008D44B384E4020947B3C4E4021387160082
:1053E0004E9763F3E400BA8493F70740D1C3A685D0
:1053F00056857D3D2A890DE5B14723A0FA008357E4
:10540000C4007D5593E707042316F400F24062447C
:10541000D2444249B249224A924A024B05618280F3
:105420000C484E86EF00103F8357C40093F7F7B740
:1054300093E707082316F4002328240144C84E9953
:10544000B38434412320240104C4528963732A01A4
:10545000528908404A86DA85EF0030471C440145EE
:10546000B38727411CC41C403E992320240179BFE7
:1054700026865685EF00504A2A895DFD0C485685E0
:1054800041339DBF83D7C500717126D34AD14ECF1A
:1054900006D722D552CD56CB5AC95EC762C566C360
:1054A00093F70708AA892E89B284B1C39C49A1E366
:1054B0009305000436C6ED3B2320A9002328A9004C
:1054C000B24615E1B14723A0F9007D55BA502A54E0
:1054D0009A540A59FA496A4ADA4A4A4BBA4B2A4C50
:1054E0009A4C4D61828093070004232AF9009307A8
:1054F0000002A30CF1029307000302DA230DF1026C
:1055000036CE930B5002971A0000938A2A39054C25
:10551000294B26848347040099C3639C7709B30C05
:105520009440638D0C00E6862686CA854E85B53587
:10553000FD576304F51AD256E69636DA834704001F
:10554000638D0718FD579304140002D002D63ED293
:1055500002D4A301010682DC83C5040015465685EA
:10556000EF00B02913841400825731E513F70701C7
:1055700009C713070002A301E10613F7870009C753
:105580001307B002A301E10683C604001307A002BB
:10559000638BE602B2572684814625460347040002
:1055A00093051400130707FD6374E6068DC63ED607
:1055B0001DA0050485B7330555413315AC00C98FCF
:1055C0003ED0A28451BF724793064700184336CE9F
:1055D000634907023AD6034704009307E002631FBA
:1055E000F704034714009307A002631BF702F24776
:1055F0000904138747009C433ACE63C107023ED299
:1056000035A83307E04093E727003AD63ED0E1B70C
:10561000B387670385462E84BA9749B7FD57C5B748
:10562000050402D2814681472546034704009305BD
:105630001400130707FD6378E606F1F283450400C2
:105640000D46171500001305E525EF00101B11CDC1
:1056500097170000938707251D8D93070004B397C4
:10566000A700025505045D8D2AD083450400194624
:10567000171500001305452393041400230CB102F1
:10568000EF00B01725C597B7FFFF9387A79795E75A
:105690000257F2471377071009CF91073ECED25732
:1056A000D2973EDABDB5B387670385462E84BA9795
:1056B000ADBF9D07E19BA107D5B77808970600000D
:1056C0009386E6CD4A860C104E8597000000E700D1
:1056D0000000FD572A8AE314F5FC8357C9007D5565
:1056E00093F70704E39407DE5255CDB37808970685
:1056F00000009386C6CA4A860C104E852129D1BF68
:105700001C46FD171CC663DA0700184E63C5E70088
:10571000A9476394F5006FF02FC51C422E851387AF
:10572000170018C22380B7008280011122CC26CA3C
:105730004AC84EC652C406CE2A89AE893284B30402
:10574000D6007D5A63149400014509A883450400DE
:105750004E864A8575370504E31645FFF2406244DC
:10576000D2444249B249224A05618280357122CD34
:1057700026CB4AC94EC706CF52C556C35AC1DEDE34
:10578000E2DCE6DAAA89AE843289368409C51C4D8A
:1057900099E3EFF01F80971700009387270C639C15
:1057A000F40C83A4490083D7C400A18BFDC79C4897
:1057B000EDC793070002A304F1029307000302D28E
:1057C0002305F10222C6930B5002971A0000938A18
:1057D000EA0C054C294B4A848347040099C3639122
:1057E000770FB30C2441638D0C00E6864A86A685AC
:1057F0004E85253FFD576307F51E9256E69636D235
:10580000834704006380071EFD571309140002C874
:1058100002CE3ECA02CCA309010482D4834509000A
:1058200015465685EF00607D13041900C24759E9FB
:1058300013F7070109C713070002A309E10413F7CF
:10584000870009C71307B002A309E10483460900D2
:105850001307A0026380E608F2474A848146254682
:105860000347040093051400130707FD6379E60A54
:10587000B5CA3ECE85A89717000093872700639589
:10588000F40083A4890005B797170000938707FBEE
:10589000E39BF4F083A4C90039B7A6854E85EFF0E9
:1058A000AFB801D97D55FA406A44DA444A49BA4949
:1058B0002A4A9A4A0A4BF65B665CD65C0D61828086
:1058C000050419BF330555413315AC00C98F3EC8D7
:1058D0002289A9B7324793064700184336C6634961
:1058E00007023ACE034704009307E002631FF70460
:1058F000034714009307A002631BF702B247090491
:10590000138747009C433AC663C107023ECA35A8C5
:105910003307E04093E727003ACE3EC8E1B7B387AC
:10592000670385462E84BA9725BFFD57C5B7050482
:1059300002CA8146814725460347040093051400A7
:10594000130707FD6376E606F1F2834504000D4672
:1059500017150000130505F54D2511CD971700000B
:10596000938747F41D8D93070004B397A700424522
:1059700005045D8D2AC883450400194617150000EB
:10598000130585F2130914002304B102BD253DC19E
:1059900097A7FFFF9387076795E74247B2471377BB
:1059A000071009CF91073EC69257D2973ED225B530
:1059B000B387670385462E84BA97BDBF9D07E19BD9
:1059C000A107D5B7780097060000938646D62686AD
:1059D0000C084E8597000000E7000000FD572A8A5A
:1059E000E314F5FC83D7C40093F70704E39C07EAAC
:1059F000125555BD780097060000938646D326863B
:105A00000C084E85012AD9BF797156CA9C49BA8AB9
:105A1000984522D426D24ECE52CC06D64AD05AC869
:105A20005EC6AA892E84B284368A63D3E700BA8719
:105A30009CC00347340419C385079CC01C4093F7DE
:105A4000070281C79C4089079CC003290400137981
:105A50006900631A0900130B9401FD5B5C449840D4
:105A6000998F634CF9041C408346340493F7070272
:105A7000B336D000A5EB13063404D2854E85829A46
:105A8000FD576303F5041C4011469840998B54441C
:105A900081446397C700B384E64063D30400814424
:105AA0001C4418486354F700998FBE940149690457
:105AB0007D5B63982405014509A885465A86D285F1
:105AC0004E85829A631E75017D55B25022549254C0
:105AD0000259F249624AD24A424BB24B4561828036
:105AE0000509ADBF3307D40013060003A301C704A3
:105AF0000347540493871600A2978906A381E704FD
:105B00009DBF85462286D2854E85829AE30E65FB2F
:105B1000050945B7797122D426D24AD04ECE06D691
:105B200052CC56CA5AC8B68983C6850193079006D7
:105B30003289AA842E8413863504638DF60263E2CB
:105B4000D706930780056387F61863EDD700638057
:105B5000062293073004638EF60A930A2404230175
:105B6000D404C9A0930730066385F60A930740065C
:105B7000E395F6FE1C40084393F60708930545009D
:105B8000C5C61C410CC363D807001307D002B30776
:105B9000F040A301E40497160000938666D12947DC
:105BA0006DA8930700076383F61663E5D702930792
:105BB000E006638AF6189307F006E390F6FA0C40C5
:105BC0001C4313F80508138547006307080608C33C
:105BD0009C438DA893075007E383F6FE9307800745
:105BE000638AF61293073007E399F6F61C43D04117
:105BF00081459386470014C383AA07005685F52E76
:105C000001C53305554148C05C401CC8A3010404CC
:105C100071A81C43930A2404938647009C4314C331
:105C20002301F4048547D5B793F607041C410CC340
:105C3000B9DAC207C18781BF93F5050408C3C9D982
:105C400083D707001307F0066387E60E9716000058
:105C5000938606C62947A30104044C400CC463C5BF
:105C6000050008406D9908C099E3B28A91CDB28AC7
:105C7000B3F5E702FD1AB69583C505002380BA0087
:105C8000B3D5E70263FFE70AA147631EF7001C4094
:105C9000858B91CB58401C4863C7E70093070003EE
:105CA000A38FFAFEFD1A3306564110C84E87CA86E6
:105CB0007000A2852685893B7D5A631E450B7D5564
:105CC000B250225492540259F249624AD24A424B8B
:105CD00045618280A382D50497160000938646BD55
:105CE0000C40084313F805081C411105630D080218
:105CF00008C313F7150001C793E505020CC041471F
:105D0000B9FB0C4093F5F5FD0CC0B1B79C4193E78E
:105D100007029CC193078007A302F40497160000B2
:105D2000938646BA75BF13F8050408C3E30308FC5D
:105D3000C207C1837DBF97160000938666B72147CF
:105D400019BFAE8735B794411C43CC4913F80608F8
:105D5000138547006306080008C39C438CC301A851
:105D600008C393F606049C43F5DA2390B700232872
:105D70000400B28A25BF14485686CA8526858299B2
:105D8000E30F45F31C40898B8DE7B2474844E35944
:105D9000F5F23E8535B785465686CA8526858299B1
:105DA000E30F65F1050A5C443247998FE345FAFE3B
:105DB000E9BF014A930A94017D5BF5B7011122CC3A
:105DC00006CE2A8409C91C4D99E732C62EC4EFF0CD
:105DD0004F9C3246A24597170000938727A8631669
:105DE000F60250401C46FD171CC663D00704184E2F
:105DF00063C7E70093F7F50F29476398E702228509
:105E00006244F24005616FE03FD697170000938728
:105E1000E7A66314F6001044F1B7971700009387C4
:105E2000E7A1E311F6FC504475BF1C4213F5F50FD2
:105E30001387170018C22380B700F240624405613F
:105E40008280411122C42A842E8523A2017606C6AF
:105E5000EFC0BF8EFD576317F500938741769C43D3
:105E600091C31CC0B240224441018280411122C42E
:105E70002E848395E50006C6DD2C634905007C4829
:105E8000AA977CC8B2402244410182808357C40053
:105E90007D777D17F98F2316F400EDB783D7C50002
:105EA000011122CC26CA4AC84EC606CE93F7071067
:105EB000AA842E843289B68991C78395E5008946E4
:105EC000014631228357C4007D777D17F98F231651
:105ED000F4008315E4006244F240CE864A86B2495B
:105EE00042492685D24405613DA8411122C42E8431
:105EF0008395E50006C6E128FD570357C400631BE0
:105F0000F500FD77FD17F98F2316F400B240224407
:105F1000410182808567D98F2316F40068C8FDB7D8
:105F20008395E50005A8411122C42A842E85B285F7
:105F3000368623A2017606C6EFC0AFFDFD57631774
:105F4000F500938741769C4391C31CC0B240224424
:105F500041018280411122C42A842E8523A2017628
:105F600006C6B124FD576317F500938741769C431D
:105F700091C31CC0B240224441018280411122C41D
:105F80002A842E85B28523A2017606C63D24FD57BC
:105F90006317F500938741769C4391C31CC0B240C0
:105FA000224441018280411122C42A842E8523A2E9
:105FB000017606C6092CFD576317F50093874176D5
:105FC0009C4391C31CC0B2402244410182804111D4
:105FD00022C42A842E85B285368623A2017606C67F
:105FE000CD2AFD576317F500938741769C4391C3F3
:105FF0001CC0B24022444101828093F5F50F2A96DD
:106000006314C5000145828083470500E38DB7FE18
:106010000505FDB7B3C7A5008D8B3307C50081E724
:106020008D4763EEC700AA876370E50A83C6050043
:1060300085078505A38FD7FEE3EAE7FE8280937686
:106040003500AA8791CA83C6050085078505A38FF9
:10605000D7FE93F63700FDB79376C7FF138606FE8B
:1060600063F0C70683A3050083A2450083AF8500C4
:1060700003AFC50083AE050103AE450103A385014F
:1060800083A8C5019385450223A0770003A8C5FF17
:1060900023A2570023A4F70123A6E70123A8D701D1
:1060A00023AAC70123AC670023AE170193874702D9
:1060B00023AE07FF75B790419107910523AEC7FE48
:1060C000E3EBD7FEE3E4E7F6828063F3A504B3864F
:1060D000C500637FD5029345F6FF8147FD176393A3
:1060E000F50082803387F600034807003387C70036
:1060F0002A9723000701DDB73387F50083460700A1
:106100003307F50085072300D700E317F6FE8280EA
:106110008147E5BF8280828081E5B2856FF04F992B
:10612000011122CC06CE26CA4AC84EC6328401EEE0
:10613000EFF00F8D0149F24062444A85D244424952
:10614000B24905618280AE84AA8981282689E374D8
:1061500085FEA2854E85EFF0AF952A8969DDA6857B
:1061600022864D3DA6854E85EFF08F89E9B7411116
:1061700022C42A842E85B285368623A2017606C6DD
:10618000B928FD576317F500938741769C4391C367
:106190001CC0B24022444101828083A7C5FF138501
:1061A000C7FF63D50700AA959C413E95828093075F
:1061B000800523A2F1767D5582809307800523A276
:1061C000F1767D5582809307800523A2F176014503
:1061D00082809307800523A2F1767D558280930704
:1061E000800523A2F1767D558280000078C3FFFFF1
:1061F000A0C3FFFFC8C3FFFFE0C3FFFFFAC3FFFF59
:106200000AC4FFFF32C4FFFF5AC4FFFF72C4FFFF7E
:106210008CC4FFFFFE006578706572696D656E74F1
:10622000616C0000626C656465732E636F6D0000C5
:106230004D6F64656C204E756D62657200000000E4
:1062400053657269616C204E756D62657200000065
:10625000CCCAFFFFF2CAFFFF0CCBFFFF2ACBFFFF28
:1062600048CBFFFF73696D706C6550726F66696C27
:10627000655F57726974654174747243420000002F
:106280004150505F4442472025733E2000000000EB
:1062900073696D706C6550726F66696C655F57727B
:1062A000697465417474724342206C656E3A2025AE
:1062B0006400000043483539785F424C455F4C49E3
:1062C000425F56312E330000686561642066696C58
:1062D00065206572726F722E2E2E00004C4942208E
:1062E000696E6974206572726F7220636F64653ABB
:1062F000202578202E2E2E0A000000002A200000E3
:106300004170705F496E69743A20424C452D6F6E42
:106310006C7920286E6F204D6573682073746163FB
:106320006B290D006C6F63616C20696D616765207E
:10633000696E666F206C656E2065727200000000E9
:106340004F54413A2073757370656E642043353540
:106350004320424C45206E6F746966790D00000041
:106360006C6F63616C20757064617465206C656E20
:1063700020657272000000006C6F63616C207665AE
:1063800072696679206C656E20657272000000008B
:106390006C6F63616C20656E64206C656E20657245
:1063A000720000004941505F454E442028424C4550
:1063B000206C6F63616C290D000000004170705FFC
:1063C000426C655F4C6F63616C5F4F74615F4861E5
:1063D0006E646C6500000000436F6E66696720475D
:1063E0006174657761790D007461726765745F64CB
:1063F000657620253034580D0A0000004449534189
:10640000424C454400000000454E41424C4544008A
:106410004465627567206D6F64652025730D0A0001
:106420004164766572746973696E6720656E616236
:106430006C65640D000000005175657279204D6532
:1064400073682041646472202D2050726F766973E6
:10645000696F6E65643A25642C20416464723A3039
:1064600078253034580D0A005175657279204D65D4
:106470007368204B6579202D2050726F766973699F
:106480006F6E65643A25640D0A000000446562750C
:1064900067206D6F6465206C6F616465642066724F
:1064A0006F6D20666C6173683A2025640A000000F5
:1064B0004465627567206D6F6465207573696E67EA
:1064C0002064656661756C743A2025640A000000DA
:1064D0004D65736820475720647374206C6F616446
:1064E00065643A203078253034580D0A00000000E9
:1064F0004D65736820475720647374206465666136
:10650000756C743A203078253034580D0A0000003C
:106510004465627567206D6F64652073617665649C
:1065200020746F20666C6173683A2025640A00004D
:106530004D657368204757206473742073617665D6
:10654000643A203078253034580D0A00434D445FBA
:10655000484541443A3078253034580D0A0000004F
:1065600053746F705F4164767200000076DAFFFF4B
:1065700084DAFFFF72DBFFFFB4DAFFFF68DBFFFFA7
:10658000DEDBFFFF574D315F25303458000000003F
:106590006D795F6E65745F616464723A25640000B2
:1065A0005265737461727420616476657274697384
:1065B000696E6720284445425547206D6F64652900
:1065C0000000000052657374617274206164766526
:1065D00072746973696E6720286E6F742070726FB1
:1065E000766973696F6E65642900000053746F707B
:1065F000206164766572746973696E672028616CC6
:1066000072656164792070726F766973696F6E6507
:10661000642900005065726970686572616C5F4939
:106620006E6974004E6F746966792045525220007D
:10663000557064617465202578202D20496E742082
:106640002578200A000000004552522E2E0000003E
:10665000496E697469616C697A65642E2E00000068
:10666000446973636F6E6E65637465642E2E205289
:106670006561736F6E3A25780A00000041647665A3
:1066800072746973696E672E2E000000436F6E6E20
:10669000656374696F6E206D61782E2E2E00000088
:1066A000436F6E6E202578202D20496E742025784A
:1066B000200A0000436F6E6E65637465642E2E00C1
:1066C000436F6E6E656374656420416476657274B1
:1066D0006973696E672E2E0057616974696E672051
:1066E000666F72206164766572746973696E672E75
:1066F0002E0000004572726F722E2E004572726F6E
:10670000722E2E25780A00005265762043484152A9
:10671000310000005265762043484152332E2E004E
:106720004F544120433535432073757370656E6453
:106730002025750D0A000000000102020303030377
:106740000404040404040404050505050505050501
:1067500005050505050505050606060606060606E1
:1067600006060606060606060606060606060606C9
:1067700006060606060606060707070707070707B1
:106780000707070707070707070707070707070799
:106790000707070707070707070707070707070789
:1067A0000707070707070707070707070707070779
:1067B0000707070707070707080808080808080861
:1067C0000808080808080808080808080808080849
:1067D0000808080808080808080808080808080839
:1067E0000808080808080808080808080808080829
:1067F0000808080808080808080808080808080819
:106800000808080808080808080808080808080808
:1068100008080808080808080808080808080808F8
:1068200008080808080808080808080808080808E8
:106830000808080808080808000000000000000018
:106840000000000000000000000000000000000048
:106850000000000000000000000000000000000038
:106860000000000000000000000000000000000028
:106870000000000000000000000000000000000018
:106880000000000000000000000000000000000008
:106890000000000000000000232D302B200000002D
:1068A000686C4C00656667454647000030313233FE
:1068B00034353637383941424344454600000000FC
:1068C0003031323334353637383961626364656666
:1068D0000000000076312E3000000000262A000063
:1068E00076312E3000000000272A0000292A0000FF
:1068F0000A18000002000000F068000076312E3017
:1069000000000000282A0000E0FF00000200000054
:1069100008690000E1FF0000E2FF0000E3FF000063
:10692000E4FF0000E5FF0000502B00200200000003
:106930000CE0040001000000F46800000200000008
:1069400012E0040001000000B62B0020020000004D
:10695000EC6800000100000024620000020000005A
:1069600012E0040001000000B42B0020020000002F
:10697000DC68000001000000D46800000200000094
:1069800012E0040001000000B52B0020020000000E
:10699000E868000001000000E0680000020000005C
:1069A00012E0040001000000BF2B002002000000E4
:1069B0000469000001000000FC6800009A28000043
:1069C0000000000000000000020000000CE00400D5
:1069D000010000000C6900000200000012E0040049
:1069E00001000000C02B002002000000146900001C
:1069F00003000000382C00200200000016E0040014
:106A000001000000AC2A00200200000012E0040097
:106A100001000000C12B00200200000018690000E6
:106A200001000000E82B00200200000016E0040036
:106A300001000000C02A00200200000012E0040053
:106A400001000000C22B0020020000001C690000B1
:106A500002000000302D00200200000016E00400BB
:106A600001000000D42A00200200000012E004000F
:106A700001000000C32B002002000000206900007C
:106A800000000000282E00200200000018E0040092
:106A900003000000EC2B00200200000016E00400C0
:106AA00001000000E82A00200200000012E00400BB
:106AB00001000000C42B0020020000002469000037
:106AC00004000000F02B00200200000016E004008B
:106AD00001000000FC2A0020862A0000762B00001E
:106AE00000000000436861726163746572697374C9
:106AF000696320310000000043686172616374655E
:106B00007269737469632032000000004368617227
:106B100061637465726973746963203300000000F7
:106B20004368617261637465726973746963203468
:106B30000000000043686172616374657269737478
:106B40006963203500000000BE3F00009A3D000050
:106B5000C63E00000201060302E0FF05FFD7070062
:106B600000000000574D315F303030300000000031
:106B7000000000000909574D315F303030300512F8
:106B800006006400020A00000000000058680000CF
:106B90007868000038680000000000000000000075
:106BA00000000000000000000000000000000000E5
:106BB00000000000000000000000000000000000D5
:106BC00000000000000000000000000000000000C5
:106BD00000000000000000000000000000000000B5
:106BE00000000000000000006847002002020200D0
:106BF00001D70700001001020A02081002FF14006A
:106C000060410000FF000000502B00200000000049
:086C100001020304050000006D
:020000040004F6
:10D000006F00C076000000000000000090000020CB
:10D010008C020020A9BDF9F590000020000000005E
:10D0200000000000900000209000002000000000A0
:10D030000000000090000020000000009000002090
:10D0400000000000900000209000002090000020D0
:10D050009000002090000020900000209000002010
:10D0600000000000900000209000002090000020B0
:10D0700090000020900000209000002090000020F0
:10D0800090000020900000209000002090000020E0
:10D090009000002001A0011113078008F3370780DA
:10D0A00093F787083EC201000100B71700409305BF
:10D0B00070052380B704130680FA2380C70401009B
:10D0C000010083C6B70493F6F60DA385D704238029
:10D0D00007049246F3A6068001000100937605023C
:10D0E000D5CEF336078093F6860836C401000100DA
:10D0F0002380B7042380C70401000100B706140091
:10D100007D89558D88C70100010001000100238041
:10D110000704A246F3A606800100010073370780CA
:10D12000137787083AC6010001002380B7042380E3
:10D13000C7040100010001000100372700409306E9
:10D140001005A303D78023800704B247F3A7078005
:10D150000100010093078008F3B7078093F7870861
:10D160003ECE01000100B717004013077005238071
:10D17000E704130780FA2380E7040100010003C7D6
:10D18000B70413670708A385E70423800704F24761
:10D19000F3A70780010001000561828093760504F2
:10D1A000BDC6F336078093F6860836C80100010035
:10D1B0002380B7042380C70401000100B7061400D0
:10D1C000938606047D89558D88C701000100010002
:10D1D000010023800704C246F3A606800100010077
:10D1E00073370780137787083ACA0100010023804C
:10D1F000B7042380C70401000100372700409306CD
:10D200002005A303D78023800704D24781B7733753
:10D210000780137787083ACC010001002380B70408
:10D220002380C7040100010098471367070C98C7C3
:10D2300023800704E24719BF011181460146814559
:10D24000114506CE7D2A93078008F3B7078093F730
:10D2500087083EC601000100B7170040130770059C
:10D260002380E704130780FA2380E704010001000C
:10D2700003C76704136717002383E70423800704A9
:10D28000B247F3A7078001000100F24005618280E8
:10D2900041118146014681451145A52213078008A9
:10D2A000F337078093F787083EC401000100B717E2
:10D2B0000040130670052380C704930680FA23807C
:10D2C000D70401000100FD552396B702238007040F
:10D2D000A245F3A50580010001007337078013778D
:10D2E00087083AC6010001002380C7042380D704C1
:10D2F0000100010003C76704136717002383E704D5
:10D3000023800704B247F3A707800100010001A0B2
:10D31000BD473305F50201007D1575FD8280411181
:10D3200022C426C206C6AA84014463179400B240F0
:10D33000224492444101828005041305803E420448
:10D34000C13F4180DDB72303048015472303E480F8
:10D3500001002302A480828083076480E3CE07FE5D
:10D3600023030480828083076480E3CE07FE0345A5
:10D370004480828083076480E3CE07FE2302A4807A
:10D380008280411126C44AC24EC006C61377F50BEF
:10D39000AD47AA892E8995446306F700194565377C
:10D3A000653F8D444E854537FD59FD146398340122
:10D3B000B240A244124982494101828013550901B9
:10D3C0001375F50F453F2209CDB7011126CC06CEC6
:10D3D000B704080051371545BD37713769372AC67C
:10D3E000A53F32459377150089EB1365150013753A
:10D3F000F50FF240E24405618280FD14E9FC01452D
:10D40000CDBF397126DC4ADA4ED852D656D45AD21C
:10D410005ED006DE62CE66CCB7E700E07D5783AA19
:10D42000070022C603AA470023A0E71823A2E71893
:10D43000B7170040130770052380E704130780FA2D
:10D440002380E70483C74704930B75FFB684E20784
:10D4500093FBFB0F8546AA892E8B32893724004027
:10D46000E187015763FA76016308D50089461307FF
:10D4700000026313D5000157D98F93F7F70FB71C3C
:10D4800000402382FC0411472303E4801305F00FBE
:10D490005D3D094CD135636D7C11B7050700DA9508
:10D4A00037870700795563F2E504B3879500636E0B
:10D4B000F702370B0800A94733EB65016399F906BA
:10D4C00089E48144513D26850DA0DA850945553D05
:10D4D00005090345F9FFFD14050B693D81C49377E8
:10D4E000FB0FFDF7DD3569FD7D55B71700401307CC
:10D4F00070052380E704130780FA2380E70403C73D
:10D500004704418B2382E704F250B7E700E023A0F1
:10D51000571123A24711E25432445259C259325A88
:10D52000A25A125B825B724CE24C21618280A54759
:10D530006395F90685691309F00FB3069900B37472
:10D540002B01B6941349F9FFB3749900856B3379B5
:10D550006901416B9387F9FFB3F7270199E363FCF6
:10D56000340193D94900C147E3E637FF99BF056904
:10D57000C1697D19D9B71305800D63886901130549
:10D5800000026384790113051008CA85DD3B353D2F
:10D5900021DD4E99B3843441D9B7DA852D45D53391
:10D5A000CA94E30099F205097D3BA30FA9FED5BFFC
:10D5B0009387F9FF93F7F70F6361FC0C83C71C0493
:10D5C00013073008631FF70437070800636BEB0489
:10D5D000B3079B00B706100063F5D704334BEB008D
:10D5E00089476393F9068980D549E38C04ECDA8591
:10D5F0000945413B11090327C9FF91472320E480D6
:10D6000003076480E34E07FE23033481FD17EDFB1F
:10D61000FD14110B81C49377FB0FE9FF7D3371F586
:10D62000E1B5B717004003C75704B70708001377E1
:10D63000070219E3B78707007955E378FBEA330758
:10D640009B00E3FFE7F855B58547E382F9F2DA85F9
:10D650002D45053B9389F4FFE38504E6293393F7D1
:10D66000390091EB832604800327090093074900C2
:10D67000E39AE6E43E89CE84F1BFB5476396F900AC
:10D680001305900BC93135BDB1471305B00AE38BC3
:10D69000F9FE99476391F904B7050800B365BB002B
:10D6A0002D45C53181448D4BA1497539639674016F
:10D6B000832704802320F9008504E39834FF83271F
:10D6C000048013172B01635507002312F900D5BB03
:10D6D0002322F900FDB39D476399F90281451305A3
:10D6E000B0044531BD442320090023220900FD591F
:10D6F0009D3993F77400CA9703C70700FD14398D4D
:10D700002380A700E39634FF6DBBA1476392F90421
:10D710006D398144630D0B008D479304C00363088A
:10D72000FB009304000563048B019304400413750C
:10D73000C507E30895D819453931393905452131EF
:10D7400026850D3909453D314931E31C05D669BBB4
:10D7500091476399F90013056006F536F53E130508
:10D7600090090DB7E38F09D4F154A9BB9731FB1F82
:10D770009381C17F1791FB1F1301C188170500001A
:10D78000130585889735FB1F9385C5871736FB1FC3
:10D790001306C6FD63FAC5008322050023A05500C9
:10D7A00011059105E3EAC5FE170500001305857311
:10D7B0009735FB1F938585FB1386818063FAC5002F
:10D7C0008322050023A0550011059105E3EAC5FE5B
:10D7D00013858180938581816377B50023200500BF
:10D7E0001105E36DB5FEFD42739002BC8D4273904E
:10D7F0004280B72200009382828873900230973271
:10D80000FB1F9382228093E2320073905230970282
:10D8100000009382622B73901234730020300D0647
:10D82000719A81473307F5006393C70082801443E0
:10D830003387F500910714C3F5B7914763EEB7023C
:10D8400017070000130787628A05BA959C41BA97AB
:10D850008287B717004003A7470B1345F5FF698F71
:10D8600023AAE70A03A7070B698F23A8E70A03A7E0
:10D87000070A798D23A0A70A8280B717004083A6E4
:10D88000470B1347F5FFF98E23AAD70A83A6070B88
:10D89000558D23A8A70A83A6070A758F23A0E70A38
:10D8A0008280B717004003A7470B498F23AAE70AD6
:10D8B00003A7070B1345F5FF45BFB717004083A625
:10D8C000470B1347F5FF758F23AAE70A03A7070A3B
:10D8D000598D4DB7B717004003A7470B498FEDB7D8
:10D8E000B71700408847420541819377050491EBC3
:10D8F0009377F5013755E801130505803345F502A7
:10D9000082809377050C130700046397E7009377F1
:10D91000F50137459C1CCDB72165130505D08280E4
:10D92000411122C406C62A84653F2947B307E50290
:10D93000B2408D83B3D7870222449507B3D7E7025D
:10D9400037370040C207C1832316F7404101828068
:10D95000716541111305052006C6D937B737004058
:10D96000130770F82381E7400D47A381E7401307B1
:10D970000004A380E74005472387E740B240410108
:10D980008280411122C491462A84138681809D653C
:10D990002D4506C69730FB1FE780A0A6B7F7070006
:10D9A00003C70701A5476313F70001A09306001002
:10D9B00001469D6525459730FB1FE78080A42384A1
:10D9C00081802244B2409146138681809D6529451D
:10D9D00041011733FB1F6700C3A2130101BF2326B8
:10D9E00011402324814023229140232021411737D5
:10D9F000FB1F0347A7D78D476310F706B7660200E2
:10DA00000146856505459730FB1FE780809F377489
:10DA1000020037A9FDFFB7D4040022851306004099
:10DA20008A85F53BB3052401930600400A86094523
:10DA3000130404409730FB1FE780A09CE31F94FC75
:10DA400005458137B76602000146B77502000545F6
:10DA50009730FB1FE780E09A856782978320C1405B
:10DA600003248140832441400329014013010141E3
:10DA700082800111914670009D652D4506CE97303C
:10DA8000FB1FE78000980347C10089469307F7FF13
:10DA900093F7F70F63E2F6029737FB1F2388E7CC73
:10DAA0009735FB1F83C585CC170500001305453D41
:10DAB0008528F2400561828085471737FB1F2307C1
:10DAC000F7CAF9BF41111305800406C69720FB1F52
:10DAD000E780605C371700408327870A1305002022
:10DAE0008D4593E707202324F70A813B953551376D
:10DAF000ED35B24001454101828081473737004012
:10DB0000A14663C3B70082800346B740E38EC6FEDA
:10DB10003306F5000346060085072304C740D5B742
:10DB20003571CAD813094108A6DAD2D4DAD02EC387
:10DB300086DEA2DCCED6D6D2DECEE2CCE6CAEAC8FB
:10DB4000AA8432C536C73AC93ECB42CD46CF4AC475
:10DB50008145014A170B0000130B4B3683870400E5
:10DB600085E789C5C205C1815285413FF65066549B
:10DB7000D6544659B659265A965A065BF64B664C09
:10DB8000D64C464D0D618280130750026389E70031
:10DB900063140A00268A814585058504C1B791C5AD
:10DBA000C2055285C181913F014A81471307B002E6
:10DBB0009305D002130500031308000293083002F6
:10DBC0008386140013861400638EE6026341D70235
:10DBD000638D0603638E1603138706FD1377F70F15
:10DBE000A54563EDE5060147254529481DA863873E
:10DBF000B600E393A6FE93E7170019A093E7070189
:10DC0000B2847DBF93E74700E5BF93E78700CDBFB0
:10DC100093E70702F5B73307070305062E971307A7
:10DC200007FD83050600938605FD93F6F60FE37462
:10DC3000D5FE830506009306E002639AD50C8305A2
:10DC40001600254593041600938605FD93F6F60FFE
:10DC5000636FD50881462545294805A89305A0028C
:10DC60007D57E398B6FC03270900138624001109A9
:10DC7000E35107FC3307E04093E707015DBFB3863C
:10DC800006038504AE96938606FD838504001386FD
:10DC900005FD1376F60FE374C5FE038604009305B5
:10DCA00080066308B6001376F6FD9305C00463137F
:10DCB000B60085040386040093058005630CB60452
:10DCC00093058007630AB604930750026307F600C2
:10DCD000854548002302F1000D3583870400A9CF54
:10DCE000854548002302F100093D81457DB51305B6
:10DCF000A0028146E393A5FA832609009304260037
:10DD00001306490063D306008146328979B7B2848D
:10DD1000FD5661B793E7070413F607045A8809E62E
:10DD2000170800001308081793FA070163880A0010
:10DD3000F99B9305000201A8FD1445BF13F61700D7
:10DD4000930500037DD6A302B1002303010093FBDA
:10DD500007020326090063830B00791741E61306C7
:10DD600000032306C1008549368C63D336014E8CEF
:10DD7000C58B330487418DE7A28C130D00026341EC
:10DD800090099307F4FF228763530400014733840B
:10DD9000E7408307610089C7854513056100B13BF2
:10DDA00063820B0293070003854513057100A303EB
:10DDB000F100A13393078007854513057100A30384
:10DDC000F100253B639D0A00A28A63435005930737
:10DDD000F4FF22876353040001473384E740930A2A
:10DDE0000003A1A06C0081491375F600429503451C
:10DDF0000500118285092380A500850575F6ADB75C
:10DE0000854513057100A303A101FD1CFD3185BFEC
:10DE1000854513055100D531FD1A45BF85451305CC
:10DE20007100A30351017D1CC939E3C989FFFD5A63
:10DE3000FD196398590193090002634F800011098D
:10DE40006DB57C00CE9783C707008545130571002B
:10DE5000A303F1005D31E9BF854513057100A303FC
:10DE600031017D145939D1BFEAF9FFFF12FAFFFFE2
:10DE70003AFAFFFF52FAFFFF6CFAFFFF496D616744
:10DE80006520466C616720253032780A000000006A
:10DE90003031323334353637383961626364656620
:10DEA0006768696A6B6C6D6E6F707172737475768A
:10DEB0007778797A000000003031323334353637E4
:10DEC00038394142434445464748494A4B4C4D4EF8
:10DED0004F505152535455565758595A000000004C
:08DEE000FF000000000000003B
:10E000006F00E2110000000000180118002801282C
:10E0100002280328002901290229032904290529A6
:10E02000062907290829002A012A022A032A042A84
:10E03000052AA62A78E8060056FD0400F002002012
:10E0400076030020C00200208E0200201C02002067
:10E050005EFF0400A6FF04004C010500D803050084
:10E06000C6040500B4FB040072FA040034FB04008B
:10E07000C4FA0400B60A05000C05002034FF0400B1
:10E0800082070500CC9F0600C4A106003CA2060042
:10E09000F66106002A62060056180600960D060074
:10E0A000A6990600B80705004669060004AA0500FF
:10E0B00092AA0500EAAA050046130500921305007E
:10E0C000FC1105002C660500E6600500C26F050026
:10E0D000927305003E7705001A530500B8520500FB
:10E0E000A0560500665305008E5205001253050028
:10E0F00040520500EA53050042540500F253050062
:10E10000F6530500905405004A5405007C54050060
:10E110009459050098590500E6530500EE53050093
:10E120008E540500965905003E550500065B050016
:10E130008685050004860500428605009068050076
:10E14000A8680500E4680500F24C0500104E0500C3
:10E15000864E05001C320500C22C05000843050050
:10E16000402D05006C3E0500C0C9060040C20600F7
:10E170001CC7060022DD060008DC060094DF06004E
:10E1800084DF06008CDF0600CCDF06005AB40600F0
:10E19000000000000000000000000000000000007F
:10E1A0003CE0060004DA06009AD9060000000000F0
:10E1B000000000000000000000000000000000005F
:10E1C00092830600B0710600367506000E730600D5
:10E1D000647D06004E9A0600000000008EB4060022
:10E1E000440C050066630600266906001E6A0600E8
:10E1F0000000000000000000000000008C6C050022
:10E20000C4820600000000000000000000000000C2
:10E21000607106001C0700203E640600B8DF06009F
:10E22000000000000000000088DF06006403050015
:10E23000E2690500C0DF0600688406003685060036
:10E24000B085060062C70600BCDF0600C4DF06001A
:10E25000220D0600C8DF060026110020EC10002069
:10E2600000000000000000000000000000000000AE
:10E27000000000000000000000000000000000009E
:10E280006373B60082801C419105110523AEF5FE33
:10E29000C5BFB72700203727002093878780130743
:10E2A00047D86373F700828023A007009107D5BF8A
:10E2B0004111B7E700E022C480433707200006C6BB
:10E2C000798C23A0E7180F10000011C199E5B7E77A
:10E2D00000E023A08710014545A893073500C20739
:10E2E000C183F19BC207C183130740036366F70232
:10E2F000372700200325079337270020832687929E
:10E300006391A602372700200327079C69D3C20721
:10E31000DD8D0545029765BF372700200325C7928D
:10E32000E1BF035765002DE7035745006362F70619
:10E33000B72600203306F7402148938686936378FA
:10E34000C8028328050003D86600138687001D8F46
:10E350002A9661172312E6002320160123130600D4
:10E3600010C12312F500130788FF2393E60023133F
:10E37000B50083D566002105B387F5402393F600E9
:10E38000B7E700E023A08710B24022444101828019
:10E390000841BDB7B7E700E003A807003707200032
:10E3A00023A0E7183378E8000F10000001E523A050
:10E3B00007118280B727002003AE0793B7270020FC
:10E3C00003A387928146F28763FC670A83A807004C
:10E3D000636BF50A63E9A80A138787006362E50A9D
:10E3E00003D66700216705076319E600372600207A
:10E3F0000347068905072308E6883726002013050A
:10E40000869383D5470003576500239307001306BF
:10E4100086932E97420741832313E5006387C70342
:10E42000372500200325C5926301F50203D5660058
:10E4300009ED83D7460023A016012107BE95A1054B
:10E440002392B6002313E600B6879843630A670257
:10E45000B726002083A6C6926304D70283566700BE
:10E4600085E283D64700835547001843A106AE9640
:10E470002392D70098C383576600A1072313F600A1
:10E48000B7E700E02DB7BE86C6873DBFB7E700E01F
:10E490009843B706200023A0D718758F0F100000EF
:10E4A00001C599C1814711E6B7E700E023A0E71055
:10E4B0008280B386F50003C80600B306F500850721
:10E4C00023800601E317F6FEC5B737E700E01C43DB
:10E4D000B70620002320D718F58F0F10000019C1B0
:10E4E00091C111E637E700E02320F7108280910503
:10E4F00003A7C5FF11057D16232EE5FEDDB737E71F
:10E5000000E01C43B70620002320D718F58F0F101A
:10E51000000001C53307C50011E637E700E02320FE
:10E52000F71082800505A30FB5FEE31DE5FEF5B7E4
:10E53000B7E700E09843B706200023A0D718758FEF
:10E540000F1000008147B306F5008386060099E6A8
:10E55000B7E600E023A0E6103E8582808507E5B798
:10E5600037E700E01C43B70620002320D718F58FBB
:10E570000F10000001C599C1014711EA37E700E01B
:10E580002320F710054582800507E309E6FE3308DE
:10E59000E500B386E5000348080083C60600E305EE
:10E5A000D8FE37E700E02320F7100145828037E7E7
:10E5B00000E01C43B70620002320D718F58F0F106A
:10E5C00000001307F6FFBA952A966317C50037E7D0
:10E5D00000E02320F7108280FD1503C71500050514
:10E5E000A30FE5FEDDB737E700E01C43B7062000C8
:10E5F0002320D718F58F0F10000001C53307C50081
:10E6000019E637E700E02320F71001458280050571
:10E610008346F5FFE397B6FEE31BE5FE37E700E030
:10E620002320F71005458280797126D2B724002077
:10E6300022D403A4C49806D64AD04ECE52CC56CA91
:10E640005AC85EC662C44DC8372A00203729002048
:10E65000B7290020814BB72A002037CBC901130A04
:10E660000A99130989939389C99D8357240099EFC7
:10E670005C44639A0B0023A6F498032CC400228503
:10E68000113B6284B9A823A6FB00C5BF83A74A98A3
:10E6900082971C443307F5406376F50003A74900D1
:10E6A0001D8F2A979306FB3763ECE60623280900A3
:10E6B0008355240003450400970005E0E78060B11E
:10E6C0005C405844B1C70C4403A64900AE97BE86CF
:10E6D00063E4B70063E4C700B386C74014C4A28BE9
:10E6E0003A8441F4B727002093878793984B894653
:10E6F00063FCE604791798CBB25022549254025925
:10E70000F249624AD24A424BB24B224C4561828066
:10E7100063950B0023A6E4988DB723A6EB00B1BF49
:10E7200003274A0219CB63EDA7003385A74083274F
:10E7300009016374F5002328A900A28B404455B752
:10E7400003A74900BA97D5B723A8070075B7B7271D
:10E75000002003A7479D411122C406C63E8411C371
:10E760000297B727002083C7279893F7F70F99E3FD
:10E77000232A049CB24022444101828001114EC6EA
:10E78000B729002083A7499606CE22CC26CA4AC8BC
:10E7900052C456C281C7829723A20996B72400208B
:10E7A000938744C883C7570037240020938444C804
:10E7B000858B1304449681CF83C774001947631671
:10E7C000F70EA3820400EF0030615C4482971C4482
:10E7D00091C3829737240020372900209307849320
:10E7E0000327899803C61700130A849383478493E9
:10E7F00093961700BA9683D60600F9C2834784938E
:10E8000063E8C70C83A74996230C0492639407120C
:10E81000B727002083A74798638E0710B7270020EB
:10E8200083A7079E2328FA00013583C7B4006393AA
:10E83000071083C7940081CF83C7740093F7F70F45
:10E8400099E7A3840400976006E0E780E007B72714
:10E85000002083A7479BF9CF83270A01E1CF83C715
:10E86000740015476368F70CB7270020938707CD1E
:10E8700083C7C700918BDDEFB727002083C7279898
:10E8800093F7F70FC5EB83461A000326899863CCEC
:10E89000D70A6244F240D2444249B249224A924ADB
:10E8A0000561170305E0670043F183C774001D4746
:10E8B000E31FF7F0A3820400EF0010521C4839B7A1
:10E8C000850793F7F70F230CF492E3E1C7F23DB706
:10E8D00086073E978355070023100700034584935E
:10E8E000B727002083A7079613172500B72A002013
:10E8F000BA979C4323900A98829783D70A98034734
:10E90000849393C7F7FF7D8D93171700032789988A
:10E910003E97835707005D8D2310A700834784939C
:10E9200081C78507230CF4920347849383471A0019
:10E93000E37AF7ECF2406244D2444249B249224AB7
:10E94000924A056182801397170032970357070098
:10E9500075F385072DBF37C700408326C720B7074B
:10E96000FCFFFD17F58F2326F72001000100B727D4
:10E97000002093878793C84F832787262326D72095
:10E980006A0593C7F7FF99835D8D8280B7270020C2
:10E9900003A3079F6303030002831305F00F828024
:10E9A0000327851163000712411122C406C683475D
:10E9B000C5008345E5042A8493F7C70F2306F500B5
:10E9C000834697000356C70013958601618563F15E
:10E9D000C508635A05060345870093F6F607A304A6
:10E9E000D700054693E627006314C50093E6170099
:10E9F0002306D4005C4389075CC3A30AB400032543
:10EA000004112E864C430905513483278411034693
:10EA10005401D44303D7C700B296118FD4C32396B1
:10EA2000E7008947A30DF400B727002003476403DC
:10EA300083C7279A6378F7048347C40093E70701E5
:10EA40002306F40081A093E717002306F40075B7AE
:10EA50009376F60F635D050203458700854513E64F
:10EA600027006314B50013E617002306C400A30AA9
:10EA7000D400A30407008547A30DF4008327841165
:10EA80009C43DDF3B240224401454101828093E77B
:10EA900017002306F400A30AD400A30407000325EB
:10EAA00004114C430905DD328327841103465401C8
:10EAB000D44303D7C700B296118FD4C32396E7007F
:10EAC0008D475DBF05458280B727002083A7C7C655
:10EAD000411122C406C6858B2A84DDEB41651305EE
:10EAE00025F5972006E0E78040E05DC18347A5005B
:10EAF0002315F50083270412B5E72320A41223224F
:10EB0000A41285472311F4042320050083476401E0
:10EB100054412316F5000347D4002304E5000547BC
:10EB2000A304E50037270020032787CA13851702AF
:10EB300015811C437D151375F50F9CC25C43DCC227
:10EB40001C479CC65C47DCC61C4B9CCA5C4BDCCAA1
:10EB50001C4F9CCE5C4FDCCE19CD9386060213076A
:10EB60000702C1BF8327441288C38357240423228A
:10EB7000A412850741BFB7270020938787B403D726
:10EB8000870005072394E700B240224441018280B8
:10EB90008347C40023090400054593C747002306A3
:10EBA000F400DDB78347850193F7E70FDDEB83477B
:10EBB0009501C5EB034625018346C50009CA3727E1
:10EBC0000020834565030347379A63E7E50013F7A1
:10EBD000060149CB014709C6C18A0357E51881C61A
:10EBE0008356251936973DCFB727002003D5479E7A
:10EBF0001307C71237460F00B335A702411113069A
:10EC00000624814622C426C206C67D543305A702C7
:10EC100097D006E0E780E07EB727002083C7779A89
:10EC2000B384A700B727002003A787BD8327070960
:10EC300063F387003E84184375FBB727002083A742
:10EC40004798829781476364A400B307A440B24009
:10EC50002244B3B7970093C7170092443E85410101
:10EC6000828081473E858280B727002003A7C7CADC
:10EC70003C5BFDFF010001008280011122CC4AC8EB
:10EC80004EC606CE26CA52C456C25AC00347B50065
:10EC900085472A842E8983290509631AF71E83571D
:10ECA0000508035BC503372A00209306CA9D83DA53
:10ECB0008600130ACA9D63F4671B834605016390AF
:10ECC000E61A03278511631C07180327450A6318F2
:10ECD00007188346F5001D476393E6180355A503FF
:10ECE000330BFB409307204E33056503832444090F
:10ECF00037460F008146130606243305F502B72771
:10ED0000002083C7679AB3549502B3B5AA02BE9494
:10ED1000C204C180231394083385AA0297D006E069
:10ED2000E780206EB307350133B5A7002E953E87E7
:10ED300083264A0019E163E4D7003387D740B384C0
:10ED40005403B7460F009387F623938606242320A7
:10ED5000E900A697B3D7D702DA97636CF70E1D8F39
:10ED60002320E900B729002083A7499883240900BC
:10ED7000829763E1A4123385A4406350050C83A7F6
:10ED80004998372B0020130BCB9D8297032709004E
:10ED90006368E510198D8357E40303578B008E07D2
:10EDA000B387E7021307003293870719B3D7E70247
:10EDB00063EDA70E374A0F00930AFA23130A0A24B9
:10EDC0008357040485072310F4048347041499E34C
:10EDD0002285512A2285971006E0E78000D87DE140
:10EDE000832604098327C40803274B00B6973E8572
:10EDF00063E4D70063E4E7003385E7408347F40129
:10EE0000835464082328A4088507A30FF4008357BC
:10EE10008B00B384F402D694B3D444036363950C9B
:10EE2000B304954083A7499823209900829763EE05
:10EE3000A40A3385A440E34505F8B727002083C71B
:10EE4000779A63E2A708B727002023A087BE014571
:10EE50009DA883264A00B387F6403E9711B7835496
:10EE6000640837470F009307F723B3845403BE9415
:10EE700093070724B3D7F40263E7F900B387F94097
:10EE80002320F900C5B503274A00BA99C5BF23A0BE
:10EE90003501C9BDB727002083A7079EBE94E1BDF9
:10EEA00083274B00998F3E95FDB5A145228597108C
:10EEB00006E0E780A0C3A305A402B727002083A72C
:10EEC000079C81EF7D55F2406244D2444249B249E9
:10EED000224A924A024B05618280894515458297F4
:10EEE000D5B7B3049740AA9435BF83274B00BE948F
:10EEF00089B72DC901116C0022CC06CE2A84B53BFE
:10EF000029CDFD576305F502372700201307079920
:10EF10005453B2479DC62547637FF700D9173EC6B5
:10EF2000B2450345940297F004E0E7808041F24047
:10EF3000624405618280372700200327079EBA9725
:10EF4000F1BF0347770163E4E700998FC9BFB72694
:10EF5000002083A6069EB697CDBF971006E0E780F7
:10EF6000404DF1B78280797126D206D622D44AD09C
:10EF70004ECE52CC56CA5AC85EC683475503034488
:10EF80007513AA843E941374F40F9307400263F63A
:10EF900087001304B4FD1374F40F03AA841383AA27
:10EFA000C413A38B841222865285D68597D006E09F
:10EFB000E7806042058915E503CBD41201498149F8
:10EFC000337B6403930B50024A865285D68597D0D3
:10EFD00006E0E7804040058915C563916903137415
:10EFE000F90F238B8412B250225492540259F249E1
:10EFF000624AD24A424BB24B456182808509E2099E
:10F0000093D989410509E31179FDE1BF832785097A
:10F0100003560504797193D60701BD8EC206C182DD
:10F02000358E1357764093575640898B058B5D8FED
:10F0300093573640918B5D8F93571640A18B5D8F10
:10F0400093171600C18B5D8F9317360093F7070255
:10F050005D8F931756009355860093F707041E069D
:10F060005D8F1376F60F518F93D7554013D63540E9
:10F07000118A898BD18F13D67540D18F13D6154045
:10F08000218AD18F13961500418AD18F13963500AE
:10F0900013760602D18F13965500137606049E054B
:10F0A000D18F93F5F50FCD8FA20745465D8F3307BE
:10F0B000C70222D42A8426D252CC56CA032A8413E9
:10F0C000832AC4135AC806D63697420741839357FA
:10F0D0007740135557400989858BC98F13553740A1
:10F0E0001189C98F135517402189C98F131517002E
:10F0F0004189C98F1315370013750502C98F131580
:10F10000570093558700137505041E07C98F1377A1
:10F11000F70FD98F13D5354013D755401189098B77
:10F12000498F13D57540498F13D515402189498FD3
:10F13000139515004189498F139535001375050204
:10F14000498F13955500137505049E05498F93F556
:10F15000F50F4D8F2207D98FB387C7024AD04ECE05
:10F160005EC662C4B697C207C18313D7774013D572
:10F1700057400989058B498F13D537401189498F2D
:10F1800013D517402189498F139517004189498F5D
:10F190001395370013750502498F1395570093D5C2
:10F1A0008700137505049E07498F93F7F70FD98FD2
:10F1B00013D5354013D755401189098B498F13D585
:10F1C0007540498F13D515402189498F1395150036
:10F1D0004189498F1395350013750502498F1395A1
:10F1E0005500137505049E05498F93F5F50F4D8F56
:10F1F0002207D98FB387C702130650025285D685DE
:10F20000B697BD8E93940601C18033F6C402137B7A
:10F21000F60F97D006E0E780001C05890DED8347C7
:10F22000D41201498149B3849702130C5002C18062
:10F230004A865285D68597D006E0E780C0190589B1
:10F24000937BF90F11C563863403850993F9F90F90
:10F250000509E31F89FD230B6413B2502254925415
:10F260000259F249624AD24A424BB24B224C4561A2
:10F2700082805E8BCDB70111B727002022CC03A47A
:10F2800087C026CA4AC84EC606CEAA8413092500DE
:10F29000854915C083C7140003473400858B630478
:10F2A000F700405CFDB71946930544004A85EFF02E
:10F2B0002FABE31835FF2285F2406244D244424925
:10F2C000B249056182804111B727002022C403A4FE
:10F2D00087C026C24AC006C693042500054901E836
:10F2E0002285B24022449244024941018280A6858F
:10F2F0001305A402974006E0E780C08DE30225FFD6
:10F30000405CF1BF0111B727002022CC03A407C045
:10F3100026CA06CE2AC42EC6854419E40145F24009
:10F320006244D24405618280834791000347140000
:10F33000858B6304F7000044CDB719469305A100FF
:10F3400013052400EFF0CFA1E31795FE0545C1BFDB
:10F35000EFF0EFBF73000000000000009712000004
:10F36000938262890383020023800200630F0300FB
:10F37000F32510342EC0970500009385A5FD7390EA
:10F380001534EF00A0477300203086DCEF00004703
:10F39000E65082800000B726002003A706C80111AE
:10F3A0004AC81C5F4EC606CE998322CC26CA858BDE
:10F3B0003689B7290020ADCF9307000637240020F7
:10F3C0001CDF930744C883C7670013070008930432
:10F3D00044C86319F70083A7C9C79C4393F7070480
:10F3E0002383F400834744C893F7070489CFB727E2
:10F3F000002083A747988297C8CC834744C893F7D7
:10F40000F70B2302F4C883C7440093F707048DE386
:10F410008547A382F400B727002083A7C7CA370710
:10F42000020098C7130700FC2382E4009848F8D331
:10F43000032709C81C5F9183858B95C31C5F93E7E5
:10F4400007011CDFB727002083A7C7CA054723A2EF
:10F450000706B7270020938747C82382E70083A7C2
:10F46000C9C7D8430583058B19C7D843759BD8C333
:10F47000D843799BD8C3F2406244D2444249B2494E
:10F4800005618280093F730020309317D50063DF48
:10F490000700B727002083A7C7CA7D57B8D7B7276B
:10F4A000002093878793D84F0507D8CF937785009F
:10F4B00099CFB7270020938747C803C72700136752
:10F4C00017002381E700130700F82382E7009377F2
:10F4D000150099CBB7270020938747C803C71700AB
:10F4E00013671700A380E700937765008DC7137734
:10F4F0004500B727002059CF03C747C81367170037
:10F500002382E7C8B727002003A707C85C57F19BF1
:10F5100093E717005CD79317F50063D20702B7276C
:10F520000020138787B483460707938787B4C18A6F
:10F53000BDCA8347070793E707022308F706931717
:10F54000E50063D60702B7270020938747C803C7A3
:10F550004700620761876355070005472382E7007C
:10F56000B727002083A7C7CA3707020098C7931799
:10F57000C50063D00702B7270020938787B403C76D
:10F580001707058B29C303C7170713672700A3882D
:10F59000E7068280938747C803C7370013671700C1
:10F5A000A381E70085B703C7070789463D8B63083A
:10F5B000D70003C707078D463D8BE312D7F81147E5
:10F5C0002388E706ADBF03C71707118B79D303C79D
:10F5D00017071367870065BFB7270020B7260020ED
:10F5E00003A6C7CA938746C803C746C8058B11C779
:10F5F00023820700A3820700828003C71700058BC0
:10F6000065FB785275F303C75700EDB73727002025
:10F61000032807C8832788039583858BC1E311C618
:10F6200083270803BD832300F60085CA832707C804
:10F63000985B4607935767016356070093E707C037
:10F64000C207C18303970600C207C18709C7BA97DB
:10F650000947B3C7E7022390F6009DCD8345150007
:10F6600085CDB7270020938747C883C767001387D6
:10F670009500894593F7070485C33A9583470500AC
:10F680000547994593F6F7066398E600E207E18798
:10F69000814563D30700B9452E8582808545EDBF3E
:10F6A000411126C206C622C44AC0B724002035ED47
:10F6B00083A6C4CAAE87F8527DFF372900201309FC
:10F6C00049C82301090037F400E03E85832704D1AF
:10F6D000B285ED9B2328F4D0832704D193E78702DA
:10F6E0002328F4D073005010975006E0E780E00A1A
:10F6F000B727002083A707C8B70680009843558F17
:10F7000098C3D857719BD8D783A7C4CAA30209004E
:10F71000A3000900094798C3832704D193E7870012
:10F720002328F4D07300501005A08D476314F5040E
:10F73000B727002083A707C8B70680009843558FD6
:10F7400098C3D857719BD8D783A6C4CAB7270020BF
:10F75000938747C803C72700058B19E703C73700FE
:10F76000058B51CB23820700B240224492440249C8
:10F77000410182808547E319F5FCB7F700E003A754
:10F7800007D16D9B23A8E7D003A707D11367870292
:10F7900023A8E7D07300501003A7C4CA8177FD17D0
:10F7A0005447F58F5CC70F10000003A7C4CAB70702
:10F7B0000200130600F81CC7B7270020938747C82C
:10F7C0002382C700B727002083A707C89C439D83D7
:10F7D000858B639FA700930760197CD354C737F7C5
:10F7E00000E0832707D193E787002328F7D01DBFC8
:10F7F0009307E01BDDB7F85231FFBDB7B7270020F4
:10F8000083A7C7CA8847D847798D09C988C7B7274A
:10F81000002003A3878963030300028382803727C4
:10F820000020B7260020138606CB130707CD834799
:10F83000D7008345B601484AAE97FD8BB355F50016
:10F84000A300F600A306F700858995E90347170191
:10F85000814613080002B3F7E7020147B355E500FC
:10F8600085899378F70F89C96395D700A30016019E
:10F870008280850693F6F60F0507E31107FF828065
:10F88000B727002083A74798011122CC26CA52C46B
:10F8900006CE4AC84EC68297B7240020938704CD6F
:10F8A0008047014A6301A406938404CD63668506FC
:10F8B000018D37270020930707CB83C7A701135477
:10F8C0005500137AF501130907CB636BF402B729CE
:10F8D00000209389C99DA1378346A90103A884000C
:10F8E00083A54900139756004297158C3A866364A6
:10F8F00007016364B7003306B74090C4E37DD4FCCE
:10F900001604336A4401F24062445285D2444249AB
:10F91000B249224A05618280B727002083A7079E4B
:10F9200033848740229571B7B727002003A7C7CA41
:10F930008967938707F47CD3B727002083A707D074
:10F9400083A60709139656006358060083A6070985
:10F9500013966600634406007453FDF28280000033
:10F96000B72700203727002083A707930327879214
:10F9700001456313F700828083D6670081E683D652
:10F98000470036959C43F5B7B727002083A5079914
:10F990003727002093870799138605222328C792CB
:10F9A00003D74700938785FFB72600204111BA97F8
:10F9B000056523A4F69206C61D05935637006374A9
:10F9C000E500930600203307D600372500202326C4
:10F9D000E59223A0E522E1162312D60023130600A8
:10F9E0001CC3998FE1172312F700231307008D3FE3
:10F9F000B240B7270020239FA79241018280B727FA
:10FA00000020B726002083A7079303A686922A87A3
:10FA1000B305B5406314F6003A8529A8938687009C
:10FA20009C43E369D7FEE377F7FE2E85E3E4D5FE3A
:10FA3000E3F2F5FE828023AC05FE1C4191E7010054
:10FA400001000CC18280BA8703A787FF6DFF23AC3A
:10FA5000B7FE8280184183A785FF6319B7001CC1D8
:10FA6000FD5723AC05FE238FF5FE8280232CF6FE86
:10FA7000C5BF411122C437E400E026C20440370765
:10FA8000200006C6F98C2320E4180F10000009E9B5
:10FA9000232094101545B2402244924441018280B3
:10FAA0000347E5FF9307F00F6306F7002320941048
:10FAB0001145D5B79700FB1FE7800067014523205C
:10FAC0009410D1BF411126C2B7E400E04AC003A997
:10FAD0000400B707200006C622C43379F90023A02A
:10FAE000F4180F10000009E923A02411B2402244A9
:10FAF00092440249410182809565938505D0C98D64
:10FB00002A842105C2054205C18141819700FB1F5E
:10FB1000E780405301CDFD572320050023128500C7
:10FB20002303F50023A024112105C9B723A0241124
:10FB300001456DBF0111B7E700E04AC803A90700FE
:10FB40004EC63707200006CE22CC26CAAA893379B2
:10FB5000E90023A0E7180F10000037250020032438
:10FB600045938144014619E499E8A1654E85EF006B
:10FB7000B00631A88347E4FF6397370395C8A6858D
:10FB800013054593C13D75D0A1654E85C92EF24040
:10FB90006244B7E700E023A0271126854249D244FA
:10FBA000B2490561828091E02286032484FF65BF0B
:10FBB000A284E5BF41114AC037E900E022C4032412
:10FBC00009003707200006C626C2798C2320E918D1
:10FBD0000F10000089E523208910154515A0B727CF
:10FBE000002083C79793AA842E8563F5F400894784
:10FBF00063EE9700BD3DB7E700E023A087100D45F9
:10FC0000B2402244924402494101828083A785FF89
:10FC100099E703C7E5FF9307F00F6308F700913DED
:10FC2000B7E700E023A087104DBF37250020238FC2
:10FC300095FE130545930135A16526850D260145E1
:10FC40002320891075BFB727002023AA079282803E
:10FC5000B727002083A7C79899E33E85828003D702
:10FC600027006316B70003C70700E308A7FEDC47B9
:10FC7000E5B7B9CD011106CE22CC26CA8147C146CF
:10FC800033D7F540058B21C312053E953147330527
:10FC9000E502372700208324079D05443314F40030
:10FCA0002EC642044180AA949C40C8408297B24527
:10FCB00023A0040023A20400A18DF2406244D24498
:10FCC0002E85056182808507E39CD7FA0144EDB754
:10FCD0002E858280BDCD797122D406D626D24AD017
:10FCE0004ECE01444147B3D78540858BB1CF120535
:10FCF000314722953305E502B727002003A9079D68
:10FD00008544B3948400C204C180BE892A99032724
:10FD1000090011C7032549002EC60297B245314795
:10FD20003304E40283A7099D3E941C4489E7232001
:10FD3000090023220900B2502254A58D0259925481
:10FD4000F2492E85456182800504E31EE4F8814472
:10FD5000DDB72E8582804111B7E700E026C28443DB
:10FD60003707200006C622C4F98C23A0E7180F101D
:10FD70000000B727002083A7079B37140020130437
:10FD8000847D91C782971C403E9508C031A0B7275B
:10FD9000002083A74798FDF70840B74703009387E3
:10FDA000D73F3305F502B7A72600938737ECB2405B
:10FDB0003E9508C02244B7E700E023A09710924484
:10FDC000410182800111B7E700E022CC80434AC89C
:10FDD0003707200006CE26CA2A892E86798C23A0D2
:10FDE000E7180F100000131506019305F004418178
:10FDF00032C69700FB1FE780E024AA8419C532466B
:10FE0000CA859700FB1FE780A041B7E700E023A069
:10FE10008710F240624426854249D24405618280BF
:10FE20007971B7E700E022D480433708200006D676
:10FE300026D24AD04ECE52CC56CA5AC85EC662C4EA
:10FE40003374040123A007190F10000005E123A05B
:10FE500087100945B250225492540259F249624A1D
:10FE6000D24A424BB24B224C45618280B7270020D8
:10FE700083A74798BA8A368AB28B2E8BAA89829733
:10FE8000B727002003A7079D3E898144B146C1479B
:10FE9000338CD40233068701104241E6C165938555
:10FEA00005F041459700FB1FE780C01919EDB72702
:10FEB000002083A7079C81C7814511458297B7E73A
:10FEC00000E023A087102D4571B7B727002003A7B6
:10FED000C79821E723A6A798230005008327099D3B
:10FEE00005473317970023260500232475012311A6
:10FEF000E50023225501E29723A0370123A26701E1
:10FF000023A4570163040A0023009A00B7E700E026
:10FF100023A0871001453DBF3E875C47F5FF48C7DA
:10FF200065BF8504E396F4F6B7E700E023A08710E9
:10FF300021450DB7B727002083A7879D411122C413
:10FF400006C6372400201304849389C782975C482F
:10FF50003E9548C84848B240224441018280B7E7F4
:10FF600000E09843B706200023A0D718758F0F1024
:10FF70000000B726002083C696936372D502372609
:10FF800000209316150003258698369583560500A4
:10FF9000D58D2310B50023A0E7100145828023A052
:10FFA000E7100D458280B7E700E09843B7062000D0
:10FFB00023A0D718758F0F100000B726002083C626
:10FFC00096936374D50237260020931615000325F7
:10FFD000869893C5F5FF369583560500F58D231059
:10FFE000B50023A0E7100145828023A0E7100D454E
:10FFF0008280011137E700E026CA0443B7062000DB
:020000040005F5
:1000000006CE22CC4AC84EC652C4F58C2320D7183F
:100010000F100000130705FF1377F70FFD4763E28A
:10002000E70AB146B306D502B727002003A7079D0C
:1000300036971C43D9C71359450005443D893315EC
:10004000A400131405014180AE894A85A2850931B7
:100050002A8A39C9A2854A85B937B727002083A7DC
:100060004798372900201309C99D82978357890033
:100070002A848146B385370313060064B3B7370378
:1000800013850532B335B500BE95EFE04110B307D7
:1000900085003E878326490063E4A70063E4D70018
:1000A0003387D7402324EA00B7E700E023A0971066
:1000B0000145F2406244D2444249B249224A0561B4
:1000C0008280B7E700E023A097100945DDB7011152
:1000D000B7E700E026CA84433707200006CE22CCCB
:1000E0004AC84EC6F98C23A0E7180F100000BD4780
:1000F00063E8A70431473307E502B727002083A749
:10010000079DBA979C438DCF05443314A400420445
:1001100041802E890145A285253EAA8911C5A28567
:100120000145513523A42901B7E700E023A097102A
:100130000145F2406244D2444249B249056182809D
:10014000B7E700E023A097100945E5B779714AD0D9
:1001500037E900E026D283240900B707200006D63D
:1001600022D44ECE52CC56CA5AC85EC6FD8C23202D
:10017000F9180F100000B727002083C79793637802
:10018000F500B727002083AB479863970B00B7E7CC
:1001900000E023A0971099A0B72900209389C99D5A
:1001A000AE8A03AB490083D58900B74736FE9387F3
:1001B00007C83E9BB387C5022A84328A8146B3B5FD
:1001C000C50213850732B337F50013060064BE95E8
:1001D000EFD0F17B6370AB02232099100145B25040
:1001E000225492540259F249624AD24A424BB24BCB
:1001F00045618280829B83D589002A891306006429
:10020000B38745038146B3B5450313850732B3373A
:10021000F500BE95EFD0B177B30725013E8903A75E
:10022000490063E4A70063E4E7003389E740D6852B
:100230002285393C09C923242501B7E700E023A022
:100240009710054569BF936504F0C205C18141451A
:100250009700FB1FE78000DF11E9B727002083A785
:10026000079C95D7A2851145829715B7372700209F
:100270008327C79895E32326A7988547232605005B
:10028000232425012311550123008500A300F50037
:10029000232205005DB7BA87D84775FFC8C7F1BFED
:1002A0007971B7E700E026D284433707200006D6ED
:1002B00022D44AD04ECE52CC56CA5AC85EC662C468
:1002C00066C26AC0F98C23A0E7180F1000002DC188
:1002D0004144B689B28A2E8A2A89B14C372B002034
:1002E000054D130C0003B30B940303270B9D5E977E
:1002F0001C43A5E39375F400B315BD0013554440AA
:10030000C2055686C1811375F50F893539C183271A
:100310000B9DDE9723A0270123A2470163840900D8
:1003200023808900B7E700E023A09710014521A0B2
:1003300023A097100945B250225492540259F24911
:10034000624AD24A424BB24B224C924C024D45611A
:1003500082800504E31984F9B7E700E023A0971031
:100360002145D1BF0111B7E700E026CA844322CC62
:100370004AC84EC63707200006CE2A84AE89328985
:10038000F98C23A0E7180F100000C9332285CE8511
:10039000C1302A8405C5B727002083D5479E1306A0
:1003A00000648146B3872503B3B52503138507325F
:1003B000B337F500BE95EFD0915D48C013351400FA
:1003C000F2406244B7E700E023A097104249D244CC
:1003D000B2490E05056182800111B7E700E04AC805
:1003E00003A9070022CC4EC63707200006CE26CA36
:1003F000AA892E843379E90023A0E7180F100000A2
:10040000EFF01F85AA8419C123110500A2854E852E
:10041000593EB727002083C7879363993701B727D1
:10042000002003D70798598C23908798B7E700E0FE
:1004300023A02711014591E01945F2406244D244BE
:100440004249B2490561828001114AC837E900E09A
:1004500022CC03240900B707200006CE26CA4EC6C8
:100460007D8C2320F9180F1000009307F00263E63B
:10047000A704B147B304F502B729002083A7099D5B
:10048000A6979C439DCB9377F5008545B395F500E2
:10049000C205C1811181893783A7099D0145A697AE
:1004A00023A0070023A2070023208910F240624402
:1004B000D2444249B24905618280B7E700E023A0F7
:1004C00087100945E5B74111B7E700E026C284432C
:1004D00006C622C437072000F98C23A0E7180F10A6
:1004E0000000EFF0EFF619E90145B2402244B7E70A
:1004F00000E023A09710924441018280B72700209A
:1005000083A7479800458297B72700209387C79D08
:100510006368A402D843B74636FE938606C83305FF
:10052000A4403697E372E5FC13070064B335E50297
:1005300003D6870081463305E502EFD0514575B7F4
:10054000D8433A94C1BF411122C426C237240020A7
:10055000B72400201307C49D938484939448584380
:10056000B727002006C683A747981304C49D63924B
:10057000E60882975440B74736FE938707C8B69778
:100580003387A7003A856364F7006364D7003305B7
:10059000D740B7240020938744C8DC53938444C8D1
:1005A00099CBB727002083A607D03707CDFF7D174B
:1005B0009C46F98F9CC611E14840B727002083A7CD
:1005C000479B829719E5DC5085C3EF60215CEF50B3
:1005D000B15ADC5091CBB727002003A707D0B7064C
:1005E00033001C47D58F1CC7B240224492444101BE
:1005F0008280829794485840B387A6003E8563E482
:10060000D700E3E8E7F83385E74061B74111B72742
:10061000002006C623ACA79C0295B240B727002055
:1006200023A8A794014541018280994763E9B70057
:10063000B72700208A0593874796BE9588C1828098
:10064000B727002023AAA79C11C5B727002005477C
:100650002381E7988280B727002023A60798B72731
:10066000002023AC079CB727002023A2079837253A
:100670000020B72700204111238107987146B72732
:10068000002081451305459606C623AA079C22C46F
:1006900026C2372400209700FB1FE78080BF130588
:1006A00084931306800281459700FB1FE78060BE9C
:1006B000EFF08FADB72700209387079903C5C703D5
:1006C00083C7D7031304849385453E958D4733052F
:1006D000F5029947B724002039051375F50F23015A
:1006E000A4003305F502130505249700FB1FE780DE
:1006F000609523A8A49C49C10346240099478145DD
:100700003306F602130606249700FB1FE78060B845
:1007100083A7049D03472400B72400209387072460
:100720000A0723A0F496BA97372700202324F798C6
:10073000EFF06FD1A5218347140083A604963706F6
:100740000500139727003697130646CD10C313876D
:1007500017001377F70F0A073706050036971306B9
:1007600026C710C313873700890793F7F70F8A0747
:10077000A300E400B69790C3B240224492444101E2
:10078000828037270020130787938347170083460B
:10079000270063F0D702B726002083A606961386AB
:1007A0001700A300C70013972700369708C33E859C
:1007B00082809307F00FE5BF1C41638C07104177DF
:1007C0007D8FB706002089476316D7100357450071
:1007D00063020710411126C21946AA849305F00F3F
:1007E000610506C622C49700FB1FE78000B90547D4
:1007F0008D47630AE50C9C4491C7D858994761C757
:10080000985C71C33724002013060004814513054A
:1008100004999700FB1FE780C0A713060004A68574
:10082000130504999700FB1FE780809F93070499A5
:1008300003D7C70009E7130700102396E70003C793
:10084000E70001E705472387E70003D7070101E732
:100850006D472398E70003C7F70001E71547A38713
:10086000E70003C7270101E705472389E70003C71E
:10087000370109E703C7F700A389E70003C757015A
:1008800001CB937637000983238ED702A38EE7022C
:1008900003C7470101E75547238AE70003C76401FF
:1008A00009E71307C003238BE7009C5791C7829782
:1008B000B72700202390A794B72700207D57A38255
:1008C000E7D6513B8147B240224492443E854101E4
:1008D000828089473E85828001114AC837290020DD
:1008E0008327C99D06CE22CC26CA52C456C24EC604
:1008F0008297130A0064B33545031309C99D835ACF
:1009000089008146568633054503EFD05108B72745
:10091000002013878793004FAA8401456306940241
:100920009389879333858440636E9400032549003F
:1009300056868146B335AA023305AA02EFD03105A7
:10094000018D269523AC9900F2406244D24442497D
:10095000B249224A924A05618280011122CC2E843A
:10096000B7E506000A8541469385C55D06CEEFD002
:10097000913B180806043A94B7270020035504FF5A
:1009800083D7679EF2406244AA9737450F0013054C
:1009900005243355F50205618280B727002083D7EF
:1009A000679E51471D45637CF70279471945637877
:1009B000F7021307200315456373F7021307B0040A
:1009C0001145637EF700130740060D456379F70074
:1009D0001307600909456374F70013B5B70F8280E8
:1009E000011122CC06CE2A842EC6EFF0CFB6B24536
:1009F000F240818D33A5A502229562441375F50F4F
:100A000005618280011122CC06CE2A842EC6EFF029
:100A10008FB4B245F240818D33A5A5022295624480
:100A20004205418105618280011122CC06CE2A84D3
:100A30002EC6EFF04FB2B245F240818D33B5A5021C
:100A40002295624405618280B727002013870799A9
:100A500018572DC3411122C426C24AC006C61389A5
:100A600007990297B72700201387879303578700BA
:100A70002A84938487930DCBBA876373A700AA87D0
:100A8000C207C183BA866373E400A286C206C1822C
:100A9000958F5147635AF7008327C90291C3829704
:100AA000EF50F17723948400B240224492440249EB
:100AB0004101828082800111B727002022CC372497
:100AC000002023A8079E93070499DC5706CE26CA68
:100AD000AA851304049981C72AC68297B245C9C161
:100AE0009C410545ADCBDC41BDC783D78500A5C77B
:100AF00083D7A500ADC3B72400201385C49D5146FC
:100B00009384C49D97F0FA1FE780807123860400C8
:100B1000B727002083A6C79D372700202322D79818
:100B2000034774011DE39387C79D03D5870093078F
:100B3000805737460F003305F50213060624814619
:100B40008145EFD0C164A30BA40037150500130540
:100B5000858D6D3C0145F2406244D244056182803E
:100B6000B7270020938787933707002023AE07001D
:100B70001307676EB727002023AEE79C3787320044
:100B80009387C79DFD56130727A1D4C398C7238613
:100B90000700B7C7004023A4D7269DBF011122CC70
:100BA0003724002093070499884706CE26CA4AC8EE
:100BB00001E90545F2406244D24442490561828020
:100BC000130404995C58F5D7185C65D77000854507
:100BD00082971844B247E30EF7FC0355C40093050F
:100BE000E004B724002097F0FA1FE780A0451387A0
:100BF000849308D3938484934DDD0356C4009305F6
:100C0000F00F014997F0FA1FE780A0688347E400DE
:100C10009050634DF900328597F0FA1FE780C0507D
:100C2000014523A0040223A2040269B78355C4002E
:100C30000844185CB3872503898105093E9508C2DD
:100C40000297E9B701114EC6B72900209387099989
:100C50009C4726CA4AC852C406CE22CC56C25AC0A5
:100C60002A8AAE843289638D071E9389099903A766
:100C70004903630407121307F01F6362A7123724A6
:100C8000002013078493832A070213048493639A32
:100C90000A0803D5C9009565938515E097F0FA1FFA
:100CA000E780403A08D02A866DC983D5C90083A75A
:100CB000490303A589008981829783A78900832A34
:100CC00004025CD089476316FA08C1476397F40CA5
:100CD00083D5C9009147938505FCB3C5F5028A0504
:100CE000D69503C725009307A0056314F70A83D799
:100CF00005006390470B4A852686910597F0FA1FF9
:100D0000E78000521C505685639357130145F2400B
:100D10006244D2444249B249224A924A024B056196
:100D200082805850E380E7FA03D5C9009565938522
:100D300025E097F0FA1FE780E030AA8A39CD83D505
:100D4000C9002A8683A7490303A589008981829760
:100D500095BF8D47631BFA00C1476390F40483D5A8
:100D6000C900938545FDF199A5BF91476318FA0025
:100D70006395440383D5C900A115F5B79307001007
:100D8000631DFA00A14763EA970083D5C900C11526
:100D9000D9BF1C5056856390570D29458DBF9D6A5C
:100DA000637C5509930A05E01947B3CAEA0203D7E1
:100DB000C900372B0020B38AEA02BE9A93078B93AF
:100DC000DC53130B8B936395570103240B021DE037
:100DD00003D5C9009305E00497F0FA1FE780802649
:100DE0002A8445DD83D5C90083A749032A868981E2
:100DF0005685829791451307A00589819397250011
:100E0000A29783C627006393E60483D60700639CFA
:100E1000460385058A052686A2954A8597F0FA1F1E
:100E2000E780004083270B02E38287EE228597F05C
:100E3000FA1FE780602FD9BD21677917E36FA7F408
:100E4000B30A5541ADB783C5370045BF83270B02B1
:100E5000E38587F4228597F0FA1FE780E02C35BF01
:100E6000B727002083A587958DD991479306A005C4
:100E70008983139727002E9703462700E31FD6F098
:100E800003560700631C460185078A072686BE9520
:100E90004A8597F0FA1FE780A0388DBD8347370059
:100EA000C1BFB727002093870799984729C3985F48
:100EB0001DCF8546631DD502411122C43724002071
:100EC00013048493105006C619CE83D5C70048502A
:100ED00089810297085097F0FA1FE780E0242320C9
:100EE000040223220402B240224441018280828013
:100EF000011122CC372400209307049956C283AAFB
:100F0000870026CA4AC84EC606CE52C42A89AE8475
:100F1000B28913040499638C0A1C1C5C99EB294563
:100F2000F2406244D2444249B249224A924A05619F
:100F300082805C58EDD79307F01F63E8A70C372A2F
:100F4000002093078A939C53130A8A93B9C70844D5
:100F500083274A02639FA70489476317F906C1479D
:100F6000E39FF4FA0355C4009147130505FC33458C
:100F7000F5029317250003250A022686CE853E95A5
:100F80009307A0052301F50023102501110597F013
:100F9000FA1FE780E028014561B70355C4009305B7
:100FA000E00497F0FA1FE780E0092320AA0245F148
:100FB000BDB78355C4005C5803260A028981829715
:100FC0001C442322FA0249BF8D47631CF900C14724
:100FD000E397F4F40355C400130545FD9377C5FF6B
:100FE00059BF91476318F900E39B24F30355C400EC
:100FF0002115EDB793070010E313F9F2A147E3E0E1
:1010000097F20355C4004115D1BF9D676378F5067B
:10101000930705E01947B3C7E7020357C400372A0F
:101020000020B387E702BE9A93078A939C53130A62
:101030008A93A1CF83274A026395570703250A02A3
:1010400091461308A0059305F00F93D72600139738
:1010500027002A97034627006316060783580700D0
:1010600003463700639C2805B306D64063C6960442
:1010700085078A072686CE853E9511BF2167791799
:10108000E36FA7E8B307F54049BF0355C4009305D4
:10109000E00497F0FA1FE780E0FA2320AA0259F94A
:1010A000BDBD8355C4005C5803260A02898156855C
:1010B000829723225A0359B72310B70093160601CB
:1010C000C18261B70356C400B3859600910513062B
:1010D00006FCE3F6C5E413863400719A1106B29655
:1010E0002301070123102701A301D70051B7372A95
:1010F000002093078A939C53130A8A93A9C303255C
:101100000A0291461308A0059305F00F93D7260015
:10111000139727002A970346270063140605835870
:1011200007000346370063982801B306D640E3D191
:1011300096F42310B70093160601C182C1BF034580
:10114000E4008357C4009305E0043305F50242052B
:10115000418197F0FA1FE780E0EE2320AA0245F1D3
:101160007DBB0356C4008345E400B385C5023386C6
:1011700096001106E3E5C5DAB9BF0145828083C751
:1011800005002300F50083D72500A300F50083D7D1
:101190002500A1832301F50083C74500A301F500C5
:1011A00011458280B727002023A60780B72700209B
:1011B00023A40780828029C1411126C206C622C409
:1011C000AA8401458DC52E84B7E5060022854146D7
:1011D0009385C55E97F0FA1FE780800483C70400FB
:1011E00005452306F40083C71400A306F400B240AB
:1011F000224492444101828001458280011122CC27
:1012000026CA06CE0947AA8432846381E504414692
:101210008147639BC500638FE6006397B6000DA806
:1012200041478147638EE600F2406244D2443E85E6
:10123000056182808A852285BD3F41468A8519A83D
:101240008A85953F41468A85228531A0E39AB6FC7E
:101250002E86A285268597F0FA1FE780A009AA8727
:10126000E1B7B727002023A4A7808280B7270020FA
:1012700023A6A7808280011122CC0354650006CEEC
:1012800026CA4AC84EC641C083298500AE842A8832
:1012900003C9090081471317890161876355070254
:1012A000B147054563FA87045114420403552800E9
:1012B000418033878900A2864E868545EFA0900C39
:1012C000B337A00085077D141355690042040589D2
:1012D0001379F90341802380F400A380A4002381C3
:1012E000240123928400014719C01387190098C470
:1012F00009476383E7000145F2406244D244424912
:10130000B249056182800545C5BFC167F917630A07
:10131000F502D94763F7B702011122CC2EC606CEDB
:101320002A84EF703055B2456368B5002285624467
:10133000F24005616F90E078F24062440545056136
:10134000828005458280C167F9176314F5006F70CC
:101350007052411106C6EF90806511E15D45B240C3
:101360004101828091476394F50283470500230081
:10137000F6008347250003471500A207D98F2311E4
:10138000F6008347350001452302F60082801145AF
:1013900082804111814522C426C206C6AA84052541
:1013A0002A8409E9B727002083A7878081C7F945E8
:1013B000268582972285B240224492444101828050
:1013C00039714ED656D25AD006DE22DC26DA4AD8F9
:1013D00052D4AA8A2E8BB28941EF36C6AD379145D9
:1013E000EF70105BAA844D492DC9B246054A23808F
:1013F00034010544630A0B00B68513851400029B73
:101400000505131405014180E20993D9894163D38D
:101410000902C1455685EF90C067654905E93386E5
:101420008400A2852685EFA000472A8905E13104C2
:101430004204418091472C085685231CF10026CE9A
:10144000231D8100EF8010702A8901C963070A00FB
:10145000268597F0FA1FE78020CDF25062544A8526
:10146000D2544259B259225A925A025B2161828067
:10147000BA84014AADBF011122CC26CA4AC84EC661
:1014800006CE2A893284B689253FAA840DE1B72782
:10149000002083A7C78081CF05476317E40003C4FA
:1014A000090005041374F40FA2854A858297F2405F
:1014B000624426854249D244B24905618280AE86A3
:1014C000B7150500014705469385E5176DB783D726
:1014D00005002300F50083D70500A183A300F500D4
:1014E0000945828083D705002300F50083D70500D6
:1014F000A183A300F50083D725002301F50083D73E
:101500002500A183A301F5001145828083D7050042
:101510002300F50083D70500A183A300F50083D73E
:1015200025002301F50083D72500A183A301F50041
:1015300083C755002302F50083C76500A302F500A9
:1015400003D58500190542054181828083D70500B6
:101550002300F50083D70500A183A300F50009450A
:10156000828083D705002300F50083D70500A1837F
:10157000A300F50083D725002301F50083D72500BC
:10158000A183A301F5001145828003D5450006051E
:1015900042054181828083D705002300F50083D76F
:1015A0000500A183A300F50003D525000905420528
:1015B0004181828083D705002300F50083D7050091
:1015C000A183A300F50083D725002301F50083D76D
:1015D0002500A183A301F50003D5450011054205AF
:1015E0004181828083C705002300F5000545828084
:1015F00083D70500411122C406C62300F50083D716
:1016000005002E841105A183A30EF5FE83D72500C6
:101610009505230FF5FE83D7D5FFA183A30FF5FE14
:1016200003C6F5FF97F0FA1FE78080BF034544002B
:10163000B24022441105410182808947639CF50034
:1016400083471500034705000145A207D98F2310E2
:10165000F60082801145828003D70500D94763FEDA
:10166000E702011122CC06CE2EC62A84EF7090200C
:10167000B24683D70600636DF50022856244F240CE
:10168000B7150500014709469385E54C05610DBB7B
:10169000F240624409450561828009458280914794
:1016A0009DC583460500FD15C2058547C18163922E
:1016B000F60213D725008D89914791E9914701CB17
:1016C00005052301D6002310E60048C281473E8568
:1016D000828009479147E39CE6FEC94733D7F5026C
:1016E000B3F5F502D1BFAE86B71505000147114627
:1016F0009385454EF1B193F7350091EB8981914780
:1017000089C52310B60048C281473E858280914733
:10171000EDBF03C745008947631AF702011122CCC8
:101720002A84C84506CEAE86014719C52EC69D45FA
:10173000EFE0EFACB2462A8722856244F240B7154B
:10174000050019469385C55005619DB909458280FC
:1017500099E1114582808347050005472311F60072
:10176000E379F7FEFD1593F5F50F33D7F502B3874F
:10177000E702E390F5FE050548C22310E6000145A7
:10178000828083C745000947AE866385E7004147ED
:101790006399E700B7150500014721469385055F6A
:1017A00005B1094582802310B60091E1014548C288
:1017B00001458280AE86B71505000147294693850D
:1017C000C554FDBE2310B60091E1014548C2014554
:1017D0008280AE86B71505000147314693852556B0
:1017E000C5B62310B60091E1014548C2014582808B
:1017F00003D74500854763FDE702011122CC2A8407
:10180000884106CE0DC12EC68545EFE04F9F2A8741
:1018100022856244B246F240B715050039469385E9
:10182000A558056171BEF240624409450561828098
:101830000945828091479DC5034705008D46914724
:1018400063F2E602FD15C205C181B3C6E5023308A5
:10185000D7026399050105052310D6002311E60080
:1018600048C281473E85828083C745000947AE86CE
:101870006385E70041476399E700B7150500014715
:1018800041469385055F2DBE09458280B335B00082
:10189000139525008280011122CC26CA06CE03C7EB
:1018A00085008547AA842E8449466310F702613C6F
:1018B0008357240049151306200963C8A700F24086
:1018C0006244D244094505618280034794008547FC
:1018D0006314F70013660604484011C58D4532C6EF
:1018E000EFE0EF913246A2866244F2402A872685D5
:1018F000D244B7150500938565590561D1B48D476C
:1019000063FFB7028347150003470500F115A207DF
:10191000D98F2310F6008347350003472500C20501
:10192000A207C181D98F2311F6002312B60089C501
:10193000110508C60145828023240600E5BF114534
:101940008280011122CC2A84884506CEAE8611C53C
:101950002EC69545EFE0AF8AB2462A8722856244BB
:10196000F240B715050059469385455B056189BC72
:10197000B335B000139525008280AE86B7150500FB
:10198000014761469385455E25BC8547114563F453
:10199000D7028347160083450600A207CD8F231088
:1019A000F7009387E6FF2311F70089476386F60067
:1019B000090650C30145828023220700E5BF014785
:1019C000814679468145EDBA83D705002300F500AD
:1019D00083D70500A183A300F5000945828083C752
:1019E000250005472300F50003D505006397E700B0
:1019F0000A050505420541818280C9473305F50284
:101A0000CDBF03D505000A0542054181828083D7F9
:101A100025002300F50003D5050083D725003305F5
:101A2000F502050542054181828003D505008280CB
:101A300003D50500828003D50500828083D7250069
:101A40002300F50003D5050083D725003305F502F3
:101A5000050542054181828083D705002300F500FA
:101A600083D70500A183A300F50083D725002301B8
:101A7000F50083D72500A183A301F50003D5450018
:101A8000110542054181828083D705002300F500BE
:101A900083D70500A183A300F50003D52500090520
:101AA00042054181828089471145639BF600834747
:101AB0001600834606000145A207D58F2310F700C4
:101AC000828003D70500D947AE8663F9E700B725C2
:101AD000050001470D469385859C71BA09458280B2
:101AE00011456393A602834716008346060001450D
:101AF000A207D58F2310F7008347360083462600C0
:101B0000A207D58F2311F700828083C725000547E0
:101B1000FD1793F7F70F6361F70483D705008DCFA7
:101B2000011122CC2A84C84106CE15C12EC6894592
:101B3000EFD0FFEC2A8722856244B246F240B725F7
:101B4000050015469385E59D05616FF0DF92F24033
:101B500062440945056182800945828095471145A7
:101B600063F9D706411122C426C24AC006C683477C
:101B70001600BA8403470600A2073284D98F239047
:101B8000F400834736000347260093054400A2076C
:101B9000D98F2391F40089472382F40009461385E5
:101BA0005400368997E0FA1FE78080679307A9FF02
:101BB0002394F4009947631BF90023A60400B24064
:101BC0002244924402490145410182801904C0C463
:101BD000FDB7828083D705008DCF011122CC2A84E6
:101BE000C84106CE15C12EC68545EFD05FE12A87D4
:101BF00022856244B246F240B72505001D46938512
:101C000025A005616FF03F87F240624409450561F8
:101C100082800945828099476395F604894741117E
:101C200006C62302F7008347160083460600B285E6
:101C3000A207D58F2310F70083473600834626007E
:101C400003464700A207D58F130557002311F7005D
:101C5000910597E0FA1FE780A05CB2400145410181
:101C60008280D14711456394F600C1474DBF828001
:101C700083D705008DCF011122CC2A84C84106CE1E
:101C800015C12EC68945EFD09FD72A872285624489
:101C9000B246F240B725050025469385E5A00561CB
:101CA0006FF06FFDF240624409450561828009458D
:101CB000828089471145639BF6008347160083465F
:101CC00006000145A207D58F2310F700828001117D
:101CD00022CC2A84C84106CEAE86014719C52EC63D
:101CE0008545EFD0DFD1B2462A8722856244F24093
:101CF000B72505002D469385A5A205616FF0AFF7C6
:101D000011456393A60283471600834606000145EA
:101D1000A207D58F2310F70083473600834626009D
:101D2000A207D58F2311F7008280011122CC2A84CB
:101D3000C84106CEAE8611C52EC68545EFD03FCC34
:101D4000B2462A8722856244F240B725050035460F
:101D5000938505A305616FF00FF293F71600114507
:101D600089EB89476387F60085822312D70010C369
:101D700001458280011122CC2A84C84106CE15C1BA
:101D80002EC68545EFD0BFC72A8722856244B2465A
:101D9000F240B72505003D46938565A305616FF0C8
:101DA0008FEDF240624409450561828083D70500CA
:101DB0008DCF011122CC2A84C84106CE15C12EC672
:101DC0008945EFD0DFC32A8722856244B246F240BC
:101DD000B725050045469385C5A305616FF0AFE9BA
:101DE000F240624409450561828009458280854749
:101DF00063FCD7022304A700A304B700834716009F
:101E000083450600A207CD8F2310F7009387E6FFD6
:101E10002311F70089476386F600090650C3014580
:101E2000828023220700E5BF114582800147814659
:101E30004D4681456FF02FE48D47114563FBD70276
:101E40008347160083450600A207CD8F2310F700B5
:101E50008347360083452600A207CD8F2311F70064
:101E60009387C6FF2312F7006386A600110610C7EA
:101E70000145828023240700E5BF011122CC2A847A
:101E8000884506CEAE8611C52EC69545EFD03FB724
:101E9000B2462A8722856244F240B72505005D4696
:101EA000938585A505616FF00FDD85471145639723
:101EB000F6008347060001452300F70082800147B2
:101EC0008146654681456FF00FDB011122CC2A84E3
:101ED000C84106CEAE86014719C52EC68D45EFD046
:101EE0001FB2B2462A8722856244F240B725050018
:101EF0006D46938585A805616FF08FCC011122CCCA
:101F00002A84C84106CEAE86014719C52EC68D4526
:101F1000EFD0FFAEB2462A8722856244F240B72551
:101F200005007546938585A805616FF06FC901119D
:101F300006CE2EC6EF80D02301C9B245F24003552C
:101F4000250005616FC0102EF24049450561828071
:101F5000B7270020A38C0782B7270020238C078295
:101F6000B727002023A00782B727002023A20782DB
:101F7000B727002023A40782B727002023A60782C3
:101F8000B727002023AE0780B727002023AC0780A7
:101F9000B7270020239A07A013064038938747A14C
:101FA0002391C70271761307400B130606B82391DD
:101FB000E7002392C70211671D46930600059305AB
:101FC000000A1305007D2392E7002393C7024147CF
:101FD0000546130810F82395E7002396E700239998
:101FE000E700239AE700239BE700239CE700239464
:101FF000E7022393B7002394B7002397D7002398D1
:10200000D700239DA700239E0700239F070023904E
:1020100007022395C7022396070323970702930815
:10202000F007239807022392E7042393E704239FF2
:10203000E7042390E7062391E7062392E706239916
:1020400017031307C01C239AC702239BC702239CB4
:102050000702239D0702239E0702239F0702239066
:1020600007042391C70423940704239507042396A8
:10207000C7042397D7042398D7042399A704239A46
:102080000704239B0704239C0704239DD704239E56
:10209000D7042393A70623940706239507062396C0
:1020A00007062397B7062398B70623990706239AAE
:1020B000E7067D57239B0706239007092391E7082E
:1020C0008280011126CAAA84214522CC06CE2E8404
:1020D00032C636C43AC2EFD0FF9E1DC9A24612478F
:1020E0003246930700FD2300F5009947A3009500B1
:1020F0002301F5002303D500A303E5002312C50047
:10210000AA8522856244F240D24405616FD09FAA1D
:10211000F2406244D24405618280B727002023A4A4
:10212000A7828280B727002023A6A7828280011180
:1021300022CC4AC806CE26CA2A890144B3048900A3
:102140006368B400F2406244D2444249056182802F
:102150002EC6EFD05FC093170501C183A183B2459E
:102160002380F4009307140093F7F70F850463F9B5
:10217000B700CA9709042380A7001374F40F7DBF2A
:102180003E847DBF411122C4372400201304449FA4
:1021900003556400C16706C6FD17630FF500B72736
:1021A000002003C687B3B725002093850583EF8001
:1021B000E05AFD572313F400B240224441018280CB
:1021C00009C925151375F50F1335850E134515002F
:1021D00082800145828023900500C9C6797122D48E
:1021E00026D24ECE52CC5AC806D64AD056CA5EC661
:1021F0003684328AAE892A8B814463F34407B3075D
:10220000940083C70700138914004209939A0701B9
:1022100093DA0A011359090163840A04CA976341D6
:10222000FA04B307240183CB07005E85513F0DC933
:102230009387FAFF2390F90063906B03130519004D
:102240002295B250225492540259F249624AD24A1B
:10225000424BB24B45618280D694C204C18071BFAB
:102260000145C5B701458280011122CC37240020E9
:1022700026CA4AC84EC69307449F06CE2E89D0CBA5
:102280008CCBC8C7AA8441469305F00F4A8597E0D6
:10229000FA1FE780800E85491304449F63193503B4
:1022A0000848C145693541469305F00F268597E0FA
:1022B000FA1FE780800C05496315250348446244F2
:1022C000F240D2444249B249C14505618DB541460B
:1022D00081454A8597E0FA1FE780200AE31535FD1E
:1022E000C1B741468145268597E0FA1FE780E0089F
:1022F000E30625FDF2406244D2444249B2490561F9
:102300008280411122C43724002026C24AC0AE84F4
:102310002A891306000281451305449F06C697E0EB
:10232000FA1FE78000F79307449FA3812701B7278F
:102330000020238E97B2EFC02071854719C18147D5
:102340004945230AF49EB240224492440249410185
:102350008280814781CD19C98547631BF50083C7FA
:10236000550093E707FCA382F50085473E858280F0
:1023700089476317F50083C7550093F7F703E5B75F
:102380000D478547E314E5FE03C755001377F703B0
:1023900013670704A382E500D1BF81478DC105C142
:1023A00003C755009306000C85471377070C630895
:1023B000D700930600048D476303D70089473E8505
:1023C0008280411122C4005D06C626C21DC8AA84AF
:1023D000085009C597E0FA1FE78000D5485009C5A5
:1023E00097E0FA1FE78040D4085409C597E0FA1F28
:1023F000E78080D3228597E0FA1FE780E0D223AC04
:102400000402B240224492444101828019E9B72774
:10241000002083C7679F91C73725002013050581DA
:102420008280372500201305C5A08280B7270020B1
:1024300003C5679F8280B727002003A507A082807D
:10244000B727002003A547A08280B727002083A7D5
:1024500087A088438280B72700209387479FD44B6B
:102460009842050798C203C537009307F00F63052C
:10247000F50091656FD0BFAE8280011122CC06CEEF
:102480002E8432C6EF80605F9147B2456310F5023B
:10249000B727002083A7C78295C303A30700630F54
:1024A000030022856244F24005610283B7270020C1
:1024B00083A7478281C703A34700D5B7F240624490
:1024C000054505618280011122CC2A84035545000F
:1024D00006CE26CA4AC84EC6EF8040383DC92A8972
:1024E000834405008349C500E93D4A85EF80101803
:1024F00003554400EF80A053372900201309898336
:1025000083470900B9CB639A9704B727002083C596
:1025100097832685293C19E12300090003554400CF
:10252000EF80A0559147631FF500B72700209387E0
:10253000479F8356440003D767006395E6007D57A5
:102540002393E700F2406244D2444249B249056114
:10255000828081499304F00F45B79307F00FE38F12
:10256000F4FA8346640003564400034524004E8772
:10257000A685813E65B779715EC6AA8B2E8552CC41
:1025800056CA5AC806D622D426D24AD04ECEAE8AD1
:10259000328B368AEF80802C7DC1045D2A89E5C0AC
:1025A0009C50614599C3130540039C5481C7510554
:1025B0004205418163050A00710542054181DC50F5
:1025C00081C75D0542054181EFD0CFCF2A8445C93F
:1025D0006146814597E0FA1FE780A0CBB72700202E
:1025E00083C947A46394090083490900930700FD48
:1025F0002300F400A947A30074012301F40023037E
:1026000064018C50231254011305840191C908C43C
:102610007146930A440397E0FA1FE78060C056852D
:102620008C5491C948C45146930A450197E0FA1F5A
:10263000E78000BF5685630C0A0008C87146D28542
:10264000930AC50197E0FA1FE78080BD5685CC50FC
:1026500099C548C85D4697E0FA1FE78060BCA2852F
:102660004E85EFD02FD52254B2509254F249624A8F
:10267000D24A424BB24B4A850259456199B3B25096
:10268000225492540259F249624AD24A424BB24B06
:102690004561828001114EC6AA892E854AC806CEA0
:1026A00022CC26CA2E89EF80601B21C9B7270020C3
:1026B00083C447A499E0834405001945EFD08FC037
:1026C0002A8405CD8145194697E0FA1FE78060BC52
:1026D000930700FD2300F400B947A3003401230150
:1026E000F40023122401A2856244F2404249B24917
:1026F0002685D24405616FD0EFCBF2406244D244CC
:102700004249B2490561828039715ECEAA8B2E851D
:1027100026DA4ED652D456D25AD006DE22DC4AD819
:10272000AE84328BB68A3A8ABE8942C6EF800013E5
:1027300021CD2A894145EFD0EFB82A8431C54146E1
:10274000814597E0FA1FE780C0B4B727002003C592
:1027500047A419E103450900930700FD2300F40095
:10276000BD472301F400B247A30074012312940073
:1027700023046401A304540123054401A305340187
:102780005CC4A285EFD00FC3F2506254D2544259B8
:10279000B259225A925A025BF24B216182807971BE
:1027A00026D2AA8439454AD04ECE06D622D42EC689
:1027B000B2893689EFD00FB121C1B2459307000D20
:1027C0002310F500B1472A842312B5002301F50038
:1027D000CE851905194697E0FA1FE78060A4230605
:1027E0002401A2852254B2500259F24913F5F40F84
:1027F000925445616FD00FBCB2502254925402598A
:10280000F24945618280411126C2B7240020938499
:10281000449F03C7340006C622C44AC09307F00F82
:10282000630CF7042A893945EFD0CFA92A8429C53A
:10283000930700FDB72500202300F500A300250124
:10284000230105009385C5A00D05194697E0FA1FE1
:10285000E780009D83D78400A28503C5340023153B
:10286000F40083C714002306F4002244B2409244CB
:10287000024941016FD00FB4B24022449244024950
:102880004101828001115AC02A8B314526CA4EC6A9
:1028900052C456C206CE22CC4AC8AE84B28A368A08
:1028A000BA89EFD02FA23DCD2A842685EF70107B08
:1028B00011C50347C500A1476314F704B7270020DB
:1028C00003C9779F930700FD2300F4009D47A300F1
:1028D00064012301F40023129400231354012314F0
:1028E000440123153401A2856244F240D244B24926
:1028F000224A924A024B4A85424905616FD08FAB0A
:10290000B727002003C9D7B3E31E0BFAB72700206F
:1029100083A7878D9C47DDD7CE865286D6852685B0
:1029200082974DB7F2406244D2444249B249224AAA
:10293000924A024B05618280011122CC2A842145F2
:1029400006CE2EC6EFD00F9821C1B245930700FDE9
:102950002300F500C5472301F50083C73500A30117
:10296000F50083D745002312F50083C765002303D4
:10297000F50083C77500AA85A303F500228562448C
:10298000F24005616FD00FA3F2406244056182807E
:10299000397162CC2A8C594526DA4AD84ED652D49F
:1029A00056D25AD05ECE06DE22DCAE8432C636C4A3
:1029B000BA8B3E8BC28A468A83590104034941047B
:1029C000EFD04F9025C93246930700FDA246230061
:1029D000F5009547A301C500A30085012301F5007B
:1029E0002A8419461105A9C2B68597E0FA1FE78027
:1029F000208323066401230A24012315740123176D
:102A000054012318440123193401A2856254F25061
:102A10004259B259225A925A025BF24B624C2685B5
:102A2000D25421616FD00F99814597E0FA1FE7805A
:102A30004086C1B7F2506254D2544259B259225A18
:102A4000925A025BF24B624C21618280411122C496
:102A5000372400201304449F8347240006C626C25F
:102A60008DCBB7240020AA8519461385048197D001
:102A7000FA1FE780E07A0345240093850481EFF094
:102A80005F8D2244B24013850481924441016FB0AE
:102A9000707CB24022449244014541018280411140
:102AA00026C2B72400209387449F06C622C44AC08A
:102AB00003C737009307F00F9384449F6304F70420
:102AC0002A892945EFD00F802A840DCD930700FD78
:102AD0002300F500A147A30025012301F50083C7CA
:102AE0002400B725002093850581A301F500194630
:102AF000110597D0FA1FE780A07203C53400A285A4
:102B0000EFD04F8B03C724008D476311F702B7271F
:102B1000002083A7878299CB03A387006308030063
:102B20002244B2409244024941010283B24022440D
:102B30009244024941018280797122D406D626D27C
:102B40004AD04ECE52CC56CA09445DCD2A8903558F
:102B50000500AE895144EF707050AA8455C53727DF
:102B60000020930787B383C747008546BA8AFD17BD
:102B700093F7F70F494463F9F6080347C500A147E7
:102B80006314F700639209089C5C4544B5EF9165B6
:102B9000938545711305C00297D0FA1FE780804ADC
:102BA00088DC2A8A4D442DC11306C002814597D086
:102BB000FA1FE780006E8357090093064A003685A6
:102BC0002311FA0071469305490036C697D0FA1FC3
:102BD000E780006589472300FA0003C5C400B246B8
:102BE0000356090083C58AB3611513351500EF80BC
:102BF000506D2A8463860900CE852685EF80A05615
:102C000001C42685EFF0EFFB2285B2502254925486
:102C10000259F249624AD24A45618280B7270020B0
:102C200083C7C7B30547FD1793F7F70F6378F70816
:102C3000894751C6011122CC26CA4AC84EC652C481
:102C400006CEAA89368AB2842E89EF7030412A8452
:102C5000D14729C9485509C597D0FA1FE780C04C0C
:102C6000F1452685EFD00F9648D4CD4705CD834654
:102C7000C40021478147639FE600630D0A000347B4
:102C8000A5010356050193062501AA854E85EF800F
:102C90002055AA8703474400630F090013676700A4
:102CA0002302E400F2406244D2444249B249224A3B
:102CB0003E850561828013674700DDB7C9473E85C1
:102CC00082809307000463EBA700B7270020938757
:102CD00047A106053E9503550500828041657D1597
:102CE0008280011122CC2A842E8526CA06CEAE848B
:102CF000EF70D0361DCDB7470F009387F7230945F6
:102D000063E4870281450A85414697D0FA1FE78030
:102D10004058A685231081000A8541802301810047
:102D2000A3010100EF809045F2406244D244056166
:102D300082804945D5BFB7270020238DA7B2828066
:102D40006F805052797152CC2A8A328522D426D291
:102D50004AD04ECE56CA5AC85EC606D662C4AE8B9C
:102D6000B28A368BBA843E89C2894684EF70102FAE
:102D700015C92A8C63140A0213774B008347450058
:102D800015CF93E727012302FC008DEC631C090299
:102D9000639A090205E8ED9B2302FC00832B8C0358
:102DA000639F0B06B250225492540259F249624A70
:102DB000D24A424BB24B224C45618280F59B93E74D
:102DC0000701D1B793E747002302FC0001CC1C4860
:102DD0004146A2852324FC0213058C0197D0FA1FDB
:102DE000E780004463910B02D5D80325CC0209C5C6
:102DF00097D0FA1FE7804033F1452685EFC09FFC4E
:102E00002326AC0261BFE30B09F80325CC0209C5F8
:102E100097D0FA1FE7804031F1454A85C5B79DC478
:102E200083A70B0299EB916593853571714597D016
:102E3000FA1FE780202123A0AB0203A50B0219C5CE
:102E40007146A68597D0FA1FE780803D6388090206
:102E500083A74B0299EB9165938525715D4597D0CA
:102E6000FA1FE780201E23A2AB0203A54B0219C55F
:102E70005D46CE8597D0FA1FE780803A1DC483A7B0
:102E80008B0299EB916593851571514597D0FA1F87
:102E9000E780401B23A4AB0203A58B0219C5514652
:102EA000A28597D0FA1FE780A0372254B2509254DF
:102EB000F249B24B224CCA865A860259424BD685F9
:102EC0005285D24A624A45616FF0EFEA011126CA83
:102ED00052C406CE22CC4AC84EC62A8AAE84EF70AF
:102EE000F01725C5AA893945EFC0DFBD2A8431CD49
:102EF000B727002003C947A46314090003C90900C8
:102F00009307000D2310F400AD472301F4009385CF
:102F1000690013053400194697D0FA1FE780403046
:102F200093F71400858085882306F400A306940097
:102F300023154401A2856244F240D244B249224A98
:102F40004A85424905616FC0FFC6F2406244D244DF
:102F50004249B249224A0561828001114EC652C4DB
:102F600056C206CE22CC26CA4AC8AA8A2E8AB2895E
:102F7000EF70D00E2DCD2A891305C002EFC09FB48B
:102F80002A8435C5B727002083C447A499E0834429
:102F900009009307000D2310F400E9472301F40012
:102FA0009305690013053400194697D0FA1FE7808E
:102FB0002027D285231554011305C400414697D01C
:102FC000FA1FE780E025CE851305C401414697D05E
:102FD000FA1FE780E024A2856244F2404249B249E8
:102FE000224A924A2685D24405616FC0BFBCF24096
:102FF0006244D2444249B249224A924A05618280DF
:10300000411122C43724002013048481084006C6DD
:1030100019C597D0FA1FE780201123200400B24081
:10302000224441018280011106CE22CC26CA4AC820
:103030002EC6EF70B00239CDB245B727002003C9C4
:1030400047A40CD5AA84631409000349050041452F
:10305000EFC05FA72A841DCD9307000D2310F50054
:10306000A5472301F50083C754009385640011052B
:10307000A30FF5FE194697D0FA1FE780601A9C54FB
:10308000A285F2405CC46244D2444A85424905614B
:103090006FC05FB2F2406244D2444249056182800F
:1030A0001D71A2CC86CE2A842EC6EF70207B05CD62
:1030B0008346C5001147AA8749456392E6029C5F93
:1030C000B24599C383C56701B7D605002308B1008F
:1030D0009386A6A7100889452285EF70907FF64059
:1030E0006644256182805145DDBFB727002083C734
:1030F000C7B30547FD1793F7F70F637AF7048947BE
:1031000021CA411122C426C24AC006C6B2842E89F1
:10311000EF70C0742A84D14705C56308090083474E
:10312000450093E727002302F5004146A6851305D5
:10313000840197D0FA1FE780A00E9C481CD48147D9
:10314000B2402244924402493E8541018280C947EF
:103150003E858280797122D406D62A842EC6EF70ED
:10316000E06F01CDB2452285230EB1006C08EF70EF
:10317000107CB2502254456182805145DDBF6F7092
:103180009004C1671387E7FF6395E502B727002026
:1031900083A7478291EB494582804945B24022444A
:1031A000924402494101828003A30700E30503FE24
:1031B0000283411122C426C24AC006C6FD172A89CD
:1031C0002E84B284639AF502B727002083A7478232
:1031D00091CF9C4381CF829711E9B7270020238CA0
:1031E0002783B7270020A38C97824DBFA6854A85E9
:1031F000EFE0FFD345F5D5B72E85EF70206651DDA2
:10320000834705000D45E39B27F922852244B24000
:103210000249A685924441016FB0D0009307000493
:1032200063E2A7064111C16722C406C626C2FD1784
:103230002A8409456382F502C547AE846313F4020C
:103240002E85EFB0B00537250020130545A10604F3
:103250002A94231094000145B24022449244410133
:1032600082809307A0036316F4002E85EFB0407CA4
:10327000D9BF9307B003E318F4FC13F5F50FEFB0D3
:10328000607BD1B709458280011106CE2AC6EFE0E6
:103290003FCCEF10C01CEFA0910EB7270020938702
:1032A000479F130700F02391E70023820700B72709
:1032B00000203245138787B3FD562301D700F24023
:1032C000238CA7B2954505616F50F06659719397AD
:1032D0000501A6D286D6A2D4CAD0CECED2CCD6CA2A
:1032E000DAC8DEC6E2C4E6C2EAC06EDEC187AE84DA
:1032F00063D3075237240020034584B337290020C5
:10330000372A0020EFC01F83AA8C22CCB72A0020C6
:10331000B72B00201304499F372C002063930C0225
:103320002165258DB650265496540659F649664AAD
:10333000D64A464BB64B264C964C064DF25D65611F
:10334000828083C70C001307200A639CE70083492F
:10335000340003D52C00C1656686FD15EFF0EF91B2
:103360009DA26247130787B38349270013071009FB
:103370006398E71683C71C001547639FE7006685BF
:10338000EFF06F946685EFC0CFEEE24703C587B3D9
:10339000EFC04FFAAA8C59B73947639BE71603D59C
:1033A0004C008567A5076316F50483A58C0003CB45
:1033B0000500631D0B00850591C9372500201946BE
:1033C0001305C5A097D0FA1FE78080E50347499F02
:1033D00085476317F71063080B00230A099E5A8577
:1033E000EFF06FC245B78947230AF99EEFB04066F8
:1033F00051BF896713872700631CE50403AB8C006A
:1034000063000B0E83470B0089EF83472B000347B4
:103410001B00A207D98F2314F40083473B00A300AD
:10342000F4000347499F8947631CF70A83470B0051
:1034300091C7230A099E03450B005DB7834514001D
:10344000035584008D47230AF99EEF50D051E5B70C
:1034500095076319F50083A78C0003C50700EFF0FB
:103460000FE40DB7F9771387A7FF2A974207418327
:10347000914663F1E6049387A7FCAA97C207C1832C
:1034800071476371F70289671387B7006310E5041A
:1034900083A70A82E38807EE9C43E685E38407EE70
:1034A000829715A0370700181307F770B357F70076
:1034B000858BA9CB83278A82E38607EC9C43E38331
:1034C00007EC66858297E31F05EA19A81387C700F2
:1034D0006311E50283A78C0083C70700E38407EA32
:1034E0009307F00FE380F9EAE6854E85EFC08FEC95
:1034F00069BDB9076318F50083274C82E38407E8A8
:10350000DC4361BF896793871704E303F5F8C9BFFC
:103510003D476399E70403D54C0089671387D700BB
:10352000E30CE5FC13879701E308E5FCCD07E319FD
:10353000F5FA03576400C167FD17631DF700832781
:103540004C82E38107E4DC43E38E07E20965E6850C
:103550004D05B9B7B727002083A7C782E38407E2E8
:103560009C43DDB71307E003E39CE7F683C72C0019
:1035700005476398E70E83C76C0037270020930D3B
:103580008781E1E783A70D00D5CF03CB0700A149D1
:1035900003C57C00138D8C00EA85EFE01FE083C734
:1035A0004C01A383AC0083D80C0103D8EC0003D7F3
:1035B0004C002A8603C53C003EC283D72C01EA8614
:1035C000DA853EC0CE87EFF0AFBC83C73C0095E7FD
:1035D000DD4783D80C0103D8EC0083C67C0083D57B
:1035E0004C003EC283D72C016A873EC0CE87054679
:1035F0005A85EF70805FA381AC0083A70D0081C75F
:103600001145EFF0FF9F138B8B8303450B00E30BFA
:1036100005D6B727002083C59783EFE05F91E303CA
:1036200005D683C63C0093071003638AF60003D6D1
:103630004C0083450B004E873685EFE09FA8238C16
:103640000B8289B3034B340099B783278A82034BDB
:103650003400914995DFDC4385DF81450145829740
:1036600005BF29476398E70A83C76C003727002006
:10367000930D8781A5EF83A70D00B5C703CB070086
:10368000A14903C57C0093868C0093772500BDCBB0
:1036900013761500138E4C0183C70C0283D8CC011E
:1036A00003D8AC0103D74C0003C53C003EC283D70E
:1036B000EC01DA8572CE3EC0CE87EFF06FAD83C7E6
:1036C0003C00724E9DFBDD4783D8CC0103D8AC0192
:1036D00083C67C0083D54C003EC283D7EC01728741
:1036E0003EC0CE8729B7034B340059BF83278A8257
:1036F000034B34009149D1D7DC43C1D78145014503
:10370000829741B7B68536CEEFE03FC9F2462A86AA
:10371000368E59B70947639CE70083A70A82E38383
:1037200007C6DC43E38007C666858297A1B92D47AB
:103730006398E70083A70A82E38607C49C47DDB746
:103740000D476397E70066868D4503D54C0039B178
:1037500019476395E7069305610213051031EFA041
:10376000A14A2C1013052031EFA0014A03D66C00AA
:103770008357810203D54C0063E8C70083D68C00D1
:103780000357610263F7E60093050002EFB00030D3
:10379000D5BE6374E6002393EC0063F4D700239452
:1037A000FC0003D7CC0083D6AC0003D68C0083D5B5
:1037B0006C0001488147EFB0202DE9B61D47E38139
:1037C000E7D231476395E7006686B145BDBF35470F
:1037D0006398E70083A70A82E38607BADC4799B7B4
:1037E0004947639DE70083278A82E38B07CEDC434A
:1037F000E38807CE814505458297DDB14D47E391CA
:10380000E7CE83278A82E38D07CCDC43E38A07CCAB
:10381000E6850945D5B793F7150089CFB72700206E
:1038200083A7078289C7DC4399C30145829713C5E3
:103830001400CDBC93F7250091CFB727002083A7B4
:10384000878291C7DC4381C781450545829713C5AF
:103850002400C9BC93F745000145E38507ACB727B1
:10386000002083A7C781372400201304449F91CFF1
:1038700085472302F400B727002083A7878291C7DA
:10388000DC4381C781450545829748442C10EF7081
:10389000507B2810EFF08F9BB727002083D767A3BA
:1038A00081CF130600643386C702B727002003C503
:1038B00087B39145EFC09F8913C54400A5B441115A
:1038C00022C4372400200325C48106C619C597D019
:1038D000FA1FE7806085232E0480B2402244410114
:1038E00082805971A2D4372400208327C48186D6D0
:1038F000A6D2CAD0CECED2CCD6CADAC80545638D00
:10390000070C9305F1041305F041EF807113930543
:10391000F1041305F041EF80B112B727002093871F
:10392000479F83C727000347F104B337F00011C353
:1039300089070327C4813EDE03453700930547000E
:10394000EFE03FA10327C4812ADC0D458345270012
:103950002EDAEFF00FB72AD81145EFF08FB6032417
:10396000C4812AD665450347A400034BB4003AD46A
:10397000EFF02FB5AA846945EFF0AFB42A897145FD
:10398000EFF02FB4AA896D45EFF0AFB32A8A7545E1
:10399000EFF02FB3AA8A7945EFF0AFB2E204625894
:1039A000F2572257B2564256D2551375F50F93FA75
:1039B000FA0F137AFA0F93F9F90F1379F90FE184DB
:1039C0002ACC56CA52C84EC64AC426C25AC0930808
:1039D00044000545EFB0400DB650265496540659A4
:1039E000F649664AD64A464B65618280011122CC6F
:1039F00006CE26CA8D472E846315F50603C735000B
:103A0000B7240020E94703D545009384449F6316FB
:103A1000F70083D764006382A706EF60306409C5AE
:103A2000835764002317F5000357A40083568400CE
:103A3000035664008355440003453400EFE09FE4DF
:103A40000357440083D764006309F7008547F240B9
:103A50006244D2443E8505618280FD572393F40081
:103A6000F5B78967CD07631DF50083C7250031478A
:103A70006385E7004547E39BE7FCEFE0AFF0F9B76C
:103A8000B1476319F500B727002003C5D7B3EFE0AE
:103A9000BFEA6DBF41677D178147E31AE5FA83C628
:103AA00055004947E395E6FA83C5450003552400D0
:103AB000300023140100EF60B04649BF411122C419
:103AC000372400208347A48326C206C64AC01307B2
:103AD000E00FAE846386E7041307F00F1304A4839A
:103AE0006387E7021145EFB0FFFD15C1930700FDA5
:103AF0002300F50089472301F5008547A3009500C1
:103B0000A301F500AA8503450400EFC0AF8AF95769
:103B10002300F400B24022449244024941018280D1
:103B20002A891145EFB01FFA75D5930700FD2300D0
:103B3000F50089472301F500A3009500A3012501A5
:103B40002244B7270020B24092440249AA8503C507
:103B5000B78341016FC00F8679714AD037290020A1
:103B60008327C98122D406D626D24ECE52CC56CA3D
:103B70004544D5EFB7240020938784B383C747001B
:103B80004944958BCDC7B72700202E8A9165A38D18
:103B9000A782AA8993857571314597C0FA1FE7807E
:103BA000604A232EA9804D4459C123003501A3004A
:103BB00005002946D285090597C0FA1FE7804066AF
:103BC0008327C981914603C7270063EDE60835EBDB
:103BD0004D472381E70003C72700136707012381AF
:103BE000E700930571001305F041EF80616583479D
:103BF0007100F1EBB727002003C7679F8D4763145F
:103C0000F70CEFE05F832C00EF70B0432800EFE08B
:103C1000FFE34545EFF0EF8A014411C91306006444
:103C20003306C50203C584B39145EFC02FD2228568
:103C3000B250225492540259F249624AD24A456122
:103C4000828085466314D700754761B7894663143F
:103C5000D7004947BDBF8D466314D700414795BF84
:103C6000554785BF9546CA8A630ED70099466316A5
:103C7000D70009472381E70031A01D466314C7021E
:103C8000238107006545EFF0CF839307F007E30A30
:103C9000F5F403A7CA818347270093E707042301AC
:103CA000F70081B721466314C7000547E1B72546F1
:103CB0006315C7002381D700F1B7A9460544E3186F
:103CC000D7F6114745BF31392A8435D1CD3E85B766
:103CD000011126CAB724002083A7C48122CC06CEB6
:103CE0004AC84944B1C783C707000D446392A7047B
:103CF00037290020034589B38945EFC0EFED03451F
:103D000089B3B72700209145239E0782EFC0CFECEF
:103D100083A7C48101478146A38087001306F10071
:103D2000854785450145A307F100EFA0505B2A8434
:103D30002285F2406244D2444249056182800111E9
:103D400006CE22CC26CA4AC88547631EF50637240C
:103D500000201304C48383570400A9CB3727002015
:103D60000347879F21E71307B003636CF702B7246B
:103D7000002003C584B38945EFC00FE60356040055
:103D80009307006403C584B33306F6028945EFC088
:103D9000EFBB23100400F2406244D2444249056163
:103DA0008280938747FC2310F400F5B7B7270020E3
:103DB00083A7C781EDD36244F240D244424903C590
:103DC0000700056131B7B724002083A7C481E1D77C
:103DD00037270020130987B383474900918BC5DF3C
:103DE00089476313F5062D452EC6EFB0BFCD2A8453
:103DF0005DD1B245930700FD2300F500E547A30020
:103E000005002301F50083C7350015051946230F6A
:103E1000F5FE83C745009505A30FF5FE97C0FA1F71
:103E2000E7800040034559009307F00F6316F50043
:103E300083A7C48103C50700A2856244F240D2442F
:103E4000424905616FB01FD7034587B38945EFC06D
:103E5000AFD86244F240D2444249B7270020239EA3
:103E6000078205616FF0BFA549458280B727002012
:103E700083C7C7B3958B638F07129307C01C63FC7E
:103E8000C70009458280F2406244D2444249B249A7
:103E9000094505618280B727002083A7C781638B0E
:103EA0000710B72700209387A78303C807001307CD
:103EB000E00F6311E810011122CC4AC806CE26CAD1
:103EC0004EC62380A700130586004205368932843A
:103ED0004181ADC991659385657197C0FA1FE780EF
:103EE0006016AA894DD1B724002003A54484938489
:103EF000448409C597C0FA1FE78000231385890011
:103F000023A0A9002286814523A0340197C0FA1F6F
:103F1000E78020389C402286CA85884397C0FA1FD4
:103F2000E78000309C40A286F240239287006244E2
:103F3000D2444249B249984305468D45054505613D
:103F40006FA0703991659385557197C0FA1FE7800E
:103F5000600FAA890DD9B724002003A5C4849384D7
:103F6000C48409C597C0FA1FE780001C1385890027
:103F700023A0A9002286814523A0340197C0FA1FFF
:103F8000E78020319C402286CA85884397C0FA1F6B
:103F9000E78000299C40A286F24023928700624479
:103FA000D2444249B249984305468D4505450561CD
:103FB0006FA0B032494582809307C01C63FCA70004
:103FC000094582800945F2406244D2444249B249DF
:103FD0000561828045CD011122CC2A8421054EC67F
:103FE0004205AE8991659385657141814AC806CEC7
:103FF00026CA97C0FA1FE780E0042A8961D5B72452
:10400000002003A544849384448409C597C0FA1F03
:10401000E7808011130589002320A90022868145AD
:1040200023A0240197C0FA1FE780A0269C40228687
:10403000CE85884397C0FA1FE780801E9C4023925C
:104040008700B727002083A7C7818DCFB72700201F
:1040500083C7C7B3958B8DCBB727002083A7478431
:1040600099CF984383D647006244F240D2444249F4
:10407000B24905468D45054505616FA0D02501472C
:104080008146DDB7014581B7494535BFB7270020D7
:1040900083A7C78195C7B727002083C7C7B3958B70
:1040A00095C3B727002083A7478481CB984383D645
:1040B000470005468D450545C9B701478146D5BF2F
:1040C00001458280494582809307C01C63FCA7009C
:1040D000094582800945F2406244D2444249B249CE
:1040E0000561828045CD011122CC2A8421054EC66E
:1040F0004205AE8991659385557141814AC806CEC6
:1041000026CA97C0FA1FE780E0F32A8961D5B72451
:10411000002003A5C4849384C48409C597C0FA1FF2
:10412000E7808000130589002320A90022868145AD
:1041300023A0240197C0FA1FE780A0159C40228687
:10414000CE85884397C0FA1FE780800D9C4023925C
:104150008700B727002083A7C7818DCFB72700200E
:1041600083C7C7B3958B8DCBB727002083A7C784A0
:1041700099CF984383D647006244F240D2444249E3
:10418000B24905468D45054505616FA010150147EB
:104190008146DDB7014581B7494535BFB7270020C6
:1041A00083A7C78195C7B727002083C7C7B3958B5F
:1041B00095C3B727002083A7C78481CB984383D6B4
:1041C000470005468D450545C9B701478146D5BF1E
:1041D00001458280494582809307C01C63F4A70093
:1041E00009458280797122D44ECE06D626D24AD095
:1041F000AE892A842DC1210591654205938575718B
:10420000418197C0FA1FE780E0E32A8909456306E8
:104210000908B724002003A584849384848409C5F5
:1042200097C0FA1FE78040F0130589002320A900FA
:104230002286814523A0240197C0FA1FE7806005EC
:104240009C402286CE85884397C0FA1FE78040FDB8
:104250009C4023928700B727002083A7C781014590
:104260008DCFB727002083C7C7B34945958B95C726
:104270006C001305D030EF903119B247014593F728
:10428000070F81CFB727002083A787848D45054579
:10429000944303D64700EFA0D004B2502254925466
:1042A0000259F24945618280B727002083A74784DD
:1042B00091CF03D647008C43411106C697C0FA1F21
:1042C000E78000F6B24001454101828009458280C5
:1042D000B727002083A747848DC7B727002003A7EF
:1042E000C784894705C3035647000C43411106C6DE
:1042F00097C0FA1FE780C0F2B24081473E85410176
:10430000828089473E858280797106D622D426D262
:104310004AD04ECE52CC8D4763FCA7008944B250A0
:104320002254268502599254F249624A456182809C
:10433000372900200347499FC144E312F7FE930742
:10434000F5FF9309499F93F7F70F8546AE842A84BA
:1043500003CA29001309499F63EAF6068DE19945CE
:104360002800EFD0DFDCB729002003C589B39145D1
:1043700023018900EFC04F8635E481444DB71946CB
:104380008145280097C0FA1FE780A0F019462C004D
:10439000268597C0FA1FE780E0F549F11946930595
:1043A000F00F280097C0FA1FE780A0EE19462C00F6
:1043B000268597C0FA1FE780E0F32DF11946A68500
:1043C000280097C0FA1FE780A0E571BFE31DE5F85C
:1043D00003A5C9002C00EF70C046AA8449D52381EB
:1043E000490135BF2800EFE06FE6AA840DED930583
:1043F00071001305F041EF70B16483447100B5FCA6
:104400008D47E31CF4F64545EFE0BF8B3DD5B7770C
:104410001800938707A03306F50203C589B39145B9
:10442000EFB05FF4EDBD23014901D5BDB7270020F2
:1044300083C7C7B3918B8DC3372500204111130566
:10444000058406C6EFD01FCEB240B72700207D57A7
:10445000239DE79E4101828001456FD0BFCCB727E5
:1044600000207D57A38DE782B72700207957238D41
:10447000E782B7270020238C07A8B7270020239EB8
:104480000782B727002023A20784B727002023A68E
:104490000784B727002023A4078437470500B727E0
:1044A00000209387078E1307876798C33747050057
:1044B0001307E7D3D8C3374705001307278E98C7DC
:1044C000B7470500372700209387C79E2320F7842E
:1044D0008280411126C2B724002083A7C48106C66A
:1044E00022C48DCF2A840D45EFB0CFDDAA8505C14A
:1044F000930700FD2300F5008D47A30085002301ED
:10450000F50083A7C48103C50700EFB0AFEA19C463
:104510002244B240924441016FF06FBAB24022444B
:10452000924441018280797152CC372A002083273E
:10453000CA814AD006D622D426D24ECE56CA0149C6
:10454000B1C703C91700B72400208547AA899384FF
:10455000449F6307F90483C74400054985EB0D4573
:10456000EFB04FD6AA8505C1930700FD2300F500E3
:104570009147A30035012301F5008327CA8103C5B4
:104580000700EFB02FE3EFF08FB30549B25022548C
:104590004A8592540259F249624AD24A4561828060
:1045A000B727002083A74784D28A85E30145EFE03F
:1045B0004FF12A8601CAB727002003C587B3894572
:1045C000EFB0DFB883A7CA8181A8944303D6470020
:1045D0009305E1000545EFD01FC069D98347050069
:1045E000858BE9D70545EFE0CFED9307B0032A842B
:1045F00063F0A704B727002003C587B35D661306E1
:1046000006708945EFB01FD6B7270020130444FC7D
:10461000239E87828327CA810947A380E70083C737
:10462000440081C72382040095B74E855D35B9BF2C
:10463000130600643306C502B5BF411122C42A84A3
:104640000D4506C6EFB00FC805C5930700FD230052
:10465000F500CD472301F500A30085002244B727CC
:104660000020B240AA8503C5B78341016FB08FD443
:10467000B24022444101828083564500011189677E
:1046800006CE22CC26CA138667002A876399C60005
:104690001C47014583C50700EFF04FC23DA81386B4
:1046A00087006397C6001C47054583C50700EDB723
:1046B000138697006395C602B727002083A7C7819A
:1046C000014595C71847034507006311050E0547C7
:1046D000A380E7000545EFA02038054509A813860B
:1046E000A700639BC6001C4703C507002D3DF24091
:1046F0006244D2440561828013866703E38AC6F868
:1047000013867703E381C6FA138687036392C60A8A
:104710001C45372400201307E00F83C4070083479C
:10472000A4831304A483638EE7021307F00F638648
:10473000E7021145EFB00FB9AA8505C1930700FD47
:104740002300F5008947A30095002301F500A3018C
:10475000050003450400EFB0EFC5F9572300F4004E
:10476000ADBFB727002003A7C7813E84014541D3D1
:104770008DEC85447D4523059100EFE08FD4231611
:10478000A10013050002EFE0CFD38327C481A30566
:10479000A1001307B100A380970074001306A100C5
:1047A00085450545EFA0A0330DBF26851D3335B7E0
:1047B00013869703E389C6F21386E7036397C6005F
:1047C0001C45094583C50700C1BD9387F703014513
:1047D000E39FF6F01C4703C5070005E96C001305CD
:1047E000D030EF906142B247414793F7070FE3861D
:1047F000E7EE9305B10013056031EF90E14003450A
:10480000B1008545EFA0202EC9BD053DF9B5B727FC
:10481000002083C7C7B3411106C6958B99CB3725B6
:1048200000201305058EEFD05F8F4D45B24041014A
:1048300082800145EFD07F8E0145CDBF03C70500C3
:10484000937625009377D70F99C2936727001318A3
:1048500085011358884113F7F7076354080013E7DD
:104860000708937685009377770F99C2936787003F
:104870001377050293F6F70D19C393E60702238019
:10488000D500634508009377A50281CB83470600D6
:1048900093E7C7002300F60082807DFD8347060072
:1048A000CD9BCDBF2D456319071403C805000947EB
:1048B0006310E814C84103471500034505002207AB
:1048C000498F42070D654187930825A0630B170B9D
:1048D000011122CC26CA4AC84EC606CEBE89B6846D
:1048E00032842E8963CEE800930705A0630DF7029A
:1048F000130515A06300A706239004000545B5A085
:10490000930745A06309F7086348F706130565AAEE
:10491000E314A7FE85472390F600DC4583C7070014
:104920002300F60091A0C84597C0FA1FE780809940
:10493000420541814E86637335012A862390C40067
:10494000420641828325C900228597C0FA1FE7806D
:10495000208D19A8DC4583D707002390060123008A
:10496000F600A183A300F6000145F2406244D24460
:104970004249B2490561828099472390F600194661
:10498000D1B785472390F600DC45014583C7070072
:104990002300F6008280DC45A9CB21472390E60066
:1049A00003D707002300E60003D707002183A300F5
:1049B000E60003D727002301E60003D72700218361
:1049C000A301E60003D747002302E60003D7470010
:1049D0002183A302E60003D767002303E60083D701
:1049E0006700A183A303F60041B723900600ADBF83
:1049F0002390060005458280828083C80500894790
:104A00006394F816DC41797122D406D626D24AD0B6
:104A10004ECE52CC56CA03C8170083C707002E8457
:104A200022083368F80042088D6713580841138341
:104A300027A0630C68102A8A3A89B684B285634C31
:104A40000301138707A0630BE802938717A0630194
:104A5000F80A854711A8138737A06303E80C13876A
:104A600067AA8D47E317E8FEB250225492540259C8
:104A7000F249624AD24A3E8545618280484432C644
:104A800097C0FA1FE7800084420541819D47E36D8E
:104A900025FDB72A0020938A2A8583C70A00B30917
:104AA0009900B24563D43701B5477DBF4844268697
:104AB000C2094A9597B0FA1FE780807603C60A00BC
:104AC000484493D9090105063306364181454E9580
:104AD00097B0FA1FE780E07BB727002083A74785C0
:104AE00099E3814751B79C438145E5DF52853DA05D
:104AF000AD47E31B09F6E39916FB8347160083468F
:104B000006005844A207D58F2310F700B7270020CE
:104B100083A74785F9D79C438545E1D78297D1B7CD
:104B2000AD47E31309F49947E390F6F84844194672
:104B300097B0FA1FE780C06EB727002083A747858C
:104B4000CDD39C43D9DF8D4555B7AD4711FF854780
:104B5000E39CF6F40347060093070008E3E6E6F05B
:104B6000DC452380E700B5BF85473E858280B727B7
:104B7000002023AA0784B7270020A3890784B7272A
:104B8000002023890784B7150020B707A00093856C
:104B9000457E938707059CC1B707E803DCC137F65C
:104BA0000600B71700209387076F1306C6C1D0C34E
:104BB000B71E002037F606000947938EFE7D1306C8
:104BC00006BF371E00202380EE00130ECE7DD0C717
:104BD00023AED70137230020B71800203718002054
:104BE0003715002037F60600B7FE06008546130687
:104BF00006C02300EE009388087E23AEC70313038C
:104C000003851308E87D1305D57D938E8EC037FE8E
:104C100006002380E8002380E7002388E700238044
:104C2000E7022388E7022380E7042300E8002384C7
:104C3000D70023950700D0CB238CD700239D0700F6
:104C400023A2D7032384D7022395070223A60702B2
:104C5000D0DB238CD702239D0702231003002300FF
:104C6000D500130E8EBF23A2C7052388E70423AE09
:104C700017052380E7062388E7062380E708B7F8AF
:104C8000060037F706001307C7BF938888C123A221
:104C9000E7082384D7042395070423A66704F0CBF1
:104CA000238CD704239D070423A217072384D70648
:104CB00023950706ECD7F0DB238CD706239D070648
:104CC00023AE07072384D7082395070823A6A70840
:104CD00037570500B7170020938707781307478ACF
:104CE00098C3375705001307A79FD8C323A407000D
:104CF0008280A54763ECA710B7E706009387C75FDC
:104D00000A053E951C41011122CC26CA06CE4AC88E
:104D1000B2842E8482879307800F63F9B7006145C0
:104D2000F2406244D2444249056182803719002032
:104D30009307096FC8571309096F09C997B0FA1F7C
:104D4000E780803EB72700202389078413061400DC
:104D5000916593850571328532C697B0FA1FE78059
:104D6000602E2326A90245DD3246814597B0FA1F01
:104D7000E78020520325C9022286A68597B0FA1F34
:104D8000E780004AB727002023898784014549BF6F
:104D90008947E396F5F803570600B72700202398C4
:104DA000E784EDB7A147E39CF5F6371500202146CF
:104DB000A6851305457E97B0FA1FE7806046F9B7D0
:104DC0008547E39EF5F4B71500209385056FD04D18
:104DD0009385850203C50400EFF05FA645BF8547B4
:104DE000E39FF5F2B71500209385056FD05D93859D
:104DF0008504CDB78547E394F5F203470600B7175E
:104E00000020A38EE77C59B7094519BF0945828068
:104E100005476302E5044111AA8706C62E8581CFA6
:104E200011476383E70425476388E7048947B24055
:104E30003E8541018280B717002083A5C77189474D
:104E4000FDD5B727002003C6278597B0FA1FE78056
:104E5000203D8147E9BFB727002083D707852390EE
:104E6000F50081473E858280B71500202146938555
:104E7000457EEF90416BF1BFB717002083C7D77D08
:104E80002380F500F9B7B72700209387378503C73C
:104E9000070015E305472380E700058909CDB7160C
:104EA000002037150020938606784146A545130556
:104EB000056F6F30406D01458280011106CE22CC16
:104EC0000546638CC50211460944639EC5023EC671
:104ED0003AC436C2EFD0EFC22A8492462247B24784
:104EE0001DE13E86BA853685EFD00FB8EFF03F92D0
:104EF000EFF0CFD3EF60F06F39A0EFD08FC02A84EE
:104F000019E1EFF0DF902285F24062440561828072
:104F100079714ECEAE896C0022D426D24AD006D604
:104F20002A89B284EF00707A2A840DE1CE854A8501
:104F3000EFC05F882A8419E93245B7160500268735
:104F40009386667A2D468145EF10C0122285B250B5
:104F5000225492540259F2494561828079714ECEB1
:104F6000AE896C0022D426D24AD006D62A89B284D1
:104F7000EF00B0752A840DE1CE854A85EFC0BF9160
:104F80002A8419E93245B726050026879386C68804
:104F90004D468145EF10000E2285B25022549254A6
:104FA0000259F24945618280397126DAAE844C009B
:104FB00022DC4AD84ED652D406DEAA893289368AF5
:104FC000EF00B0702A8431EDA6856303090283D710
:104FD00004002C002314F10083D724002315F100D2
:104FE000930720302316F100930780022307F10076
:104FF0004E85EFC00FF92A840DE55946A6851305A5
:10500000A1002304210197B0FA1FE7806021124517
:10501000B716050052879386067525462C00EF10BB
:1050200060052285F2506254D2544259B259225A34
:1050300021618280797126D2AE846C0022D44AD05C
:105040004ECE06D6AA893289EF0030682A840DE157
:10505000A6854E85EFC0EFF72A8419E93245B716C9
:1050600005004A879386467C3546A685EF1080006A
:105070002285B250225492540259F24945618280ED
:10508000BD47638CF50663E9B702A5476387F5065C
:1050900063EDB7009947638CF5049D47638FF50472
:1050A0009547638CF50401458280B5476387F50415
:1050B00063E1B704AD47F5B7DD47638EF50263EAF8
:1050C000B700C947638BF502D9476386F502C54728
:1050D000C9BFF5476383F50263E4B700ED47D1B775
:1050E00093072005638BF5009307200D5DBF4845AE
:1050F00082800841828008458280484182809307EF
:10510000F00F630EF506011126CAAA8413050002EA
:1051100022CC4AC84EC652C456C206CE3A89B68977
:10512000B28A2E8AEFA01F9A2A844D4515C893078C
:1051300000FB2300F400A3005401231144012302C7
:10514000340113058400614663050902CA8597B0DE
:10515000FA1FE780E00CA2852685EFA0BFA50145D8
:10516000F2406244D2444249B249224A924A05611D
:105170008280814597B0FA1FE780A011E9BF0945F9
:105180008280011122CC06CE2A842306B100A30618
:10519000C100EF50A06C15C18346C500B7270020A1
:1051A0002147938787B3639EE60003C567007800B5
:1051B0009306E0070146A2859937F24062440561F3
:1051C000828078009306E0070146A28503C5570058
:1051D000E5B7930700643306F6026FB06F8C05C91C
:1051E0000347050085469307270093F7F70F63F001
:1051F000F602411122C42A843A8506C6EFB0CFA434
:10520000FD572300F400B240224441018280828095
:10521000035705009307000B6313F702834745000C
:105220004947639CE7000347150185476399E700F9
:105230000355250085456F3090646D47C5BF82805A
:1052400001112314B1006C0022CC26CA4AC806CE34
:105250002A89B6842315C100EF0030472A840DE166
:105260002C004A85EFC02FC82A8419E93245B716A9
:10527000050026879386E66915462C00EF00905FAF
:105280002285F2406244D2444249056182807971AC
:10529000930720302314B1002315C1002316F10019
:1052A0002C0093078002014606D62307F100EFF099
:1052B000BFCFB25045618280C177797185073EC406
:1052C000894726D22316F100AE84930780024C0052
:1052D00022D44AD006D62A892307F100EF00F03EF7
:1052E0002A840DE12C004A85EFC00FD82A8419E9E1
:1052F0001245B726050026879386468345462C002F
:10530000EF0050572285B250225492540259456101
:105310008280B28605466FF03FC9797126D2AE848D
:105320006C0022D44AD04ECE06D6AA893289EF002C
:10533000D0392A840DE1A6854E85EFC0EFB12A84CD
:1053400019E93245B71605004A879386A6630D46CC
:10535000A685EF0030522285B25022549254025951
:10536000F249456182807971930720202314B100AE
:105370002315C1002316F1002C009307800201467B
:1053800006D62307F100EFF03FC2B250456182809C
:10539000011122CC06CE2A842EC632C436C2EF506A
:1053A000E04B0DCD0345C500B7270020A1469387EC
:1053B00087B312472246B245631CD50003C5670078
:1053C000B2862E86A2856244F24005616FF03FD31B
:1053D000B28603C557002E86A285F5B7F240624417
:1053E0000545056182806FF0BFB26FF07FB26FF04C
:1053F0007FC46FF03FC479714ECEAE896C0022D469
:1054000026D24AD006D62A89B284EF00102C2A84EC
:105410000DE1CE854A85EFC0AFBD2A8419E932453A
:10542000B716050026879386267E3D468145EF0008
:1054300070442285B250225492540259F249456177
:105440008280B28601466FF03FB6011122CC2E84D5
:105450006C0026CA06CEAA84EF003027DD47630A17
:10546000F500930710102314F400A2852685EFC0E1
:105470008FC2F2406244D2440561828023940500C9
:1054800083D7850099E36FF07FAD09458280FDB732
:10549000B727002003C7E788854763F9E7020111B2
:1054A00022CC2E846C0026CA06CEAA84EF00F021FE
:1054B00009E9930700102314F400A2852685EFC0A4
:1054C0008FBDF2406244D24405618280594582809A
:1054D000B727002023ACA7848280B727002023AE03
:1054E000A7848280011122CC26CA06CE2A84AE84EB
:1054F000EF50C036A6852285EFB03FE10DE9228549
:1055000023169100EF5080351DC18346C500B72793
:1055100000202147938787B36390E60203C56700A5
:1055200078009306F0070146A285EFF05FBDF240D8
:105530006244D2440561828003C55700D5B701118A
:1055400026CA06CEB68422CCDD4663E2B608D9462A
:1055500063FED50AA5466381D50A63EEB604954677
:10556000638CD50899466387D50A054441687D1840
:10557000631606093AC6EFB01FDD33068540324791
:1055800042064182420441803305C4004205BA8587
:10559000418132C6EF30D03FAA8749C181C432462B
:1055A0002390C400B30580406244F240D2443E855B
:1055B00005616FA0CFC4C5466380D504C9460D44BC
:1055C000E395D5FAC167FD17E31EF6FA65B7F54610
:1055D0006380D50463E4B600ED46D5B79306200595
:1055E0006388D5029306200DE391D5F8C167FD17B6
:1055F0000D446319F600BDBF09448DBF9306200D0D
:10560000E392D5F8310642064182ADBF15445DBF35
:105610000D444DBFC167FD171D447DB7F240624484
:10562000D24405618280011122CC26CA06CE03C66F
:1056300045002E841307000281469945AA8401374C
:105640002AC629CD8357040003464400930554001D
:105650002310F100835724002311F10089472312FE
:10566000F100930780022303F10097B0FA1FE7804F
:1056700020BB834744008A8526852314F100EFC0B0
:105680004F892A8411C5324597B0FA1FE780C0A917
:105690002285F2406244D244056182804D44CDBFF0
:1056A0005D7186C6A2C4A6C2CAC04EDE8947630623
:1056B000F600C14709446319F6040144B1C52E89B7
:1056C0004C0832C6B689AA84EF0030002A843246DC
:1056D00005EDC1778507CA851305D1013ECC230EA0
:1056E000C10097B0FA1FE780A0B32C082685253F9C
:1056F0002A8419E95245B71605004E879386666FCE
:105700001D462C08EF0010172285B640264496440B
:105710000649F25961618280797122D436844AD077
:105720004ECE52CCB2892E8A3A8981461307100296
:105730002286D94526D206D6AA8411352AC629C181
:105740002286CA85231481002312410123133101CB
:1057500097B0FA1FE780C0AC4C002685EFC06F9E63
:105760002A8411C5324597B0FA1FE780E09B228555
:10577000B250225492540259F249624A45618280E1
:105780004D44F5B7011122CC26CA06CE4AC8DD47E2
:105790002A84AE84638DF5028147035504006C00B2
:1057A0002306F100EFC06F9D0545638DA4080345F6
:1057B0008400B165938505B8EFA0BF83E547230159
:1057C000F400B7270500938707975CC09DA803479F
:1057D00055013149B2863306270318499C42329756
:1057E0001043E31BF6FA83D7460003564700E31540
:1057F000F6FA8C46084797B0FA1FE780A0AF49DD5C
:105800008347540103474401850793F7F70FA30A21
:10581000F40063FFE702B387270318480355040029
:10582000BA97984783D6470003D6270083D5070049
:10583000E5353DF103458400B165938505B8EFA0DA
:105840004FFB5945F2406244D2444249056182808F
:105850008347640199B7011122CC26CA06CEDD47E1
:105860002A84AE84639BF50603550500EFB0BFADF7
:105870000356C40183562401035744016D162A962A
:1058800042064182B307D640C207231EC400C1832B
:1058900063F0E7089305C5FF3308F740635BB80280
:1058A000BA96918EC206184C835504010355040024
:1058B000C1823E97953515E103458400B165938516
:1058C00005B8EFA00FF35945F2406244D244056198
:1058D00082806D1593160501F9B7814703550400C1
:1058E0006C002306F100EFC04F890545E38EA4FC50
:1058F00003458400B165938505B8EFA08FEFE547B8
:105900002301F400B7270500938707975CC065BFA4
:105910008547E9B7397126DAAE842C0022DC4AD8F3
:105920004ED606DE2A89B2894D232A8421ED4A8586
:10593000EFB07FA183D644006D1563C5A600931612
:105940000501C182984403D6240083D504004A850A
:10595000EFF09FDC2A841DE53146A6850808230662
:10596000010097B0FA1FE780A08B83D7240022455F
:10597000B72605004E879386E68F5D466C00231E92
:10598000F100CD2D2285F2506254D2544259B259C1
:105990002161828041B7BDBF797126D206D622D45B
:1059A0004AD04ECE52CC56CA5AC88944C5C159CEE7
:1059B0002E842A89BA8A368B328AEFB0DF98930513
:1059C00044008147711503D705006352A70A850774
:1059D00093F7F70FB105E318FAFE8A854A85F5219A
:1059E000AA842DE531453305AA029165938515708A
:1059F000CD4497A0FA1FE780E064AA8921C9314607
:105A00003306CA02A28597B0FA1FE7806081184466
:105A10008356440003562400835504004A85EFF062
:105A2000BFCFAA841DED0245B726050085475687DE
:105A30009386E68F5D464C002302F1004EC4230698
:105A40004101A3060100230761012D25B250225414
:105A5000268502599254F249624AD24A424B456124
:105A600082804E8597A0FA1FE780006CC5B7ED4491
:105A7000F1BF79714ECE37F60600AE89C16526D2E8
:105A80000147AA848946130646C2FD15054522D45E
:105A900006D64AD0EF10301A054431CD2A891307B3
:105AA000300281461146F5452685EFF05FA92AC6EA
:105AB000554431C18357A900CE8601462314F10015
:105AC00091472315F10085472300F500B2472C00CC
:105AD0002685A38007003247FD572301F700324790
:105AE000A301F700EF10F00A2A8411C5324597A0F0
:105AF000FA1FE78060632285B25022549254025903
:105B0000F24945618280411106C6EFF06FD719C591
:105B1000B240410117A3FA1F67000361B24041017F
:105B20008280011106CE2AC6EFB0CFE73245B727F3
:105B3000002023AC0784B727002023AE07849145BB
:105B4000B7270020A38CA7B2EF30E05EF2400561DA
:105B50006F20F0387971939705014AD006D622D488
:105B600026D2C187014963DE070AB727002003C593
:105B700097B32E89EF901FFC2A844DC1034705007F
:105B80009307000A6319F70885474C08A305F1003D
:105B9000EFB06FEEAA840DED834761017147637921
:105BA000F708138717FE1377F70F9306000263F8C1
:105BB000E608858BD5CBB727002083A78785994436
:105BC00081CB035524001306B1004C088297AA84A8
:105BD0008347B10099C7084409C597A0FA1FE78019
:105BE000A05495E05247B7070001938707F07D8FD7
:105BF000B707120093870710630FF700034761018F
:105C0000ED47631AF700035524008545EF30204720
:105C1000CD476388F4002285EF90BFE5A167334943
:105C2000F900B25022544A8592540259456182804B
:105C30003707301405073357F700058B3DDB37274F
:105C400000200327C78549D70347510151F3230695
:105C5000F10099472308F100035524006C00231735
:105C60000100EFB0DF85ADB7B727002083A7C78558
:105C70009DC3035524001306B1004C08829729D90F
:105C8000AA8483475101A9F7834761012308910042
:105C90002306F100D1B79944EDB7397122DC26DA39
:105CA00006DE4AD84ED652D456D25AD0A5472A84B8
:105CB000B2846399F5108347450203570600835A5F
:105CC000260085072302F5029307F7FFB387FA0240
:105CD0005442C207C183B69703C9170083C70700A0
:105CE0008346C50022093369F90085476390F602AF
:105CF00033075703231006008149014A130B35016E
:105D0000931A070193DA0A0163E15907C167FD1786
:105D10006302F90C83570401637EF90A05094209FD
:105D20008346C4001359090123172401054703556D
:105D300004009305E400639FE6002315F100930738
:105D400020302316F100930780022314210123073A
:105D5000F1002C00EFB0FFA203458400B1659385EC
:105D600005B8EFA00FA95945BDA083D62400DC409B
:105D700083452401ED1613865900C206C1823E9662
:105D80005A85EFB0AFC705C9630C3A01C84003D6C6
:105D90002400B3053501529597A0FA1FE7804048CB
:105DA00083D724003E9A83D70400420A135A0A017B
:105DB00085072390F40083D72400BE99C20993D9A4
:105DC000090199B703474600A9476310F7028347C3
:105DD000450281CF0145F2506254D2544259B25922
:105DE000225A925A025B2161828083462401130960
:105DF000340137F506004A8689451305C5C1EFB061
:105E0000EFBF19C10545C1BF8346240137F5060020
:105E10004A868945130505C2EFB04FBE65F5834636
:105E2000240137F506004A868945130545C1EFB0C0
:105E3000EFBC69F98346240137F506004A86894597
:105E4000130505C0EFB08FBB55FD03C74400BD4728
:105E5000E3EAE7FAA56793874712B3D7E700858B94
:105E6000D5D38347440285072302F40203D92400D3
:105E700071BDB727002003C607B4B727002003A7CA
:105E8000078681476315F600814636858280BA868B
:105E900013078702835587FDE389A5FE850793F7DE
:105EA000F70FCDB7011106CE2EC6E13701CD8347DE
:105EB000A500B245138717006396E50093F707F82E
:105EC0002305F500F24005618280011106CE2EC641
:105ED0004D3705C5B24591C188C183478500130779
:105EE000E00F5D456388E7001307F00F014563830A
:105EF000E7005945F240056182800945E5BF41113F
:105F000022C42A84210506C626C24AC0EFF02FAD5E
:105F100083472400A51793F7D70F91EB0347C400DD
:105F200085476310F7061C4881443149A9E3FD57B2
:105F300023010400A304F400230204021305C40097
:105F40002244B2409244024961468145410117A36F
:105F5000FA1F67000334B38724033E95084509C53B
:105F600097A0FA1FE780401C850493F4F40F834741
:105F700044010848E3E1F4FE97A0FA1FE780C01A45
:105F80007DB7084C75F965B7411122C4416406C656
:105F900026C29307E4FF630CF500AA8491EDD13D7E
:105FA00019E51305F4FFF13519C123109500B2402E
:105FB000224492444101828085476394F504EFF0C6
:105FC0005FEB2A846DD5FD572310F50083478400CD
:105FD0001307F00F6384E7021307E00F638BE700FA
:105FE000834624000345940001475146A685EFF0FF
:105FF0000F9122852937FD572304F400230504005F
:106000007DB78947E395F5FA8545EF40902845F13E
:106010002685EFF01FE62A8455F951BF39C9034799
:1060200085009307F00F6306F704011122CC06CE1A
:106030002A848346250083550500034595000147C2
:106040005D46EFF0CF8B03472400E1476319F7006B
:10605000035504006C0023060100EFB01F92F957AE
:106060002304F4002285EFF09FE9F24062440561C9
:10607000828082809307F00F6306F706011122CC1D
:1060800026CA2A844EC6AE84B689AA8593068500A0
:10609000376505004AC852C43A89328A1305C501DA
:1060A000794606CEEFF0EF92A304240123014401C8
:1060B0002322340185C01305C4006244F2404249E2
:1060C000B249224AA685D2446146056117A3FA1F48
:1060D00067000315F2406244D2444249B249224A61
:1060E000056182808280B72700202382A786828074
:1060F0009547639CF506834745028546850723023D
:10610000F50283570600584203462600FD17C207D2
:10611000C1836318D6048A07BA9703C7170083C7D9
:1061200007002207D98F0357E50063F9E7044111FF
:1061300006C622C485072316F5002A849305C500E8
:1061400003550500EFB02FDA03458400B165938550
:1061500005B8EF901FEAB2402244D9473E8541017D
:106160008280C946B387D70245BF83464600294788
:1061700085476396E6000347450211C381473E8584
:1061800082809D476392F506834745028356E5006A
:1061900085072302F502835706005842FD178A0738
:1061A0003E978347170003470700A207D98F01478F
:1061B00063F6D704411106C622C485072A84231634
:1061C000F5009305C50003550500EFF0CFC5034565
:1061D0008400B165938505B8EF90BFE1B2402244D9
:1061E00059473A854101828083464600A9470547C1
:1061F0006396F60003474502133717003A858280FD
:10620000411122C406C626C2B5472A84639BF50401
:1062100083474502B28485072302F5020355050032
:10622000EFB06F9283D704001307F5FF014563C5F4
:10623000E7020357E400035504009305C400BA972E
:106240002317F400EFB0EFD803458400B1659385C0
:1062500005B8EF901FDA5945B240224492444101FB
:106260008280034746009D470545E317F7FE034537
:10627000440213351500CDB7C547639EF506835715
:10628000060003572600FD17B387E70203474502C0
:1062900005072302E5025842C207C1833E978347A0
:1062A000370003472700A207D98F41677D17639501
:1062B000E70081473E858280138717002316E5009B
:1062C0000357E500E3F7E7FE411122C49305C5003B
:1062D0002A840355050006C6EFB00FD90345840094
:1062E000B165938505B8EF90DFD0B2402244D9471D
:1062F0003E85410182808346460029478547E39BCE
:10630000E6FA0347450255F775B7011122CC26CAB4
:106310004AC852C406CE4EC683C7250015472A8AEE
:10632000AE8432843689639DE7043686A28526854D
:10633000EFF01FDCAA8955E985476318F40A034783
:106340004900A9476301F70203C594004A878546BF
:106350000146D285EFE0BFDA19E585454A85EFE0D1
:106360003FD21334150083C6240003C594000147AF
:106370006946D285EFE0BFD82685EFF05FB851A01F
:106380001D476398E7003686A2852685EFF07FDFFC
:1063900055B725476398E7003686A2852685EFF036
:1063A000DF8F49BF35476398E7003686A28526858B
:1063B000EFF01FE541B745476398E7003686A285B1
:1063C0002685EFF07FEBBDB75D47639FE70003C70E
:1063D000C50085473686A2852685631DF702EFF046
:1063E0006FBA8547631BF5048549A5476317F40217
:1063F000835709009DE30544E38709F6D947E39DE8
:10640000F9F62285F2406244D2444249B249224A16
:1064100005618280EFF02FC4E9B703C594004A8775
:10642000A2860146D285EFE09FCD71F5A2854A850F
:10643000EFE01FC513341500C1B70544D9B7397152
:1064400022DC06DE26DA4AD84ED652D456D283D77C
:1064500005001944B1E783C925002A89328A938748
:1064600059FE93F7D70FAE84DDE7B727002083C628
:1064700047861307F00F938A478619446382E60222
:10648000F5476394F904EFF0DF9EAA8921C1034622
:10649000A5000DCE93178601E18763DD0700014457
:1064A0002285F2506254D2544259B259225A925A19
:1064B00021618280F5454A85EFE0BFCC83C7A90002
:1064C00093E707F82385F900D9BF814983D64400B3
:1064D000904483C5140003C504003800EFB0EFCA30
:1064E0002A845DFD83C6240003C50A0038000146E6
:1064F000CA85EFE0DFC02A8445F5B24799C323007F
:106500000A0083C724007547E39BE7F8E38909F88D
:106510002385F90071B7EFF0DF95AA8A49D1854745
:106520006391F90A83D5440088443000EFA09FE3CB
:106530002A843DF503C72A00C54763F2E70ADD4711
:106540006301F70CB727002003C59A0083C797B3F0
:10655000639CA70A014403C72A008D47631FF70401
:106560008357810003D7CA0063F4E7002396FA003B
:1065700083D5CA004A85EFE0FFF6B727002083D70E
:10658000079A6D47637BF70283D5CA005D47637640
:10659000B7021387350091056349F7001307B00F61
:1065A000BE856374F7009305B00F1166C20513062C
:1065B0000629C1814A85EF8060475685EFF03F94F8
:1065C000C5B5834725001144E39C37ED5C41E38961
:1065D00007EC83D5440088443000829791BFB727E9
:1065E00002009387072AB3D7E700858BA1DF03C694
:1065F00024003400D6854A85EFF03FD12300AA005D
:1066000045B583A70A01DDB783C6240038000146DB
:10661000CA85EFE0DFAE2A841DFD83C52400280073
:10662000EFE01FA605D923000A0035B7011122CCDF
:106630003724002006CE26CA4AC84EC652C4930943
:1066400084B303C589009307800291653305F50281
:1066500093856570372900209304098697A0FA1F57
:10666000E780409E03C68900930780028145330678
:10667000F60288C097A0FA1FE780A0C19C404D4554
:10668000A1C3930484B3130909860144130A800249
:10669000FD5983C78400636DF40237650500130557
:1066A000E543EFE0FFE237650500130545EAEFA09B
:1066B0005FBB37650500130585F8EF40A034014541
:1066C000F2406244D2444249B249224A0561828082
:1066D000B30744030325090061468145050413748B
:1066E000F40F3E95231035012301050023143501D5
:1066F0002305050023020502310597A0FA1FE78054
:1067000040B941BF01458280B727002083C617B436
:10671000814763E5D70001473A8582802E8791053E
:1067200003D6C5FFE30AA6FE8507E5B70DCD83476F
:1067300025000547890793F7F70F6376F7024111A4
:1067400022C406C62A848355050003453500014747
:10675000F9465D46EFE0BF9AF9572311F400B240C5
:106760002244410182808280B727002003C717B4EA
:10677000FD56814763E3E70082802310D5002301A3
:10678000050085071105FDB70145828037160020F9
:106790001306B67F930700022300F6003717002088
:1067A000FD57230DF77E37170020A306F77E371716
:1067B00000202306F77E8545B7170020239CB77E6F
:1067C000B727002023930786B727002023A8078632
:1067D000B727002023A00788B727002023AA078611
:1067E000B7160020B7F706009386067F938707C188
:1067F000DCC2B727002023840786B71700209387C1
:10680000C77809472380E6002380E7002388E70054
:106810002380E7022388E70237F70600130747C003
:10682000D4C7D8DBB7F606000D47238CE702938662
:1068300006C037270020D4CB0327C78637F50600CC
:10684000B7F606001305C5C1938646C2C8C32384A4
:10685000B70023950700238CB700239D0700D0CFF6
:10686000D4D3238407022395070223A60702239D7E
:106870000702D8DFB7170020377705009387C77C5A
:106880001307479423A00700D8C323A407008280DE
:10689000411106C6EFF05FE711C503452500B24080
:1068A000410182800145E5BF411122C426C24AC090
:1068B00006C6AA842E893284EFF01FE511E94165EE
:1068C000CA857D15EFF05FE4C54711C5231095001B
:1068D000230185008147B2402244924402493E850B
:1068E0004101828029E789483547639316050111E4
:1068F00006CE22CC26CA034716000346060093C7DD
:10690000F7FF2207598EF18F32C68DE7C4452A84DE
:10691000A685EFF0FFF732460147630FA6002285F8
:106920006244F240A685D24405616FF0FFF72D471F
:106930003A85828013070008F2406244D2443A85C7
:106940000561828083C8050009486395080303A890
:1069500045008347180003480800A207B3E7070172
:10696000C2070D68C18713082890639507018947FE
:106970006FF05FF705458280011122CC37140020AB
:106980001304D47E0347040006CE26CA4AC84EC666
:106990009307F00F6300F704AA892945B2842E8972
:1069A000EF904F9205C99307100B2310F5002302B7
:1069B0000500231135012313250123149500AA8511
:1069C000034504006244F240D2444249B2490561A1
:1069D0006F904F9EF2406244D2444249B2490561F1
:1069E00082804111B727002026C2AE8483A5C786C6
:1069F00022C406C62A84EFF0BFE9098909C92285A5
:106A00002244B240A685924441016FF08F86B24085
:106A100022449244054541018280411122C426C28C
:106A20004AC006C6AA84130445001309850B835780
:106A300004009DC3084409C59790FA1FE780C06E03
:106A400022853146814597A0FA1FE7808084310472
:106A5000231A04FEE31D24FDB2402244FD57239077
:106A6000F4000249924441018280B727002003C606
:106A700017B4B727002003A7878781476315F6005F
:106A8000814636858280BA861307870B835587F443
:106A9000E389A5FE850793F7F70FCDB7B727002049
:106AA00083A7078889CB03D747006314A7008847CB
:106AB00082809C43C5BF01458280411106C6F93FD3
:106AC00009C50845B240410182800145E5BF011179
:106AD00026CA9384450022CC4EC606CE4AC852C46C
:106AE00056C25AC0268781490144814681473D45A7
:106AF0000356070055CED9E20354470083572700B9
:106B0000B286A297C207C18385093107E392A9FE25
:106B100025C82E8991659385457022859790FA1F27
:106B2000E78040522A8B29CD814A014A8C4485C591
:106B300003D6440033054B019790FA1FE780406E5F
:106B400083D7440088443E9A420A135A0A01979018
:106B5000FA1FE780605D63890A003146814526851A
:106B60009790FA1FE780E072850AB104E3E03AFDEE
:106B70002326690123148900054521A0630DD60051
:106B80000145F2406244D2444249B249224A924A03
:106B9000024B0561828003562700E313F6FE03567D
:106BA00047003294B2974204C2074180C183A9BF13
:106BB0000545E37835FDA9BFB727002083A74787A0
:106BC00099E30145828098470357A7006315A70002
:106BD0001385470082809C43E5B7411106C6E93F13
:106BE00011C503550500B240410182800145E5BF52
:106BF000411106C6D13711C503452500B2404101F8
:106C000082804145E5BF411122C42A842E8506C6F3
:106C1000C537AA8505462285EF307047954763053D
:106C2000F500BD476313F5002145B2402244410100
:106C300082804111B727002022C406C603A44787DB
:106C400081469387478729C018440356A7001840F8
:106C50006317A60285CA98C22E8581C9214693056D
:106C600044009790FA1FE780A05B22859790FA1F57
:106C7000E780804B0145B240224441018280A286D8
:106C80003A84D1B798C3C9BF0545F5B73727002067
:106C900083270788014613070788A9C703D8470039
:106CA0009443631CA802011106CE22CC26CA0DCA49
:106CB00014C2AA843E852E849790FA1FE780C046AE
:106CC0002C002685EFF0FFF601E519C0B2471CC085
:106CD000F2406244D244056182803E86B68775BF29
:106CE00014C3C1BF05458280411122C42A8409050D
:106CF00006C6EFE0CFCEFD57A301F400B240224418
:106D000041018280B727002003C717B4B7270020AE
:106D100083A7C7872A86050781463E8583D7070054
:106D20006388C700850693076500E3E8E6FE014532
:106D30008280411122C4416406C626C29307E4FF43
:106D4000630EF500AA8485E1EFF0DFFB01E913058E
:106D5000F4FFEFF03FFB19C123109500B24022442D
:106D600092444101828085476394F504EFF09FF9D6
:106D70002A846DD5FD572310F5008347240013079F
:106D8000F00F6384E7021307E00F638AE70003450F
:106D900034000147F9465146A685EFE04FB62285FB
:106DA000EFF09FF4FD572301F400230204007DB7A8
:106DB0008947E395F5FA8545EF30B04D45F12685D5
:106DC000EFF05FF42A8455F951BF1D71A6CACEC6F3
:106DD00086CEA2CCCAC8D2C4D6C2DAC05EDEAE8429
:106DE00083C52500F947AA896397F504EFF09FF161
:106DF0002A8411ED01442285F6406644D644464972
:106E0000B649264A964A064BF25B25618280834743
:106E100025000547890793F7F70FE37DF7FC034546
:106E200035000147F9460146CE85EFE04FAD22859A
:106E3000EFF09FEBC1B703AB0400B70700019387E6
:106E400007F037071200B377FB0013070710B28A69
:106E50000149638AE7022EC6EFF0DFEA2A89B245CC
:106E60001DC10346450005C293178601E187E3C3B0
:106E700007F84E85EFE0EFB08347490093E707F846
:106E80002302F90085BF371A00200347AA7F930722
:106E9000F00F130AAA7F1944E30FF7F4E147E3EC7C
:106EA000B7F493D71500FD1713973700B7E706001F
:106EB00093874762BA9703A80700E30E08F283ABF3
:106EC0004700E38A0BF2420B135B0B0163050B00D7
:106ED000C947E392F5F283D64400904483C5140079
:106EE00003C50400380802982A84E31605F02C082C
:106EF0004E85829B2A8421C983C71400E39D07EE37
:106F000083C72400230AA10039472308F1006399AD
:106F1000E70262478347170003470700A207D98F9C
:106F20000C084E852319F100EFA06FD9E30405EC9E
:106F300014080546D9454E85EFE08FC52A8465BD06
:106F400083578101F1BF83C624009147E384F6EAA9
:106F500003450A0038080146CE85EFE04F9A2A849F
:106F6000E31B05E883C524002808EFE06F9119C1F1
:106F700023800A009840B7070001938707F07D8FB0
:106F8000B707120093870710E306F7E6E30409E664
:106F900083C724002302F900B9BD011106CE2EC615
:106FA000EFF05FD601CD83474500B2451387170048
:106FB0006396E50093F707F82302F500F2400561B8
:106FC0008280B727002003A7478719E3014615A849
:106FD0001C4703D8A700636B050183584700B3869D
:106FE00008016355D5008146639416011843F1BF2B
:106FF0003E86C10703D3A7FF6317A30099C123905F
:107000000501328582808506C206C182F1BF3971D1
:1070100052D42E8A4ED69305E101AA89528522DCEC
:107020004AD856D206DE26DA328936C63AC4BE8A35
:10703000EFF03FF9054435C5AA840355E101394411
:10704000EFF0DFA539CD03284500630C0804224783
:10705000B246D6874A86A6854E8502982A8431E1B3
:107060009307E00F638FFA0203C704008947631A8E
:10707000F702D8408347170003470700A207D98FBC
:10708000C2070D67C18713072790639CE7008347FA
:10709000190003460900D285A2075D8E4E85EFF0E8
:1070A000BF8D2285F2506254D2544259B259225AAD
:1070B000925A21618280797122D4035425004ECEE8
:1070C000AA89228556CA06D626D24AD052CC5AC898
:1070D0005EC662C4AE8AEFF05F9901E92285EFA037
:1070E0001FDE594429E90144B9A003C78900854737
:1070F000AA840144631AF702AA8513858900EFF078
:107100001F9D29CD03D7640083D68400D04483D546
:10711000440003D52900E147EFF07FEFD9472A84E7
:107120006318F50223A604002685EFF01F8F49C0DF
:10713000D947E30AF4FA2285B250225492540259F4
:10714000F249624AD24A424BB24B224C456182809C
:1071500061DD83D744002390FA00F9B71389440016
:10716000014AB94B594C3D4B83550900D5DDE147E8
:1071700063067A010357C90011C3D9470357290091
:10718000835649000326890003D52900EFF03FE824
:107190002A846319850123240900050A3109E315AE
:1071A0006AFD59B77DD9835709002390FA00F5B7D6
:1071B00003D529002DB701112317C1009307E00F54
:1071C0001306E1000147894606CEEFF05FE4F24086
:1071D00005618280797122D42A840355850026D2E4
:1071E000AE849305210106D64AD0EFF09FDD6308F7
:1071F000050E834785002AC693F707028DCF0355F6
:107200002101EFF09F8BAA87B24501ED83578400DF
:1072100039452390F400B2502254925402594561EA
:107220008280035524004946829711C58357840004
:107230002390F400CDB7035924004A85EFF0FF8274
:1072400011ED41657D15EFF05F8219E583578400EC
:1072500025452390F400C1B72310250113074500ED
:107260008147BD46035607002DE63147B387E70245
:10727000130984003146CA8591073E959790FA1FFD
:10728000E78000FA3146CA8548089790FA1FE780E0
:1072900020F90356C4000355240041478146DD45CB
:1072A000EFE0EFA92ACE19E58357840045452390E6
:1072B000F40095B70C480356C4009790FA1FE78076
:1072C00020F6035524004C08EFA03FBB29D55945B3
:1072D00099B785073107E397D7F8254581BF05455D
:1072E000B1B7797122D42A840355850026D2AE84A1
:1072F0009305E1014AD006D63289EFF09FCC51C503
:107300008347850093F70702A9E703471401930712
:10731000200519E3834744008356A4005044835555
:107320008400035524000147EFF07FCEAA8721E9AE
:107330008347140199E703552400EFA03FAFD947D5
:1073400011E18147B2502254925402593E85456161
:1073500082802AC60355E101EFF02FF6AA8705C9FE
:10736000B2450355240049468297AA8759DD035741
:1073700084002390E4000347140161F7E1B7594703
:10738000E317E5FE230009006DBF8547CDB7B94778
:10739000F9BF397122DC4AD84ED652D406DE26DA3D
:1073A000AA892E8A32C63689EFF0DF95094415C5C1
:1073B000834725001307E00FAA845D44638FE7002D
:1073C0001307F00F5944639AE700324605E2D2856D
:1073D0004E85EFA0BFB22A8415CD2285F2506254AB
:1073E000D2544259B259225A2161828003550A006F
:1073F0009305E101231F0100EFF0BFBC0355E1013C
:10740000EFF00FFFAA8505464E85EF3040482A84ED
:107410005DDDE1B79307F00FE301F9FC3765050087
:10742000938624007946A6851305C572EFD07FDACE
:10743000A38124015DB73971B727002026DA83A420
:10744000478752D45AD05ECE62CC06DE22DC4AD8C0
:107450004ED656D266CA2A8BAE8B328C368A99E0CB
:107460008149B9A0804483DC44000149835AA400C7
:10747000631499018440E5B78357A400A28963F897
:10748000670105094209135909014104D5B7E3EA27
:10749000FBFE630C0A00834504004840D2866286E6
:1074A0003AC6EF90BFD5324769DD19C323105701A3
:1074B000F25062544E85D2544259B259225A925ACD
:1074C000025BF24B624CD24C2161828003D70500F3
:1074D00083D62500854763E9E60439C7411183C691
:1074E000450026C237F506009384550022C426863F
:1074F0002E841305C5C1894506C6EF903FD0C1470C
:1075000011CD8346440083552400035504000147F0
:107510002686EFF05FF2814711E1A947B24022448D
:1075200092443E85410182803E8582802E860355AD
:10753000060083D52500854763E2A50205C1834681
:10754000460041110147150606C6EFF0DFEE814700
:1075500011E1A947B2403E85410182803E8582808B
:107560002E860355060083D52500854763E2A502D4
:1075700005C18346460041110147150606C6EFF0D6
:107580009FEB814711E1A947B2403E8541018280CE
:107590003E85828039714ED683D7250083D9050078
:1075A00006DE22DC26DA4AD852D456D25AD05ECE33
:1075B00062CC66CA6AC863E037198547638E0914CE
:1075C000416BAE8A2A8A2314010002C60144014994
:1075D0007D1B894B054CC94C054D83D52A000147BD
:1075E000814601464E8523130100EFF0DFE4AA84B3
:1075F0006300051209EC13072002930661005A8606
:1076000095455285EFD0BFF32A84630805120357CE
:10761000810083C7040045C70347A100630CA70787
:1076200041476385E7022C005285EFA00FCE09CDBC
:1076300034001546D9455285EFD09FD511C5324546
:107640009790FA1FE78040AE8147F9A083D7A40046
:107650004146130524002300F40083D7A400A1832E
:10766000A300F400CC409790FA1FE78060BB490468
:10767000835781008507C207C1832314F10063F992
:10768000270983D7A400638567098509C20993D9AF
:107690000901A1B7E39977F983D7A4000946130537
:1076A00024002300F40083D7A400A183A300F400E6
:1076B000CC409790FA1FE780A0B6110455BF22C6B0
:1076C0000359610003C7A4001305240063827703F4
:1076D00033599903230571012300E40083D7A400E3
:1076E0004146A183A300F400CC401379F90FA5BF54
:1076F000230581012300E40083D7A4001359290046
:107700001379F90FA183A300F4000946CC4055B7C3
:107710008357810089FBA947F2506254D2544259E1
:10772000B259225A925A025BF24B624CD24C424DF1
:107730003E85216182808547C5B7C547F1BFB72720
:10774000002003C7E788854763F3E706011122CCD1
:1077500026CA4AC806CE2A843289AE84EFF08FDA70
:1077600001C9034725009307E00F5D456308F70053
:10777000631C0900A6852285EFA02FF5F240624424
:10778000D24442490561828003D504009305E1009B
:1077900023170100EFF0FF820355E100EFF04FC522
:1077A000AA8505462285EF30800E69D5C1BF5945AF
:1077B000828013F7050201C7B2856FF0CFC4411173
:1077C00026C24AC006C622C413F98500AA846317DC
:1077D0000900139785016187635D0702328536844E
:1077E000EFF00FC1AA8505466313090001462685FF
:1077F000EF30E00901E90145B240224492440249D8
:107800004101828083479400E5DB83478400E5F7EC
:10781000E5B793F72500E5F30D45F9BF7971AE861D
:1078200022D42A8403D506009305E10106D636C684
:10783000EFF02FF909CD83458500B2460356E101EB
:107840002285EFF01FF7B250225445618280054532
:10785000DDBF13F7050201C7B2856FF0CFBA411142
:1078600022C426C206C693F485002A8491E41397A5
:1078700085016187635007023285EFF06FB7AA85F3
:10788000054691E0014622852244B24092444101DE
:107890006F20F07F93F72500014591E30D45B2403D
:1078A00022449244410182807971AE8622D42A8496
:1078B00003D506009305E10136C606D6EFF06FF05A
:1078C000B24601CD834585000356E1012285EFF0E4
:1078D0005FF8B2502254456182800545DDBF797161
:1078E00026D2AA840355A500C16722D44AD04ECE21
:1078F00006D623170100FD173284B6890149630DAE
:10790000F500050583C60400D04042051307E100D9
:107910004181EFF05FB22A8983C60400D04037F579
:10792000060089451305C5C1EF905F8D1DC503D4C1
:10793000A4002285EFF06FAA09C57D142A944204A1
:1079400041806384090023908900B25022544A8503
:1079500092540259F2494561828083C60400D040A6
:1079600037F506008945130505C2EF903F8961F19F
:1079700083C60400D04037F506008945130505C0CD
:10798000EF90DF8719C9E30609FA8357E100E39214
:1079900087FA0354A9007D145DB703D4A40055B73A
:1079A000397122DC26DA4AD84ED652D456D25AD071
:1079B00062CC06DE5ECEBE8983C785002A8AAE848D
:1079C000C18B328C36843A89C28A468B9DE783CB41
:1079D00004008947638BFB046285EFF02F8C1DC187
:1079E00083280500638008025A88D6874E87CA8696
:1079F0002286A6855285829839A03285EFF0EF8BDA
:107A0000AA8711ED3945F2506254D2544259B25905
:107A1000225A925A025BF24B624C216182802946C3
:107A2000A6855285829745D5F9BFD8408347170070
:107A300003470700A207D98FC2070D67C1879306C6
:107A400007906384D72263CEF60693062780638E61
:107A5000D70C63C1F60213070780E3CFE7F62D4585
:107A6000E39309FADC4403C60700CC432310C900A2
:107A7000228569A213073780E390E7F62D45E3944A
:107A800009F885472310F900DC44814583C70700C6
:107A90002300F40003D5A400050542054181EFF061
:107AA0004FD2835709006317051291072310F9007D
:107AB00011468145130514009780FA1FE780607D09
:107AC00029A2930627906383D71863CED712930613
:107AD0003790638CD71813074790E39FE7EE2D4547
:107AE000E39309F2DC441D472310E90003C70700B4
:107AF0002300E40003C71700A300E40003D7270016
:107B00002301E40003D727002183A301E40003C776
:107B100047002302E40003D76700A302E40083D7F1
:107B20006700A1832303F4004DA02D45E39D09ECDC
:107B3000DC446C0083C9170003C70700A209B3E93E
:107B4000E90011472310E90083C707004E85230091
:107B5000F400DC4483C71700A300F400EFF06FC605
:107B6000AA8435C50356C100C1659306E100FD1521
:107B70008329C500EFF0BFD619ED83C60400D040BD
:107B800037F506008945130505C2EF902FE701E59B
:107B9000FD572317F10003C7090089476310F70257
:107BA00083A549000946130544009780FA1FE78022
:107BB00020678357090089072310F9008357E100E4
:107BC0002301F400A183A301F40001452DBD231777
:107BD0003101EDB7034705008907BA972310F90073
:107BE0008357A500A300F4008357A500A1832301B8
:107BF000F400034605004C41130534009780FA1F3A
:107C0000E7800062D9B7C8449780FA1FE780806B8D
:107C100093170501C1832A871D45E3E637DF639982
:107C2000F90023100900CC4403560900CE9589B50C
:107C30004207B3863A01418363C7E600B387374101
:107C40002310F900CDB723105901F1BF2D45E39C56
:107C500009DACC445285EFE0BFC323107901230039
:107C6000A4002181A300A4008DB72D45E39D09D870
:107C7000DC442310790183C707002300F400DC44AF
:107C800083C71700A300F40089B71D71CAC82A89E9
:107C900003552500A2CCCEC6D2C4D6C2DAC05EDE61
:107CA00062DC66DA6ED686CEA6CA6AD8AE8AEF9055
:107CB0008FE9130CF5FF93170C01B72B0020C1833C
:107CC0002A8A814913840B8F3EC6372B0020B72C9C
:107CD0000020C16D8357C90063F6F9008357040083
:107CE00063CC87010355290093850B8FEFA08F8804
:107CF0002A8D15CD594D25A8832789001397190082
:107D00009305E101BA9783C4170083C70700A20453
:107D1000DD8C2685EFF0EFAAAA8515E923909A005D
:107D20004840054D09C59780FA1FE780E03FF640BF
:107D300066446A85D6444649B649264A964A064B61
:107D4000F25B625CD25C425DB25D2561828032484A
:107D50008348490083A60C870356E1010355290097
:107D6000814713076B86EFF0BFC32A8D13880C87FA
:107D700009C523909A00484075B75C4085E70355D4
:107D80002900514781461386FDFFBD45EFD02FFBEB
:107D9000B727002048C01388078709E523909A0079
:107DA000454D71B78357040003576B8693046B8668
:107DB0003E976347470113C7F7FF52972390E400AC
:107DC000484003D60400832508003E958509978026
:107DD000FA1FE780E0448357040003D70400C20978
:107DE00093D90901BA972310F400EDB5397122DC5B
:107DF0002A840355250006DE26DA4AD84ED652D408
:107E00005AD05ECE62CC66CA2E8B56D26AC8EF902C
:107E10008FD32A8A8346C4008355A4000355840067
:107E200078001306D400130CBAFF651AEFF0AFE028
:107E3000420A37290020AA898144135A0A01B72B24
:107E40000020B72C00201309098F6386090463D42E
:107E50008405938A0C878348440083A60A0003564E
:107E6000C100035524005288814713876B86CE8555
:107E7000138D6B86EFF0DFB215C5814A0356C10042
:107E80008355A4004E859306E100EFF05FA5AA8913
:107E9000639D0A065DF9E5E08357840029452310B8
:107EA000FB0089A083570D0003560401E317F6FC7D
:107EB00083A50A0048489780FA1FE780A04355DD54
:107EC00083274900A1E303552400416645478146C5
:107ED0007D169D45EFD0AFE605E583578400454507
:107EE0002310FB00F2506254D2544259B259225A24
:107EF000925A025BF24B624CD24C424D216182801D
:107F00002322A90083DAA90095BF83274900A697F9
:107F10002380570193871400139707018327490093
:107F2000418393DA8A00BA9723805701138724008C
:107F30008326490093873400420791044183C20796
:107F4000C204C183C180369711CD8356E10023005E
:107F5000D70003274900BA970357E1002183238004
:107F6000E700E5B5FD562300D70003274900BA977F
:107F70002380D7000DB703552400B7250020898042
:107F80002398958E9385058FEF90DFC421DD5945A9
:107F900091BF411122C406C693F705012A84328598
:107FA00085C3EFE0FFC4AA8505462285EF20300E89
:107FB00095476305F500BD47631DF502214515A8EA
:107FC00093F7450099CBEFE0BFC20546AA8522850D
:107FD0002244B24041016F20900B93F7050489C7FA
:107FE000EFE01FC10146DDB713F51500133515008D
:107FF0000605B24022444101828079714AD04ECEBA
:1080000052CC06D622D426D22A8AAE89014983D7F9
:1080100049006364F9000145A1A083A70900131476
:108020001900930414003387970003470700A297B1
:1080300003C5070022079305E100598DEFE07FF8A3
:1080400005E983A7090005453E9403470400238002
:10805000E70083A70900BE9403C70400A380E700DC
:10806000B250225492540259F249624A45618280C8
:10807000834585000356E1005285EFF09FF105C16D
:1080800083A709003E94034704002380E70083A7E9
:108090000900BE9403C70400A380E700D1B7050917
:1080A000420913590901A5B7011122CC2A8403D52D
:1080B00005009305E10006CEEFE0BFF001CD83455A
:1080C00085000356E1002285EFF0BFECF2406244E8
:1080D000056182800545DDBF1D71CAC82A89035527
:1080E000250086CEA2CCA6CAD2C4D6C2DAC05EDE35
:1080F00062DC66DA2E8ACEC66AD86ED6EF90AFA45E
:108100002AC68346C9008355A9000355890078080B
:108110001306D900EFF02FB2B247B7240020416B0D
:10812000938AA7FFC20AAA8B014493DA0A01372C6B
:108130000020B72C00209384048F7D1B63860B18CE
:108140000356C10183C58B0003552900EFF07FE47E
:10815000AA8D631605168348490083A60C8703562B
:10816000C101035529005688814713076C86DE85B7
:10817000EFF01F83AA8D93096C86138D0C87631013
:10818000051429C003D7090083D72400110763977A
:10819000E7003247A2976D1763CAE706B7250020AC
:1081A0009387058F03D72700035529009385058FF3
:1081B0003354E40223908700EF905FBFAA8D15C16E
:1081C000D94D05A003552900494781465A86C54522
:1081D000EFD0EFB6C8C015E583D7AB00C54D23106F
:1081E000FA00F64066446E85D6444649B649264AAA
:1081F000964A064BF25B625CD25C425DB25D2561E1
:10820000828083D7090091072391F400DC4003D7D3
:10821000AB009306E101A2972380E70093071400C7
:1082200013970701DC4041835E85BA9703D7AB0003
:1082300021832380E7000356C1018355A900EFF095
:108240000FEAD440130724000356E101420741839B
:1082500036972300C700D84093073400C207C18374
:10826000BA970357E101AA8B110421832380E70009
:10827000C8404204418003D6090083250D002295A1
:1082800063950B029780FA1FE78080F983D7090076
:108290003E9442044180E31304F083578900231085
:1082A000FA00E3900DF4A94D2DBF9780FA1FE780E7
:1082B00020F783D709003E944204418041B583D71B
:1082C000AB002310FA00C1BF814DF1B75D71A6C2AA
:1082D000CAC0AA840359850003552500A2C44EDEF6
:1082E00052DC5AD85ED662D466D286C656DA6AD0D6
:1082F0006ECE2E8BEF902F85930BD5FF7115131A31
:108300000501B72900200144135A0A01372C002027
:10831000B72C00209389098F6359741583C6C40054
:1083200083D5A4001307E1001386D4004A85EFF03B
:108330008F902A8D630B05120359A5008345850094
:108340000356E10003D52400EFF0BFC46314051207
:1083500083C8440083A60C870356E10003D524009C
:108360005288814713076C86EA85EFF06FE3930D1F
:108370006C8613880C87631F050E1DC883D70D00FC
:1083800003D729008907630CF706B7250020138758
:10839000058F8357270003D524009385058F335419
:1083A000F40223108700EF90BF8C15C5594525A016
:1083B00003D5240041664D4781467D16A545EFD083
:1083C0000F98B727002023A2A900138807871DE173
:1083D00023102B014545B640264496440649F259E0
:1083E000625AD25A425BB25B225C925C025DF24DF1
:1083F0006161828083D70D0089072391F90083D7BB
:108400000D00A29763D3770783A749000357AD00F8
:10841000930A2400A2972380E70005049317040120
:1084200003A44900C183C20A3E948357AD0083254B
:10843000080093DA0A01A1832300F40003A5490090
:1084400003D60D0056959780FA1FE78060DD03D4B0
:108450000D00C167FD17569442044180E30EF9EA0E
:10846000050942091359090145BD294519FC231085
:108470002B0195B76DDC11BF8357050081E7894754
:108480003E858280411126C2444122C406C64AC0AC
:1084900083C60400D0402A8437F5060089451305B9
:1084A000C5C1EF80BFD519C9834724002547E5170B
:1084B00093F7F70F6377F702E14729A883C6040013
:1084C000D04037F506008945130505C2EF801FD35C
:1084D00061FD8947B2402244924402493E854101F0
:1084E0008280371900208356897F85471309897F49
:1084F000F5D2035704003697C166E3CDE6FC9165DB
:108500009385257031459780FA1FE780A0B3AA8430
:10851000CD4769D1314681459780FA1FE78060D702
:10852000835704008355090001460147B386E500DF
:10853000C206C182636BF702AE97C207C18319C23C
:108540002310F90023A004002146A28513854400CE
:108550009780FA1FE780C0CCB72700209387478712
:10856000984311EF84C38147B5B7504013154700B6
:1085700005072A962315D60005464DBF3E871C43A6
:10858000F5FF04C381BF011106CE22CC26CA4AC81A
:1085900009E98944F240624426854249D244056192
:1085A00082802AC62A84280036892314B100230534
:1085B000C100EFF07FECAA8471FDE30D09FC835745
:1085C000A400E1DB91659385557031459780FA1FD2
:1085D000E78040A715C58357A40023200500232466
:1085E00025012312F500B7270020938707889843B9
:1085F00001E788C345B73E871C43F5FF08C359BF51
:10860000CD4449BFB72700209387878603C707005B
:1086100015E305472380E700058909CDB71600203B
:10862000371500209386C67C414691451305C578D1
:108630006FF07FF501458280B7170020A386A77EE3
:108640008280C167FD176315F5002E856FE0CF911D
:10865000411106C6EFE04F8B11C5FD572310F50001
:1086600023010500B2404101828001114AC806CEB3
:1086700022CC26CA85472A896393F5044A85EFE010
:10868000CFBE39E9C16437F606009385F4FF1307BE
:10869000E1008946130646C00545EFE0DFD92A848C
:1086A000FD140DC44C444A85EFF0BFF90356E100B8
:1086B00022858146A685EFF08FA22A84DDB78947FF
:1086C0006396F5008545EF20C03C4DD9F2406244E9
:1086D000D244424905618280EFE02FB465B70111B1
:1086E00026CAB7240020938484B322CC03C5940007
:1086F0003724002013048487B72700203727002061
:1087000006CE4AC84EC62320040023AE0786232681
:10871000078649C91389C7879307200C3305F502DB
:108720009165938515709309C786190542054181A6
:108730009780FA1FE780009103C694009307200CEE
:1087400081453306F60208C019069780FA1FE780B4
:1087500040B41C4003C7940081459386870B7D5528
:1087600063ECE5069306800BB306D7020146FD5580
:108770000507B6972320F900BE862390B600A38193
:10878000B6002381B6002382060005069906E3663B
:10879000E6FEF9562390D70099463307D702BA97D9
:1087A00023A0F900377505001305A5DCEFC0FFD243
:1087B000377505001305A5F9EF805FAB3775050028
:1087C000130525D3EF200024F2406244D2444249ED
:1087D000B2490145056182802394A6F41386C6F44C
:1087E00023100600232406003106E31BD6FE850570
:1087F0009386860BB5B7411106C622C42A84EFC002
:108800000FB7EFD0BFF8B71700202386877EB727B2
:10881000002003A5C786EFD03FF5B7170020238DB2
:10882000877E2244B240378505001305A5664101C5
:108830006F20401D93970501C18763D30734B71795
:10884000002003C5C77E797122D45AC806D626D225
:108850004AD04ECE52CC56CA2E8BEF70AFAD2A8482
:1088600029C9034705009307000B6311F704B724D8
:108870000020854793840487A304F1009C402315BE
:108880000100A9E7EF00007F91659385357097702F
:10889000FA1FE780207B88C015E98347910099C7BC
:1088A0008345440013058400EFD0EFA52285EF70C7
:1088B0004F9CB250225421653345AB00925402596B
:1088C000F249624AD24A424B45618280372A0020EF
:1088D0006146814513050A8F9780FA1FE780609BE8
:1088E00003494400894793040A8FD289930A0A8F67
:1088F0006314F906EF0000782390A40003552400C8
:1089000093050A8FEF90EF9B0357240083D7040051
:108910008356840011ED63E4F6002314F4008355BC
:1089200084003A85EFC01FBC2285EFC07F8EB5B7AB
:1089300063E4F6002314F40083578400D94593863A
:10894000098F0D463A852390FA00EFC07FA48D452C
:1089500061DD1385098FD1A09947631AF902930548
:10896000A1002285EFF08FC8AA845DDDD947639608
:10897000F40E0509035524001379F90FD9459386A0
:10898000098F4A86EFC0DFA0CA8559DDD9B7A14754
:108990006318F9009305A1002285EFF03F93E9B732
:1089A000A947631FF906035584006C00EFE06FE1EF
:1089B0002A89630D05140355240041669306E100DE
:1089C00055477D16AD45EFC09FB7C8C0AA8649C1BF
:1089D000834844000358E1000356C10003552400B6
:1089E000814713070A8FCA85EFE09FFBAA84631EA5
:1089F000050E0355240093050A8FEF904FAD0DD55A
:108A00000355240093060A8F2D46D945EFC05F9881
:108A1000E30C05F0AD4513050A8FEFD0CF8E29B7D3
:108A2000B147631BF90E035584006C00EFE06FD96A
:108A3000AA8469CD0355240041669306E100594795
:108A40007D16B545EFC0BFAF23A2AA00AA8629E9CB
:108A500083578400C5442315F10003471400D14710
:108A6000E304F7EC83474400035524009385098F02
:108A70002380FA008357A10023829A002391FA00F1
:108A8000EF80FFA3E30205EA035524009386098FD4
:108A90000546D945EFC0DF8FE30805E8854555BD9C
:108AA000834844000358E1008357A4000356C100E3
:108AB00003552400A68513070A8FEFE07FEEAA84F2
:108AC0000DE50355240093050A8FEF900FA6E30DE3
:108AD00005E403552400D94593060A8F3546EFC0B7
:108AE0003F8BB545E30205E4ADB5D9476393F40088
:108AF000814403A54A009770FA1FE780E062E3858E
:108B000004E2835784002315F10081BF835784005A
:108B100085442315F10091B7B9476318F90093050F
:108B2000A1002285EFF06F9681B5C1476318F90067
:108B30009305A1002285EFF02FDA3DB5C947631AEE
:108B4000F900130691009305A1002285EFE06FF96B
:108B500021BDD947631DF9009305A1002285EFE0EF
:108B60006FE7AA84E31405E0A304010075BBE147A5
:108B7000E31CF9DA9305A1002285EFE0CFD3EDB332
:108B800001458280EDC2011152C42E8A854522CC56
:108B90004EC656C206CE26CA4AC8AA8AB6893284AA
:108BA000EF10306FD1471DC5B727002037270020B1
:108BB00083C7C7888346D788814419E0B684BE86B8
:108BC000372700200327478893974400BA9763ED1F
:108BD000D400D547F2406244D2444249B249224AC5
:108BE000924A3E85056182803E89C10703D727FFEF
:108BF00009C7850493F4F40FD9BF25C09565938503
:108C000025C0130500029770FA1FE780A0432326B2
:108C1000A90061D113060002814593840404977072
:108C2000FA1FE7800067231199002300090023132E
:108C300059011DC437270020834794000326C7A984
:108C40002304F900118C8327C90011841180238E1D
:108C5000870023A029018147B5BF23260900F1B76A
:108C600023044901FDB785473E858280B727002050
:108C700083C5C788B727002003A747888147639526
:108C8000F50081463685828003562700BA8619C2D0
:108C9000E30AA6FE850793F7F70F4107CDB7B7277D
:108CA000002003C6C788B727002003A7478881474D
:108CB0006315F60081463685828083552700BA8683
:108CC00089C583454700E388A5FE850793F7F70F1D
:108CD0004107F9BFB727002083C5F788B7270020D1
:108CE00003A7C7A981476395F50081463685828031
:108CF00003560700BA8619C2E30AA6FE850793F752
:108D0000F70F4107CDB7B727002003C8D788B7278B
:108D1000002083A7478801476315E8008146368510
:108D2000828003D62700BE8619CA03D6670063185F
:108D3000A600D04709C603562600E302B6FE050783
:108D40001377F70FC107C9BF411122C4404526C29E
:108D500006C6AA8415C0484409C59770FA1FE78063
:108D6000A03C484809C59770FA1FE780E03B228580
:108D70009770FA1FE780403B2685414681459770F2
:108D8000FA1FE7800051B2402244FD57A384F4004B
:108D9000924441018280011122CC2A84035525008E
:108DA00006CE2EC6EF10F018324622858145EF0020
:108DB000B07222856244F24005616FF0FFF80DC584
:108DC00003572500411122C406C62A8411CBDD4574
:108DD000EF00707422852244B24041016FF0DFF64B
:108DE000B2402244410182808280411126C2B146B4
:108DF0009304C5FFB386D402B72700201387C7AA00
:108E000006C622C436978356A7006398B602484325
:108E10000DC51384C7AA9307F00F6306F6008347B6
:108E20000500639CC7009770FA1FE780E02FB147E9
:108E3000B387F402A29723A20700B24022449244CF
:108E400041018280411122C42E8426C24946AA844F
:108E50008145228506C69770FA1FE7808043A5C02A
:108E600083C7C40113974700B727002083A7C7A96A
:108E7000BA9703D707002310E40003D7270083D74E
:108E800067002311E400372700200357A788231227
:108E9000E40003D704002313E40003D724002314C1
:108EA000E40003D744002315E40003D7640023162D
:108EB000E40003D784002318F4002317E400B24031
:108EC0002244924441018280B727002083C5C7888D
:108ED000B727002003A8C7A9B727002003A6478803
:108EE000014781476394E5003E8582808346060002
:108EF00081CE544691CA83C6C6019206C2966315B6
:108F0000D500850793F7F70F05071377F70F41068D
:108F1000D1BF130600643386C50293069500AA8567
:108F2000379505001305E5DB6F708FB7411122C43B
:108F300006C62A8403459500EF700FD1FD57A304A0
:108F4000F400B240224441018280011122CC4AC87F
:108F50004EC652C456C25AC006CE26CA2A89AE8907
:108F60000144372A0020B72A00201D4B8347DA88A6
:108F70006365F40463990902B7290020372A0020A9
:108F8000930AF00F83C7C9886367F4061144A144AC
:108F90002285050442041306F00FCA854180EFF0D4
:108FA000DFE4E31794FEF2406244D2444249B249FE
:108FB000224A924A024B0561828083A74A88931411
:108FC0004400BE9483C704009DC383D764006390AC
:108FD00027036396690103D52400EF108075268569
:108FE0004E868145EF00504F2685EFF0FFD50504F2
:108FF0001374F40FA5BF83274A8893144400BE94CA
:1090000083C704009DC383C794006380570383D73D
:109010006400639C27012685EFF05FF12685D1452A
:10902000EF00704F2685EFF03FD205041374F40F64
:1090300091BF41677917630BE502411122C406C64F
:1090400085472A846399F50022852244B2408145F0
:1090500041016FF09FEF89476396F5008545EF105A
:1090600050237DD1B24022444101828082809D45BF
:109070006FF0BFEDB727002003D5A7888280B72700
:10908000002003C78788011106CE2317A1002316ED
:10909000B10085476318F70070009305E1000545AE
:1090A000EF509019F24005618280A947631CF604D5
:1090B00083C7150003C70500A207D98F2310F50049
:1090C00083C7350003C72500A207D98F2311F500F8
:1090D00083C7550003C74500A207D98F2312F500A7
:1090E00083C7750003C76500A207D98F2313F50056
